:1080000000000120197D02009151020091510200EF
:1080100091510200915102009151020000000000B4
:10802000000000000000000000000000915102006C
:1080300091510200000000009151020099C6010018
:1080400091510200915102009151020091510200A0
:108050009151020091510200915102009151020090
:108060009151020091510200915102009151020080
:108070009151020091510200915102009151020070
:108080009151020091510200915102009151020060
:108090009151020091510200915102009151020050
:1080A0009151020091510200915102009151020040
:1080B0009151020091510200915102009151020030
:1080C0009151020091510200915102009151020020
:1080D0009151020091510200915102009151020010
:1080E0009151020091510200915102009151020000
:1080F0009151020085E1010091510200915102006D
:1081000091510200D1DF0100915102009151020012
:108110009151020085D70100915102009151020056
:1081200091510200915102009151020091510200BF
:1081300091510200915102009151020061FA010037
:108140003DED010091510200915102009151020058
:10815000915102009151020091510200915102008F
:1081600091510200196402009151020091510200E4
:10817000915102009151020091510200915102006F
:10818000915102009151020091510200915102005F
:10819000915102009151020091510200915102004F
:1081A000D1EC010091510200915102009151020065
:0C81B00091510200915102009151020017
:10840000FFFFFFFFFFFFFFFFFFFFFFFF7EF9FFFF03
:1084200010B5054C237833B9044B13B10448AFF3AE
:1084300000800123237010BD0012FF1F0000000008
:10844000ECB2020008B5034B1BB103490348AFF37C
:10845000008008BD000000000412FF1FECB2020003
:1084600010B516F097FC064B00221A70054B1B68DE
:108470009847054B9B69BDE810405B69184700BFF2
:10848000340BFF1FB001FF1FD89D0200431E2DE9D2
:10849000F0471546072B00F24D82DFE813F0080085
:1084A0000E000E0050006A00BB00FA00B301FFF797
:1084B000D7FF47F6A8532B603FE0A34BA34C0228FD
:1084C0000ABFA14699461C46A14BDF68A9F10409E1
:1084D000043C4FF0FF364FF000084FF0010A3B68B4
:1084E000D9F804001B6998473B686068DB689847C7
:1084F0003B6854F8040F5B6998473B6859F8040FD0
:108500005B6A984718B90AFA08F326EA03063B683B
:1085100020689B6998473B68D9F800005B6A9847D8
:1085200018B10AFA08F326EA030608F10108B8F1BF
:10853000110FD4D1C6F310062E60002021E029606F
:1085400003291DD8DFE801F0020A0E12804BDB6917
:108550001B681A88322353431B14ACE77C4BDB693E
:108560005B68F6E77A4BDB699B68F2E7794B1B693E
:10857000A1E7012929601DD04EB226B102292FD0D2
:108580000220BDE8F087724BDD68D5E90030DB687A
:1085900068309847D5E90030DB6888309847D5E9DE
:1085A00000305B6968309847D5E900305B698830F6
:1085B0009847C2E7664BDC68D4E90030DB68C83016
:1085C0009847D4E90030DB68A8309847D4E90030F8
:1085D0005B69C8309847D4E900305B69A830E7E7A9
:1085E0005B4BDC68D4E90030DB6800F5A470984789
:1085F000D4E90030DB6800F5B4709847D4E9003066
:108600005B6900F5A4709847D4E900305B6900F518
:10861000B470CDE70129296026D04EB2CEB102292F
:10862000AED14B4BDC68D4E90030DB6800F5A470B8
:108630009847D4E90030DB6800F5B4709847D4E976
:1086400000305B6900F5A4709847D4E900309B695D
:10865000DDE73F4BDD68D5E90030DB6888309847BF
:10866000D5E900301B699DE7394BDC68D4E900305F
:10867000DB68C8309847D4E90030DB68A8309847F9
:10868000D4E900305B69C8309847D4E900309B6971
:10869000A4E7296000295FD001297FF471AF2C4B3A
:1086A000DC68D4E90030DB6800F5D9609847D4E98C
:1086B00000309B6900F5D9609847D4E90030DB6849
:1086C00000F5DD609847D4E900309B6900F5DD6076
:1086D0009847D4E90030DB6800F5E1609847D4E9B9
:1086E00000309B6900F5E1609847D4E90030DB6811
:1086F00000F5E5609847D4E900309B6900F5E56036
:108700009847D4E90030DB6800F5E9609847D4E980
:1087100000309B6900F5E9609847D4E90030DB68D8
:1087200000F5ED609847D4E900309B6900F5ED60F5
:108730009847D4E90030DB6800F5F1609847D4E948
:1087400000309B695BE000BF445EFF1F805FFF1F3E
:10875000D89D0200340BFF1F774BDD68D5E9003050
:10876000DB6800F5D9609847D5E900305B6900F512
:10877000D9609847D5E90030DB6800F5DD6098479F
:10878000D5E900305B6900F5DD609847D5E9003038
:10879000DB6800F5E1609847D5E900305B6900F5DA
:1087A000E1609847D5E90030DB6800F5E56098475F
:1087B000D5E900305B6900F5E5609847D5E9003000
:1087C000DB6800F5E9609847D5E900305B6900F5A2
:1087D000E9609847D5E90030DB6800F5ED6098471F
:1087E000D5E900305B6900F5ED609847D5E90030C8
:1087F000DB6800F5F1609847D5E900305B6900F56A
:10880000F160D5E6296000294AD001297FF4B8AE8D
:10881000494BDC68D4E90030DB6800F5B16098476B
:10882000D4E900309B6900F5B1609847D4E9003085
:10883000DB6800F5B5609847D4E900309B6900F526
:10884000B5609847D4E90030DB6800F5B960984717
:10885000D4E900309B6900F5B9609847D4E900304D
:10886000DB6800F5BD609847D4E900309B6900F5EE
:10887000BD609847D4E90030DB6800F5C1609847D7
:10888000D4E900309B6900F5C1609847D4E9003015
:10889000DB6800F5C5609847D4E900309B6946E085
:1088A000254BDD68D5E90030DB6800F5B1609847FD
:1088B000D5E900305B6900F5B1609847D5E9003033
:1088C000DB6800F5B5609847D5E900305B6900F5D5
:1088D000B5609847D5E90030DB6800F5B960984786
:1088E000D5E900305B6900F5B9609847D5E90030FB
:1088F000DB6800F5BD609847D5E900305B6900F59D
:10890000BD609847D5E90030DB6800F5C160984745
:10891000D5E900305B6900F5C1609847D5E90030C2
:10892000DB6800F5C5609847D5E900305B6900F564
:10893000C5603DE6042024E6D89D020038B5064C0B
:108940002368C31AB3F5FA7F054604D3034B9B692A
:108950009B699847256038BD1C12FF1FD89D0200F7
:108960003A4B3B4ADB685B6803F59471116003F195
:108970004801516003F18801916003F1C801D160A1
:1089800003F58471116103F5B471516103F5D4717C
:10899000916103F5F471D16103F50A71116203F578
:1089A0001A71516203F52A71916203F53A71D1622D
:1089B00003F54A71116303F55A71516303F56A7146
:1089C000916303F57A71D16303F585611164214ADE
:1089D00003F10801116003F12801516003F16801FE
:1089E000916003F1A801D16003F1E801116103F581
:1089F000A471516103F5C471916103F5E471D16112
:108A000003F50271116203F51271516203F52271CF
:108A1000916203F53271D16203F54271116303F57E
:108A20005271516303F56271916303F5727103F53D
:108A300081631364084BD16301221A70074B084A03
:108A40005A65084ADA65084A9A657047D89D020057
:108A5000445EFF1F805FFF1F340BFF1F885EFF1FF8
:108A60008D840000618400003D8900007047022071
:108A700070470220704770477047022070470220FD
:108A800070470220704701207047704702207047EE
:108A900070478369124A134910B5C3E98122124B0A
:108AA000C365124BC361C0E90A1311490362C0E9EF
:108AB0000C13104B8364104BC364104B8363C0E9E9
:108AC00010330F4B436600230E4CC3660E4B0F4A08
:108AD0008265C463C0E914140266C0E91C3310BD8A
:108AE000878A00006F8A00006D8A0000738A000088
:108AF0007B8A0000778A0000798A00007F8A000064
:108B00008B8A0000838A00008D8A0000918A000011
:108B1000704700BF0A480B4B0022012110B44FF0F0
:108B2000FF3480F88C201A8083F81012C0E92141AC
:108B3000C0F89030C0F8802010BC7830FFF7A9BF93
:108B4000885EFF1F2C12FF1F084A094800234FF0C0
:108B5000FF314FF0010C138082F810328261C0E9BE
:108B6000031C03758360FFF794BF00BF4C14FF1F05
:108B7000885EFF1F00230649184611F8012B02F0FA
:108B800003029A4002330E2B40EA0200F5D17047EF
:108B90006C16FF1F0549431E063011F8012B02F029
:108BA000030203F8012F8342F7D170476C16FF1FB1
:108BB000074B1A7802705A7842709A788270DA7885
:108BC000C2701A7902715A7942719B798371704728
:108BD0006C16FF1FF8B5094B094D0A4FDE680024DB
:108BE00015F8011B7A6C33681059DB6901F0030139
:108BF000043498471C2CF3D1F8BD00BFD89D020067
:108C00006C16FF1F0800FF1F064A0723013B00F0F8
:108C1000030113F0FF0302F8011B4FEA9000F5D1A6
:108C2000D8E700BF6C16FF1F014B586AECE700BF86
:108C30000800FF1F0549431E063013F8012F02F0FC
:108C40000302834201F8012BF7D1C3E76C16FF1F23
:108C5000074B02781A7042785A7082789A70C278FC
:108C6000DA7002791A7142795A7182799A71B1E790
:108C70006C16FF1F024B0022C3F88020704700BF14
:108C8000885EFF1F10B50348144617F0BAFC206039
:108C900010BD00BFA016FF1F10B50F4C01462046A7
:108CA00017F01BFD002016F027FE6F21204617F05D
:108CB000A8FCC0F30061002016F0C2FE012016F0EF
:108CC0001BFE7F21204617F09CFCBDE81040C0F33E
:108CD0000061012016F0B4BEA016FF1F014817F076
:108CE00082BC00BFA016FF1F012808B503D816F0EC
:108CF000EBFD002008BD0820FCE7012808B503D8DB
:108D000016F0BCFD002008BD0820FCE70021F4E7B8
:108D10004942F2E7F1E70129F8B506461D46084643
:108D200000F2CA82A32A00F0938143D8072A00F0F8
:108D3000EC8022D8032A00F0C1800AD8012A00F072
:108D4000B18040F2A480002E40F0B48016F06EFF97
:108D5000A0E0052A00F0C38040F2B68020248C40B9
:108D600044F01004E4B22146B848002E40F0BF8021
:108D700017F047FCC0F304208CE0322A00F0FC809E
:108D80000AD81C2A00F0DE801D2A00F0F080082A94
:108D900000F0D08004267EE08C2A00F0F980A22A20
:108DA00000F03E81332AF5D1002E40F0ED8016F020
:108DB00089FF6FE0AB2A00F0008232D8A72A4FEA81
:108DC000011000F0BE811AD8A52A00F06A8140F295
:108DD000548140F06C00C4B221469C4817F011FC4D
:108DE000214600F480479948002E40F09F81002FD3
:108DF00000F0968117F005FCC0F302104AE0A92AA2
:108E000000F0BE8140F2A98140F06D00C4B221465D
:108E10008E48002E40F0C88117F0F3FBC0F303200A
:108E200038E0B32A00F009821BD8AD2A00F0E781B0
:108E3000C0F0D881AE2AADD10C0144F06D04E4B28B
:108E400021468248002E40F0EF8117F0DAFB001433
:108E500000F07F0310F0400018BF6FF07F00184350
:108E600018E0B52A00F00B82C0F0FC81B82A00F0AF
:108E70000E82CE2A8ED1002E8CD1080140F06F01D7
:108E8000C9B2724817F0BDFBC0F3090002E026B971
:108E900016F0ACFE28603046F8BD196816F014FDD7
:108EA0000026F8E716B916F091FEF3E7196816F0F8
:108EB0002DFEF5E7196816F0E1FCF1E7002E7FF4CE
:108EC00069AF16F0A3FEE5E716B916F0CFFEE1E7AD
:108ED00019680029B8BF494216F034FEE0E716B918
:108EE00016F0B4FED6E7196816F0DBFFD8E717F0E6
:108EF00088FB2B681B0203F4F85320F4F8521A4342
:108F00002146524817F06FFBCAE720248C4044F0FA
:108F10001004E4B221464D4826B917F072FB00F068
:108F20001F00B7E717F06DFB2B6820F01F0203F05E
:108F30001F03E4E7002E7FF42DAF16F023FDC0F3EE
:108F40000010A7E70C0144F06C04E4B221463F484E
:108F500026B917F056FBC0F380409BE717F051FB92
:108F60002B689B0403F4802320F48022C7E7002EA3
:108F70007FF410AF0020A4E716B916F095FE89E73C
:108F8000197816F0FBFD8BE7196816F007FE87E7E6
:108F900056B9080140F06C0101F0FC012B4817F0B4
:108FA00030FBC0F3036075E71B68102B32D00EDC7A
:108FB000022B2BD005DC012B17D04FF0FF332B6099
:108FC0006EE7042B24D0082BF7D105230EE0402BAD
:108FD00022D003DC202BF0D1032307E0802B1DD00F
:108FE000B3F5807FE9D1002300E00823040144F0B9
:108FF0006C04E4B22B602146144817F002FB2B6886
:109000001B0603F0706320F0706278E70723EDE73A
:109010000623EBE70423E9E70223E7E70123E5E77B
:109020000C0144F06C04E4B22146084826B917F05C
:10903000E8FAC0F3C1302DE717F0E3FA2B68DB0341
:1090400003F4C03320F4C03259E700BFA016FF1F5D
:109050000C0144F06C04E4B22146984826B917F09C
:10906000D0FAC0F3803015E717F0CBFA2B689B03DA
:1090700003F4804320F4804241E740F06C00C4B226
:1090800021468E4826B917F0BCFAC0F3003001E73C
:1090900017F0B7FA2B681B0303F4805320F48052B7
:1090A0002DE740F06C00C4B22146844817F0A9FABD
:1090B0002146074600F4804380487EB923B117F06B
:1090C000A0FAC0F3C310E5E617F09BFAC0F3021351
:1090D00017F4006018BF43F0080370E743B117F0BE
:1090E00090FA2B68DB0103F4F06320F4F06206E7EA
:1090F00017F087FA2A68120120F0700002F070025F
:10910000024321466D4817F06EFA21466B4817F06E
:1091100078FA2B681B0203F4006320F40062EEE689
:1091200017F06FFAC0F3C3102860B9E6002FD6D04D
:1091300017F067FA2B681B0103F0700320F0700230
:10914000DDE640F06C00C4B221465C48002E4ED1F2
:1091500017F057FA00F00F009CE640F06D00C4B223
:109160002146564826B917F04CFAC0F3C03091E6B4
:1091700017F047FA2B68DB039BB220F40042BEE6EF
:1091800040F06D00C4B221464C4826B917F039FAB8
:10919000C0F341307EE617F034FA2B685B0303F42A
:1091A000C04320F4C042AAE617F02BFA2B681B023A
:1091B00003F4706320F47062A1E60C0144F06D04C6
:1091C000E4B221463D4826B917F01BFAC0F341101E
:1091D00060E617F016FA2B685B0103F0600320F0DD
:1091E00060028CE60C0144F06D04E4B2ACE717F0C9
:1091F00008FA2B6820F00F0203F00F037FE60C0142
:1092000044F06D04E4B221462C4826B917F0F9F970
:10921000C0F300603EE617F0F4F92B681B0603F07C
:10922000807320F080726AE617F0EBF92B681B045C
:1092300003F4FE0320F4FE0261E60C0144F06C042A
:10924000E4B221461D4826B917F0DBF9C0F34040CF
:1092500020E617F0D6F92B685B0403F4003320F402
:1092600000324CE6002E7FF495AD080140F06F010E
:10927000C9B2124817F0C5F9C0F304400AE616B99E
:1092800016F004FD06E6196816F06AFC08E60C0103
:1092900044F06C04E4B22146084826B917F0B1F94D
:1092A000C0F34030F6E517F0ACF92B685B0303F42C
:1092B000005320F4005222E60826ECE5A016FF1F1A
:1092C00007B5019201AB02460120FFF724FD03B070
:1092D0005DF804FB1346024600201CE5014817F028
:1092E000E4B900BFA016FF1F022804BF0C4B93F87F
:1092F000F00038B90B4BDB681B685B690A4AD2F88F
:1093000094021847012809D1054B93F8F030012B3E
:1093100004D1044BDB681B689B69EFE7704700BF13
:10932000885EFF1FD89D0200A016FF1F70B50020A9
:10933000FFF7DAFF0C4B0D4CDD68D4F894022B6874
:109340009B6898472B68D4F8A4029B6898472B68C1
:10935000D4F8A8029B68984716F05EFD044BBDE860
:1093600070405B68184700BFD89D0200A016FF1F21
:10937000E00AFF1F0346052B10B5084614460BD024
:1093800006D8022B06D316F09DFC2060002010BDED
:10939000182BF8D00420FAE716F0B0FCF5E738B542
:1093A0000D46044620B916F031FC2860204638BD31
:1093B0000820FCE7022810B5144611D0032817D066
:1093C000012819D10D4B0E4ADB68D2F8A4021B68A4
:1093D0005B6A9847003018BF01202060002010BD54
:1093E000064B074ADB68D2F8A8021B685B6AF0E705
:1093F000084616F0C7FAF0E70420F0E7D89D02000F
:10940000A016FF1F012838B504460D4608D816F0EF
:10941000DDFB2B68C11829602046BDE8384063E4B5
:10942000082038BD38B5002016F0F0FB08B1002048
:1094300038BD012016F0EAFB05460028F7D10C4C98
:10944000204617F01FF90B4816F06EFC2B46D4F897
:109450008C22D4F88412284616F0BCFA01202B4640
:10946000D4F89022D4F8881216F0B4FA0120DFE77D
:10947000A016FF1FA0860100022806D3052801D9E7
:10948000182802D100201060704704207047034B59
:10949000D3F8B0320846DB6811461847A016FF1F04
:1094A0002DE9F0415A4C5B4D5B4FD4F890205B4B5B
:1094B0000121284617F0C9F8FE68736803F16802B5
:1094C000C5F8942203F1E802C5F8A82203F58472D6
:1094D000C5F8A42203F5A472C5F88C2203F5B47272
:1094E00003F59470C5F8882203F5C47203F502737E
:1094F000C5F8AC323368C5F89022DB68C5F8840241
:1095000098473368D5F88C02DB6898473368D5F8FC
:109510008802DB6898473368D5F89002DB68984783
:109520003368D5F89402DB6898473368D5F8AC0205
:10953000DB6898473B693A4803F11402C5F8B0224A
:10954000D5F8AC229A6116F0EFFB0023D5F88C22F7
:10955000D5F88412184616F03DFAD5F88812D5F8D9
:1095600090220023012016F035FAD4F890302D4ACD
:10957000C3F804222C4AC3F8082201221A802B4B7C
:10958000C4F89C302A4BC4F898302A4BC4F8943065
:10959000294BC4F8A030294BC4F8B430284BC4F888
:1095A000B030284BC4F8A430274BC4F8A830274B60
:1095B000C4F8C430264BC4F8C030264BC4F8D030B1
:1095C000254BC4F8CC30254BC4F8C830244BC4F824
:1095D000DC30244BC4F8D83032224FF48F73C4E906
:1095E0002132214BC4F8D430204BC4F8E83002209B
:1095F0001F4B84F88C00C4F8EC301E4CFFF774FE4F
:10960000236898470021A3680846BDE8F041184741
:10961000885EFF1FA016FF1FD89D0200947F0200E6
:10962000A086010025940000DD920000FB8C000064
:10963000158D0000118D00000D8D0000D5920000E9
:10964000C1920000E98C000005940000DD8C000050
:10965000858C0000998C0000B59300009F9300005A
:10966000E9920000758C00002D93000079940000B1
:1096700075930000E00AFF1F014B1046DB6B184793
:109680000800FF1F034B10B51B6C14469847206061
:1096900010BD00BF0800FF1F062873B504460E4624
:1096A0007BD8404D68462B6B013C98472B46042CD9
:1096B00004D8DFE804F00866696C6F009DF800309C
:1096C000336000200BE09DF80120E978914208D139
:1096D0009DF80200297B884203D10020306002B04F
:1096E00070BD1979914206D19DF80200597B8842DC
:1096F00001D10123E4E75979914206D19DF8020096
:10970000997B884201D10223DAE79979914206D107
:109710009DF80200D97B884201D10323D0E7D97993
:10972000914206D19DF80200197C884201D10423A0
:10973000C6E7597A914206D19DF80200997C884289
:1097400001D10523BCE7997A914206D19DF8020028
:10975000D97C884201D10623B2E7197A914206D119
:109760009DF80200597C884201D10723A8E7D97AE5
:10977000914214D19DF802201B7D9A420FD10823FB
:109780009EE79DF803309BE79DF8043098E79DF82D
:10979000053095E79DF8063092E704209FE71020FA
:1097A0009DE700BF0800FF1F07B5034B68461B6B12
:1097B000984703B05DF804FB0800FF1F70B5002058
:1097C000FFF7F2FF1E4B1F4CDD68206B2B689B6878
:1097D00098472B68E06A9B6898472B68E0689B680D
:1097E00098472B68A0689B6898472B6860689B68BF
:1097F00098472B6820689B6898472B68A0699B68EE
:1098000098472B68E0699B6898472B68A06A9B681B
:1098100098472B6860699B6898472B68206A9B680B
:1098200098472B68606A9B6898472B6820699B68FB
:10983000984716F0F1FA044BBDE870405B68184792
:10984000D89D02006019FF1FE00AFF1F10B50446F3
:1098500018B916F039F8204610BD0820FCE710B5FD
:10986000044618B916F00AF8204610BD0820FCE797
:109870000021F4E74942F2E7F1E7062873B505460F
:109880000C465DD8022903D901285BD10F2959DC88
:109890002D4E6846336B98473346052D06D8DFE8D2
:1098A00005F0030B4346494C8DF800406846DB6ADF
:1098B0009847002002B070BD082CF7D8DFE804F00C
:1098C000050C11161B20252A2F00F2788DF8012097
:1098D000327B8DF80220E9E732798DF80120727B26
:1098E000F7E772798DF80120B27BF2E7B2798DF853
:1098F0000120F27BEDE7F2798DF80120327CE8E778
:10990000727A8DF80120B27CE3E7B27A8DF80120FB
:10991000F27CDEE7327A8DF80120727CD9E7F27AA8
:109920008DF80120327DD4E78DF80340BEE78DF835
:109930000440BBE78DF80540B8E78DF80640B5E771
:109940000420B7E71020B5E70800FF1F002015F03E
:10995000D3BF38B5154618B1012807D0042038BD4B
:10996000084616F00FF828600020F8E7094B0A4D6A
:10997000DC680A4B606800F59470D8616B6C5861C4
:109980002368DB6898476A6C236850699B6998472D
:10999000EAE700BFD89D02000800FF1F6019FF1F03
:1099A00038B50D46044648B916F010F92B68C118B1
:1099B0002960204615F088FF204638BD0820FCE7C6
:1099C00070B5054616460C4600295DD10B2810D807
:1099D00006283CD202282ED004D808B3012825D06E
:1099E000042421E004282ED029D9084616F02EF9A7
:1099F0001FE013280CD80E283CD20C282FD00D289D
:109A0000EED1224B224ADB68106B1B685B6A2CE0AC
:109A1000322835D03328E3D1084616F053F908E050
:109A200016F0E4F82C463060204670BD084616F06B
:109A3000CDF83060F8E7084616F0F8F8F9E7084680
:109A400016F0E4F8F5E7084616F010F9F1E70828F3
:109A5000C6D1084615F096FFC0F30010E9E70B4B9E
:109A60000B4ADB68D06A1B685B6A9847003018BFF6
:109A70000120DEE70E381146C0B2FFF70DFED3E736
:109A8000084616F011F9D4E70824CDE7D89D020066
:109A90006019FF1F30B585B0054601920C460029BC
:109AA0006ED10B2812D8062846D2022837D004D807
:109AB00048B301282CD004242EE0042834D00528F3
:109AC000F9D11146204616F0ECF925E013280FD8FD
:109AD0000E2845D20C2836D00D28ECD142F2107356
:109AE0009A42E8D8274B91B29B682046984713E0EA
:109AF000332837D08C283AD03228DCD1D1B2204656
:109B000016F03CF808E0114615F0DEFE2C4603E0A6
:109B10001146204615F0FAFF204605B030BD11462B
:109B2000204615F0ABFEF7E782EAE271A1EBE271A5
:109B3000204616F007F8EFE706381146C0B2FFF7E7
:109B40009CFE0446E8E7104B1049DB68C86A1B68B6
:109B5000154612B15B699847DEE79B699847D5E7E0
:109B60000E38EAE71146204616F018F8D4E701A9A6
:109B70000120FFF791FD064B04469B6B02A8EAE724
:109B80000824C9E7E00AFF1FD89D02006019FF1FE3
:109B90000800FF1F6E4B2DE9F041DE686D4C7068C8
:109BA0006D4F00F5E473236300F5D473E36200F5B1
:109BB0002273E36000F52A73A36000F51A736360F3
:109BC00000F50273236000F55A73A36100F5527328
:109BD000E36100F16803A36200F5A473636100F51B
:109BE0006A73236200F572736362336800F59470E0
:109BF000DB682061984733686069DB6898473368A1
:109C0000206BDB6898473368E06ADB689847336805
:109C1000206A1B6998473368606A1B6998477B6CA8
:109C2000E2681A60A2685A6062689A602268DA6024
:109C3000A2691A61E2695A61A26A9A6100257A6C86
:109C400033685059DB6898477A6C336850599B6980
:109C5000043598471C2DF2D1404DD5F890304FF087
:109C6000000883F800804FF4003016F05DF8D4E966
:109C700004124346404615F0ADFE44F620614046CE
:109C800015F060FF46F2A811404616F00AF9344B71
:109C9000C5F89C30334BC5F89830334BC5F8943039
:109CA000324BC5F8A030324BC5F8B430314BC5F853
:109CB000B030314BC5F8A430304BC5F8A830304B2C
:109CC000C5F8C4302F4BC5F8C0302F4BC5F8CC3089
:109CD0002E4BC5F8D0302E4BC5F8DC30012385F86B
:109CE0008C3002202B4BC5F8D430FFF75DFD404689
:109CF00015F08CFF10B1284B9B78ABB1BB6A98472D
:109D00004FF4003016F010F80023D4E9041218467E
:109D100015F060FE44F62061002015F013FF46F2B6
:109D2000A811002016F0BDF83368206BDB68984757
:109D3000206B1A4C0423437533681B6898472368CB
:109D400098470021A3680846BDE8F041184700BFC6
:109D5000D89D02006019FF1F0800FF1F885EFF1FCB
:109D60005F980000799800007598000071980000D5
:109D7000C1990000959A00004D980000A19900003B
:109D80007996000085960000539900004D990000D7
:109D9000A9970000BD970000340BFF1FE00AFF1FCA
:109DA0001B4B70B5DD681B4C2B68A0685B6998473E
:109DB0002B6820689B6898472B6860689B68984769
:109DC0002B68206A9B6898472B68606A9B68984755
:109DD0002B68E0689B6898472B6820699B689847C8
:109DE0002B6860699B6898472B68A0699B689847B7
:109DF0002B68E0699B6898472B68A0689B68984728
:109E000016F00AF8044BBDE870405B68184700BFC5
:109E1000D89D0200A019FF1FE00AFF1F10B51446CD
:109E2000062805D8DFE800F0062523343F444E001D
:109E3000042010BD146844F620639C424ED8284B81
:109E4000284ADB68106A1B6842F210718C42DB6999
:109E500094BF00210121984742F21173B4FBF3F142
:109E600003FB1141204B89B29B68002098470020DA
:109E7000DFE71B4B2468DA68D2E9003000F5F470A4
:109E80001CB1DB6900219847F1E79B689847EEE732
:109E9000134B1168DB68134A1B681069DB690031DA
:109EA00018BF0121EFE7084615F06CFD2060DEE7E2
:109EB0000B4B0C4ADB6858681B6800F59470106106
:109EC000DB68E3E7064B074ADB6858681B6800F667
:109ED0000801D1605B6900F55270D7E71020A8E750
:109EE000D89D0200A019FF1FE00AFF1F10B503480C
:109EF000144616F070FC206010BD00BFC45FFF1F49
:109F000010B5094C0146204616F003FD002015F05F
:109F1000F3FC6F21204616F05EFCBDE81040C0F354
:109F20000061002015F08CBDC45FFF1F014816F0D2
:109F300044BC00BFC45FFF1F10B5044618B915F03C
:109F4000C3FC204610BD0820FCE710B5044618B934
:109F500015F094FC204610BD0820FCE70021F4E732
:109F60004942F2E7F1E770B504461D460E46002966
:109F700040F04E85A52A00F08F8256D8172A00F0AF
:109F8000478126D8042A00F0E8800ED8012A00F084
:109F9000AD80002A00F09E80022A00F0B280032AE1
:109FA00000F0BA800424204670BD072A00F0068124
:109FB00007D8052A00F0DF80062A00F0E780042495
:109FC000F1E7082A00F01181152A00F01781042416
:109FD000E9E7322A00F0B28113D81B2A00F063812E
:109FE00007D8182A00F039811A2A00F04481042485
:109FF000D9E71C2A00F06F811D2A00F08681042415
:10A00000D1E7A22A00F0008207D8332A00F0A1810C
:10A010008C2A00F0A9810424C5E7A32A00F00C8251
:10A02000A42A00F021820424BDE7B42A00F0B583FD
:10A0300024D8AA2A00F018830CD8A72A00F0CE82D0
:10A04000C0F08682A82A00F0E082A92A00F0F482FB
:10A050000424A8E7AD2A00F0518307D8AB2A00F00A
:10A060001B83AC2A00F0308304249CE7AE2A00F066
:10A070005D83B32A00F07983042494E7BB2A00F0BF
:10A08000278413D8B82A00F0C88307D8B52A00F06F
:10A090009083B62A00F09A83042484E7B92A00F05A
:10A0A000D683BA2A00F0ED8304247CE7C02A00F0AE
:10A0B0006C8407D8BC2A00F03384BF2A00F04684A1
:10A0C000042470E7CC2A00F07B84CE2A00F096842A
:10A0D000042468E720B9002015F088FD286062E7B5
:10A0E0001968002015F0F0FB00245CE718B915F0A2
:10A0F0006DFD286057E71968304615F007FD3446B6
:10A1000051E718B915F092FD28604CE71968002056
:10A1100015F0B4FB002446E7002840F07C8415F0DD
:10A12000C3FD18B915F072FD28603CE7204615F014
:10A13000C9FD12210646B14816F04DFBC0F31302CB
:10A140007A20D317A6FB00011DF02CFC00F11303AD
:10A15000262B98BF0020286025E718B915F086FD4A
:10A16000286020E719680029B8BF4942304615F039
:10A17000E9FC344617E718B915F068FD286012E7C6
:10A180001968002015F08DFE00240CE710219B4873
:10A190002CB916F020FBC0F30420286003E716F06A
:10A1A0001AFB2B681B0203F4F85320F4F8521A43ED
:10A1B0001021924816F001FB0024F4E610218F488C
:10A1C0002CB916F008FB00F01F002860EBE616F033
:10A1D00002FB2B6820F01F0203F01F031A4310211B
:10A1E000864816F0EAFA3446DDE6002840F0168488
:10A1F00015F0C8FBC0F300102860D4E6002800F07A
:10A2000010841A687D48112116F0D7FA0024CAE696
:10A210007B4E80B91521794816F0DDFA48B14FF030
:10A22000807393FBF0F0B042A8BF30462860002452
:10A23000B9E63046FAE71B686BB14FF0807292FBCB
:10A24000F3F2B242A8BF32462A6015216B4816F0DD
:10A25000B4FA0024A7E63246F6E728B93321674866
:10A2600016F0B9FA28609EE61A686448332116F0A1
:10A27000A4FA002497E66C2160482CB916F0ABFADA
:10A28000C0F3804028608EE616F0A5FA2B689B0488
:10A2900003F4802320F480221A436C21574816F0DF
:10A2A0008CFA00247FE66C2154482CB916F093FAFE
:10A2B000C0F3C040286076E616F08DFA2B68DB0408
:10A2C00003F4002320F400221A436C214B4816F0BB
:10A2D00074FA344667E638B90146484816F07BFA06
:10A2E000C0F3400028605EE60021444816F073FA8F
:10A2F0002B685B0003F0020320F002021A430021E6
:10A300003E4816F05AFA00244DE6002840F08C83AF
:10A3100015F0D8FC12210646384816F05CFAC0F356
:10A3200013027A20D317A6FB00011DF03BFB00F1BE
:10A330001303262B98BF0020286034E618B915F0C7
:10A34000B3FC28602FE61978304615F017FC344628
:10A3500029E618B915F0B6FC286024E61968002033
:10A3600015F01CFC00241EE650B96C21234816F0A1
:10A3700032FA4FF48073C0F3036003412B6012E69E
:10A380001B68102B35D00FDC022B2ED006DC012BE6
:10A3900018D04FF0FF332B60102404E6042B26D096
:10A3A000082BF6D105230EE0402B24D003DC202B14
:10A3B000EFD1032307E0802B24D0B3F5807FE8D1D1
:10A3C000002300E008232B606C210C4816F003FAF0
:10A3D0002B681B0603F0706320F070621A436C2137
:10A3E000064816F0EAF90024DDE50723EBE706232B
:10A3F000E9E70423E7E70223E5E700BFC45FFF1FA7
:10A40000FFFF0F000123DEE76C21BB482CB916F0DB
:10A41000E2F9C0F3C1302860C5E516F0DCF92B681D
:10A42000DB0303F4C03320F4C0321A436C21B2487A
:10A4300016F0C3F93446B6E56C21AF482CB916F0D6
:10A44000CAF9C0F380302860ADE516F0C4F92B6876
:10A450009B0303F4804320F480421A436C21A648F6
:10A4600016F0ABF900249EE56C21A3482CB916F038
:10A47000B2F9C0F30030286095E516F0ACF92B680E
:10A480001B0303F4805320F480521A436C219A4832
:10A4900016F093F9002486E56C21974804BB16F06A
:10A4A0009AF910F480464FF06C01934805D016F0ED
:10A4B00092F9C0F3C310286075E516F08CF96C2191
:10A4C00004468D4816F087F92205C0F3021002D425
:10A4D0002860002467E540F008002860344662E503
:10A4E00016F079F910F480444FF06C0182480ED0D8
:10A4F00016F071F92B68DB0103F4F06320F4F062CD
:10A500001A436C217C4816F058F934464BE516F096
:10A5100062F96C21784816F05EF92A68120220F47C
:10A52000006002F4006202436C21734816F045F9A2
:10A530006C21714816F04FF92B681B0103F0700372
:10A5400020F070021A436C216B4816F036F92AE5A8
:10A550006C216948ECB916F03EF910F480444FF0D4
:10A560006C01654806D016F036F9C0F30210286079
:10A57000002418E516F02FF96C2106465E4816F007
:10A580002AF93305C0F3C310A2D540F008002860B3
:10A5900009E516F020F910F480444FF06C0156489C
:10A5A0000ED016F018F92B681B0103F0700320F091
:10A5B00070021A436C21504816F0FFF80024F2E4B0
:10A5C00016F009F92B68DB0103F4F06320F4F06264
:10A5D0001A436C21484816F0F0F8E4E46C21464830
:10A5E0002CB916F0F8F800F00F002860DBE416F044
:10A5F000F2F82B6820F00F0203F00F031A436C21CE
:10A600003D4816F0DAF83446CDE46D213A482CB9CD
:10A6100016F0E1F8C0F3C0302860C4E416F0DBF8AF
:10A620002B68DB039BB220F400421A436D213248B1
:10A6300016F0C3F80024B6E46D212F482CB916F0AB
:10A64000CAF8C0F341302860ADE416F0C4F82B68B6
:10A650005B0303F4C04320F4C0421A436D21264833
:10A6600016F0ABF800249EE46D2123482CB916F0B7
:10A67000B2F8C0F30320286095E416F0ACF82B681C
:10A680001B0203F4706320F470621A436D211A48B0
:10A6900016F093F8344686E46D2117482CB916F06D
:10A6A0009AF8C0F3411028607DE416F094F82B6806
:10A6B0005B0103F0600320F060021A436D210E4835
:10A6C00016F07BF800246EE46D210B482CB916F0CF
:10A6D00082F800F00F00286065E416F07CF82B6823
:10A6E00020F00F0203F00F031A436D21024816F009
:10A6F00064F8002457E400BFC45FFF1F6D21BD480C
:10A700002CB916F068F8C0F3006028604BE416F02E
:10A7100062F82B681B0603F0807320F080721A43E6
:10A720006D21B44816F049F834463CE46D21B14837
:10A7300064B916F050F8001400F07F0310F04000E8
:10A7400018BF6FF07F00184328602CE416F043F820
:10A750002B681B0403F4FE0320F4FE021A436D2150
:10A76000A44816F02AF800241DE46C21A1482CB955
:10A7700016F031F8C0F34040286014E416F02BF8CE
:10A780002B685B0403F4003320F400321A436C217D
:10A79000984816F012F8002405E4002840F047819C
:10A7A0006F21944816F017F8C0F304402860FFF7B3
:10A7B000FABB20B915F06AFA2860FFF7F4BB1968F4
:10A7C000002015F0CDF90024FFF7EDBB8A4E88B9C3
:10A7D0001421884815F0FFFF50B14FF0807393FBB0
:10A7E000F0F0B042A8BF304628600024FFF7DBBB82
:10A7F0003046F9E71B6873B14FF0807292FBF3F2B9
:10A80000B242A8BF32462A6014217A4815F0D5FF1B
:10A810000024FFF7C8BB3246F5E76C21754834B910
:10A8200015F0D9FFC0F340302860FFF7BCBB15F02E
:10A83000D2FF2B685B0303F4005320F400521A4349
:10A840006C216C4815F0B9FF3446FFF7ACBB6C21A6
:10A85000684834B915F0BFFFC0F303502860FFF714
:10A86000A2BB15F0B8FF2B681B0503F4700320F49E
:10A8700070021A436C215F4815F09FFF0024FFF718
:10A8800092BB5D4E88B913215A4815F0A4FF50B110
:10A890004FF0807393FBF0F0B042A8BF30462860C1
:10A8A0000024FFF780BB3046F9E71B6873B14FF017
:10A8B000807292FBF3F2B242A8BF32462A601321A3
:10A8C0004C4815F07AFF0024FFF76DBB3246F5E7E0
:10A8D0007021484834B915F07EFFC0F30720286086
:10A8E000FFF761BB15F077FF2A68120220F47F4062
:10A8F00092B2024370213F4815F05FFF31463D4858
:10A9000015F069FF2B68002B20F0040218BF042308
:10A910001A433146374815F050FF3446FFF743BB22
:10A92000702134482CB915F056FFC0B22860FFF7EB
:10A930003ABB15F050FF2A7820F0FF000243702147
:10A940002C4815F03AFF0024FFF72DBB40B97021C9
:10A95000284815F040FFC0F301402860FFF723BBF3
:10A960001B68032B66D87021224815F034FF2B6832
:10A970001B0403F4403320F440321A4370211D4875
:10A9800015F01BFF0024FFF70EBB7021194834B9E6
:10A9900015F021FFC0F380402860FFF704BB15F0DD
:10A9A0001AFF2B68002B20F4802218BF4FF480235D
:10A9B0001A4370210F4815F000FF3446FFF7F3BA31
:10A9C00070210C4834B915F006FFC0F3015028601F
:10A9D000FFF7E9BA15F0FFFE2B681B0503F44013DF
:10A9E00020F440121A437021024815F0E6FE0024BC
:10A9F000FFF7D9BAC45FFF1FFFFF0F00E8B96F214F
:10AA00000F4815F0E8FEC0F309002860FFF7CBBA45
:10AA10000824FFF7C8BA0424FFF7C5BA0424FFF7D7
:10AA2000C2BA0424FFF7BFBA0424FFF7BCBA042457
:10AA3000FFF7B9BA1024FFF7B6BA0424FFF7B3BA88
:10AA4000C45FFF1F07B5019201AB02460120FFF76B
:10AA50008AFA03B05DF804FB134602460020FFF7B4
:10AA600082BA014815F03DBFC45FFF1F08B5002042
:10AA700015F0CCF810B1094B987870B1084815F072
:10AA800019FF4FF4003015F04FF90649002318461E
:10AA9000D1E9001214F09EFF012008BD340BFF1F06
:10AAA000C45FFF1FA019FF1F022804BF0B4B93F8C0
:10AAB000F00030B90A4BDB681B685B69094A906893
:10AAC0001847012809D1054B93F8F030012B04D128
:10AAD000034BDB681B689B69F0E77047885EFF1FCC
:10AAE000D89D0200A019FF1F0346052B10B508468C
:10AAF00014460BD006D8022B06D315F0E3F82060DD
:10AB0000002010BD182BF8D00420FAE715F0F6F855
:10AB1000F5E738B50D46044620B915F077F82860FA
:10AB2000204638BD0820FCE7012910B5044608D1AD
:10AB3000044A702115F041FE2046BDE8104015F092
:10AB40008FBE10BDC804050038B50D46044648B98F
:10AB500015F03CF82B68C1182960204614F0B4FEAB
:10AB6000204638BD0820FCE7022806D3052801D975
:10AB7000182802D100201060704704207047054B50
:10AB8000DB6E0846114603B11847034B1B68DB68B0
:10AB9000FAE700BF885EFF1F4862FF1F2DE9F04102
:10ABA0006B4D6C4FD5F890206B4BDFF80C826B4CE3
:10ABB0003846012115F037FE6949384615F0A5FEE3
:10ABC000D8F80C60736803F16802A26003F5947210
:10ABD000226003F5A472626003F5D472226203F569
:10ABE000E472626203F55272E26003F55A7203F591
:10ABF0006A70226103F5627203F57273E361336870
:10AC000062611B69A06198473368E0691B699847D6
:10AC1000336860691B69984733682068DB68984728
:10AC200033686068DB6898473368A068DB689847DA
:10AC300033682069DB6898473368E068DB689847C9
:10AC40003368606ADB6898473368206ADB68984736
:10AC50003368606A9B6998473368206A9B699847A4
:10AC6000336860699B6998473368E0689B699847D7
:10AC7000D8F810203B4B02F114011960736803F5FA
:10AC8000027393614FF4003015F04EF80023D4E9BD
:10AC90000012184614F09EFED5F89030324AC3F8E0
:10ACA0000422324AC3F808220122AF671A80304BCF
:10ACB000C5F89C302F4BC5F898302F4BC5F8943011
:10ACC0002E4BC5F8A0302E4BC5F8B4302D4BC5F82F
:10ACD000B0302D4BC5F8A4302C4BC5F8A8302C4B08
:10ACE000C5F8C4302B4BC5F8C0302B4BC5F8D0305D
:10ACF0002A4BC5F8CC302A4BC5F8C830294BC5F8CB
:10AD0000DC3085F88C204FF4F0733222C5E9213213
:10AD1000254BC5F8D430254BC5F8E8300220244B2C
:10AD2000C5F8EC30FFF7C0FE3368606ADB6898470F
:10AD3000606A204C0423437533681B689847236876
:10AD400098470021A3680846BDE8F041184700BFB6
:10AD5000885EFF1FC45FFF1F94810200A019FF1FC0
:10AD600029AB00004862FF1F6DAA000063AA000023
:10AD70004B9F0000659F0000619F00005D9F0000E9
:10AD800059AA000045AA0000399F000049AB000005
:10AD90002D9F0000ED9E0000019F00001D9E000001
:10ADA00013AB0000A9AA0000A19D000069AB000040
:10ADB000E9AA0000E00AFF1FD89D020038B5184B31
:10ADC000184CDD6820682B685B6998472B686068C1
:10ADD0009B6898472B68A0689B6898472B68E06839
:10ADE0009B6898472B6820699B6898472B68606927
:10ADF0009B6898472B68A0699B6898472B68E06917
:10AE00009B6898472B68206A9B68984715F004F860
:10AE1000054B5B689847002384F8243038BD00BF99
:10AE2000D89D0200D419FF1FE00AFF1F10B5034888
:10AE3000144615F0ECFD206010BD00BF5062FF1FEE
:10AE4000014815F0D6BD00BF5062FF1F10B5044683
:10AE500018B914F039FD204610BD0820FCE710B5E4
:10AE6000044618B914F00AFD204610BD0820FCE77E
:10AE70000021F4E74942F2E7F1E770B504461D46C8
:10AE80000E46002940F04E85A52A00F08F8256D844
:10AE9000172A00F0478126D8042A00F0E8800ED84F
:10AEA000012A00F0AD80002A00F09E80022A00F006
:10AEB000B280032A00F0BA800424204670BD072A1D
:10AEC00000F0068107D8052A00F0DF80062A00F08E
:10AED000E7800424F1E7082A00F01181152A00F028
:10AEE00017810424E9E7322A00F0B28113D81B2A23
:10AEF00000F0638107D8182A00F039811A2A00F07F
:10AF000044810424D9E71C2A00F06F811D2A00F037
:10AF100086810424D1E7A22A00F0008207D8332AD0
:10AF200000F0A1818C2A00F0A9810424C5E7A32A9E
:10AF300000F00C82A42A00F021820424BDE7B42A88
:10AF400000F0B58324D8AA2A00F018830CD8A72AC9
:10AF500000F0CE82C0F08682A82A00F0E082A92A02
:10AF600000F0F4820424A8E7AD2A00F0518307D84A
:10AF7000AB2A00F01B83AC2A00F0308304249CE74A
:10AF8000AE2A00F05D83B32A00F07983042494E7AD
:10AF9000BB2A00F0278413D8B82A00F0C88307D84A
:10AFA000B52A00F09083B62A00F09A83042484E73F
:10AFB000B92A00F0D683BA2A00F0ED8304247CE796
:10AFC000C02A00F06C8407D8BC2A00F03384BF2A62
:10AFD00000F04684042470E7CC2A00F07B84CE2A5B
:10AFE00000F09684042468E720B9002014F0FEFDE8
:10AFF000286062E71968002014F066FC00245CE712
:10B0000018B914F0E3FD286057E71968304614F0CA
:10B010007DFD344651E718B914F008FE28604CE76E
:10B020001968002014F02AFC002446E7002840F0AC
:10B030007C8414F039FE18B914F0E8FD28603CE770
:10B04000204614F03FFE12210646B14815F0DFFC01
:10B05000C0F313027A20D317A6FB00011CF0A2FC58
:10B0600000F11303262B98BF0020286025E718B9AC
:10B0700014F0FCFD286020E719680029B8BF494298
:10B08000304614F05FFD344617E718B914F0DEFDC2
:10B09000286012E71968002014F003FF00240CE771
:10B0A00010219B482CB915F0B2FCC0F30420286095
:10B0B00003E715F0ACFC2B681B0203F4F85320F4F3
:10B0C000F8521A431021924815F093FC0024F4E63C
:10B0D00010218F482CB915F09AFC00F01F00286051
:10B0E000EBE615F094FC2B6820F01F0203F01F0321
:10B0F0001A431021864815F07CFC3446DDE6002812
:10B1000040F0168414F03EFCC0F300102860D4E632
:10B11000002800F010841A687D48112115F069FCA0
:10B120000024CAE67B4E80B91521794815F06FFCE2
:10B1300048B14FF0807393FBF0F0B042A8BF3046A7
:10B1400028600024B9E63046FAE71B686BB14FF07F
:10B15000807292FBF3F2B242A8BF32462A601521F8
:10B160006B4815F046FC0024A7E63246F6E728B9FE
:10B170003321674815F04BFC28609EE61A68644846
:10B18000332115F036FC002497E66C2160482CB979
:10B1900015F03DFCC0F3804028608EE615F037FCCA
:10B1A0002B689B0403F4802320F480221A436C2133
:10B1B000574815F01EFC00247FE66C2154482CB93A
:10B1C00015F025FCC0F3C040286076E615F01FFCA2
:10B1D0002B68DB0403F4002320F400221A436C21C3
:10B1E0004B4815F006FC344667E638B90146484836
:10B1F00015F00DFCC0F3400028605EE600214448D5
:10B2000015F005FC2B685B0003F0020320F002023E
:10B210001A4300213E4815F0ECFB00244DE60028BF
:10B2200040F08C8314F04EFD12210646384815F08C
:10B23000EEFBC0F313027A20D317A6FB00011CF02B
:10B24000B1FB00F11303262B98BF0020286034E6E1
:10B2500018B914F029FD28602FE61978304614F04B
:10B260008DFC344629E618B914F02CFD286024E63C
:10B270001968002014F092FC00241EE650B96C21DD
:10B28000234815F0C4FB4FF48073C0F303600341FF
:10B290002B6012E61B68102B35D00FDC022B2ED052
:10B2A00006DC012B18D04FF0FF332B60102404E68E
:10B2B000042B26D0082BF6D105230EE0402B24D0FA
:10B2C00003DC202BEFD1032307E0802B24D0B3F540
:10B2D000807FE8D1002300E008232B606C210C481C
:10B2E00015F095FB2B681B0603F0706320F070626D
:10B2F0001A436C21064815F07CFB0024DDE507238A
:10B30000EBE70623E9E70423E7E70223E5E700BFCD
:10B310005062FF1FFFFF0F000123DEE76C21BB48D7
:10B320002CB915F074FBC0F3C1302860C5E515F0E9
:10B330006EFB2B68DB0303F4C03320F4C0321A43E6
:10B340006C21B24815F055FB3446B6E56C21AF4888
:10B350002CB915F05CFBC0F380302860ADE515F02A
:10B3600056FB2B689B0303F4804320F480421A436E
:10B370006C21A64815F03DFB00249EE56C21A348F6
:10B380002CB915F044FBC0F30030286095E515F0AA
:10B390003EFB2B681B0303F4805320F480521A43B6
:10B3A0006C219A4815F025FB002486E56C2197480E
:10B3B00004BB15F02CFB10F480464FF06C01934851
:10B3C00005D015F024FBC0F3C310286075E515F017
:10B3D0001EFB6C2104468D4815F019FB2205C0F3B5
:10B3E000021002D42860002467E540F008002860BD
:10B3F000344662E515F00BFB10F480444FF06C010D
:10B4000082480ED015F003FB2B68DB0103F4F063D8
:10B4100020F4F0621A436C217C4815F0EAFA3446B5
:10B420004BE515F0F4FA6C21784815F0F0FA2A682B
:10B43000120220F4006002F4006202436C2173489F
:10B4400015F0D7FA6C21714815F0E1FA2B681B0151
:10B4500003F0700320F070021A436C216B4815F062
:10B46000C8FA2AE56C216948ECB915F0D0FA10F455
:10B4700080444FF06C01654806D015F0C8FAC0F35F
:10B4800002102860002418E515F0C1FA6C21064668
:10B490005E4815F0BCFA3305C0F3C310A2D540F0E6
:10B4A0000800286009E515F0B2FA10F480444FF066
:10B4B0006C0156480ED015F0AAFA2B681B0103F058
:10B4C000700320F070021A436C21504815F091FA75
:10B4D0000024F2E415F09BFA2B68DB0103F4F0631F
:10B4E00020F4F0621A436C21484815F082FAE4E433
:10B4F0006C2146482CB915F08AFA00F00F0028603C
:10B50000DBE415F084FA2B6820F00F0203F00F0340
:10B510001A436C213D4815F06CFA3446CDE46D2198
:10B520003A482CB915F073FAC0F3C0302860C4E46F
:10B5300015F06DFA2B68DB039BB220F400421A432E
:10B540006D21324815F055FA0024B6E46D212F48DC
:10B550002CB915F05CFAC0F341302860ADE415F069
:10B5600056FA2B685B0303F4C04320F4C0421A432D
:10B570006D21264815F03DFA00249EE46D212348F4
:10B580002CB915F044FAC0F30320286095E415F0B7
:10B590003EFA2B681B0203F4706320F470621A43B6
:10B5A0006D211A4815F025FA344686E46D211748B6
:10B5B0002CB915F02CFAC0F3411028607DE415F089
:10B5C00026FA2B685B0103F0600320F060021A4347
:10B5D0006D210E4815F00DFA00246EE46D210B4824
:10B5E0002CB915F014FA00F00F00286065E415F08E
:10B5F0000EFA2B6820F00F0203F00F031A436D219F
:10B60000024815F0F6F9002457E400BF5062FF1F0E
:10B610006D21BD482CB915F0FAF9C0F3006028601F
:10B620004BE415F0F4F92B681B0603F0807320F04F
:10B6300080721A436D21B44815F0DBF934463CE4BE
:10B640006D21B14864B915F0E2F9001400F07F03F0
:10B6500010F0400018BF6FF07F00184328602CE402
:10B6600015F0D5F92B681B0403F4FE0320F4FE0249
:10B670001A436D21A44815F0BCF900241DE46C2187
:10B68000A1482CB915F0C3F9C0F34040286014E478
:10B6900015F0BDF92B685B0403F4003320F400328D
:10B6A0001A436C21984815F0A4F9002405E40028F9
:10B6B00040F047816F21944815F0A9F9C0F3044088
:10B6C0002860FFF7FABB20B914F0E0FA2860FFF712
:10B6D000F4BB1968002014F043FA0024FFF7EDBB17
:10B6E0008A4E88B91421884815F091F950B14FF06D
:10B6F000807393FBF0F0B042A8BF3046286000246E
:10B70000FFF7DBBB3046F9E71B6873B14FF080727F
:10B7100092FBF3F2B242A8BF32462A6014217A4863
:10B7200015F067F90024FFF7C8BB3246F5E76C2136
:10B73000754834B915F06BF9C0F340302860FFF755
:10B74000BCBB15F064F92B685B0303F4005320F4D1
:10B7500000521A436C216C4815F04BF93446FFF740
:10B76000ACBB6C21684834B915F051F9C0F30350F3
:10B770002860FFF7A2BB15F04AF92B681B0503F4FC
:10B78000700320F470021A436C215F4815F031F900
:10B790000024FFF792BB5D4E88B913215A4815F07B
:10B7A00036F950B14FF0807393FBF0F0B042A8BF70
:10B7B000304628600024FFF780BB3046F9E71B685D
:10B7C00073B14FF0807292FBF3F2B242A8BF3246DF
:10B7D0002A6013214C4815F00CF90024FFF76DBBCB
:10B7E0003246F5E77021484834B915F010F9C0F336
:10B7F00007202860FFF761BB15F009F92A681202DB
:10B8000020F47F4092B2024370213F4815F0F1F8D6
:10B8100031463D4815F0FBF82B68002B20F0040260
:10B8200018BF04231A433146374815F0E2F834466E
:10B83000FFF743BB702134482CB915F0E8F8C0B2CB
:10B840002860FFF73ABB15F0E2F82A7820F0FF00F5
:10B85000024370212C4815F0CCF80024FFF72DBBD3
:10B8600040B97021284815F0D2F8C0F30140286093
:10B87000FFF723BB1B68032B66D87021224815F005
:10B88000C6F82B681B0403F4403320F440321A43FB
:10B8900070211D4815F0ADF80024FFF70EBB702194
:10B8A000194834B915F0B3F8C0F380402860FFF7A9
:10B8B00004BB15F0ACF82B68002B20F4802218BFD5
:10B8C0004FF480231A4370210F4815F092F8344644
:10B8D000FFF7F3BA70210C4834B915F098F8C0F3AB
:10B8E00001502860FFF7E9BA15F091F82B681B05A5
:10B8F00003F4401320F440121A437021024815F05B
:10B9000078F80024FFF7D9BA5062FF1FFFFF0F003D
:10B91000E8B96F210F4815F07AF8C0F309002860E4
:10B92000FFF7CBBA0824FFF7C8BA0424FFF7C5BA5B
:10B930000424FFF7C2BA0424FFF7BFBA0424FFF7B8
:10B94000BCBA0424FFF7B9BA1024FFF7B6BA04242E
:10B95000FFF7B3BA5062FF1F07B5019201AB024671
:10B960000120FFF78AFA03B05DF804FB1346024694
:10B970000020FFF782BA014815F0C1B85062FF1FDE
:10B9800008B5002014F042F910B1094B987870B155
:10B99000084815F0A1F84FF4003014F0C5F9064935
:10B9A00000231846D1E9011214F014F8012008BD53
:10B9B000340BFF1F5062FF1FD419FF1F022804BF62
:10B9C0000B4B93F8F00030B90A4BDB681B685B69DE
:10B9D000094A10681847012809D1054B93F8F0303F
:10B9E000012B04D1034BDB681B689B69F0E77047B0
:10B9F000885EFF1FD89D0200D419FF1F10B51446A2
:10BA0000062805D8DFE800F006181627323741006F
:10BA1000042010BD136844F62062934239D842F2E4
:10BA20001172B3FBF2F102FB11311B4B89B29B681F
:10BA3000002098470020ECE7184B2468DA68D2E928
:10BA4000003000F5F4701CB1DB6900219847F1E784
:10BA50009B689847EEE7114B1168DB68104A1B683A
:10BA60005069DB69003118BF0121EFE7084613F088
:10BA700089FF2060DEE7094B094ADB6858681B68CC
:10BA800000F594705061DB68E3E70220FFF796FF52
:10BA9000D0E71020BDE700BFE00AFF1FD89D0200DD
:10BAA000D419FF1F0346052B10B5084614460BD0CA
:10BAB00006D8022B06D314F005F92060002010BD33
:10BAC000182BF8D00420FAE714F018F9F5E738B588
:10BAD0000D46044620B914F099F82860204638BD78
:10BAE0000820FCE738B5194C054694F824000128D5
:10BAF0001CD002281FD02946154815F018F8002040
:10BB000013F0FAFE002013F03DFF10F008041BD1E3
:10BB1000820619D56F210E4814F079FFC30113D5A1
:10BB200020460221BDE8384013F006BFA56202237B
:10BB300084F82430DFE7A36AEB1AB3F5FA6FDAD999
:10BB4000FFF73CFF0323F3E738BD00BFD419FF1F05
:10BB50005062FF1F012910B504460DD1074A70211C
:10BB600014F047FF2046064A0A2114F042FF2046FF
:10BB7000BDE8104014F08CBF10BD00BF1E000CC407
:10BB80000004080038B50D46044648B914F01EF804
:10BB90002B68C1182960204613F096FE204638BD58
:10BBA0000820FCE7022806D3052801D9182802D16D
:10BBB00000201060704704207047054BDB6E08467C
:10BBC000114603B11847034B1B68DB68FAE700BF57
:10BBD000885EFF1F4C62FF1F2DE9F0415C4C5D4FFA
:10BBE000D4F890205C4BDFF8D0815C4D38460121C1
:10BBF00014F031FF5A49384614F095FFD8F80C601C
:10BC0000736803F168022A6003F594726A6003F5B1
:10BC1000A472AA6003F5E472EA6003F552722A6125
:10BC200003F55A7203F562706A6103F56A7203F5EF
:10BC300072732B623368EA611B69A86198473368A5
:10BC40002868DB68984733686868DB68984733681A
:10BC5000A868DB6898473368E868DB68984733680A
:10BC60006869DB68984733682869DB6898473368F8
:10BC7000E8685B6998473368A8699B6998473368A7
:10BC800028699B699847D8F81020364B02F11401B7
:10BC90001960736803F5027393614FF4003014F078
:10BCA00043F80023D5E90112184613F093FED4F8A7
:10BCB00090202D4BC2F804322C4BC2F808320123DD
:10BCC000A76713802A4AC4F89C202A4AC4F89820FF
:10BCD000294AC4F89420294AC4F8A020284AC4F864
:10BCE000B420284AC4F8B020274AC4F8A420274A20
:10BCF000C4F8A820264AC4F8C420264AC4F8C020A4
:10BD0000254AC4F8D020254AC4F8CC20244AC4F8D7
:10BD1000C820244AC4F8DC2032214FF4F072C4E970
:10BD20002121214AC4F8D420204AC4F8E820204A1E
:10BD300084F88C30C4F8EC201E4C85F8243023683D
:10BD400098470021A3680846BDE8F041184700BFA6
:10BD5000885EFF1F5062FF1F94830200D419FF1FEB
:10BD600055BB00004C62FF1F81B9000077B900008D
:10BD70005FAE000079AE000075AE000071AE00004D
:10BD80006DB9000059B900004DAE000085BB000040
:10BD900041AE00002DAE0000E5BA0000FDB9000084
:10BDA000CFBA0000BDB90000BDAD0000A5BB0000CA
:10BDB000A5BA0000E00AFF1FD89D0200024B002236
:10BDC000C3F88020704700BF885EFF1F014814F051
:10BDD000EBBE00BF0C1AFF1F10B50348144614F049
:10BDE00016FF206010BD00BF0C1AFF1F38B51546A6
:10BDF000044628B9084613F0C5FD2860204638BD22
:10BE00000420FCE710B5044618B913F05DFD204688
:10BE100010BD0820FCE710B5044618B913F02EFD3C
:10BE2000204610BD0820FCE70021F4E74942F2E774
:10BE3000F1E7014814F0A8BF0C1AFF1F10B54FF42A
:10BE40000030074C13F070FF0023D4E9A21218460B
:10BE500013F0C0FD2046BDE8104014F07EBF00BFC7
:10BE60000C1AFF1F022804BF0C4B93F8F00038B9DE
:10BE70000B4BDB681B685B690A4AD2F884021847DF
:10BE8000012809D1054B93F8F030012B04D1044B64
:10BE9000DB681B689B69EFE7704700BF885EFF1F88
:10BEA000D89D02000C1AFF1F38B50020FFF7DAFFFB
:10BEB000144B154CDD68D4F884022B689B689847B6
:10BEC0002B68D4F888029B6898472B68D4F88C02BA
:10BED0009B6898472B68D4F890029B6898472B681A
:10BEE000D4F894029B6898472B68D4F898029B6812
:10BEF00098472B68D4F89C029B689847BDE8384067
:10BF000013F08ABFD89D02000C1AFF1F08B5014626
:10BF1000034814F0D7FE0020BDE8084013F0ECBC45
:10BF20000C1AFF1F38B50D46044648B913F04EFEF3
:10BF30002B68C1182960204613F0C6FC204638BD86
:10BF40000820FCE708B519BB052823D8DFE800F076
:10BF500003090E22131B1146002013F0B5FC00202C
:10BF600008BD1146002013F0D1FDF8E7114600206E
:10BF700013F084FCF3E782EAE271A1EBE2710020A6
:10BF800013F0E0FDEBE71146002013F08AFFE6E72F
:10BF90000820E5E70420E3E710B5144629BB06288E
:10BFA00025D8DFE800F0040A0E12161A1E00002041
:10BFB00013F01CFE2060002010BD002013F006FED0
:10BFC000F8E7002013F032FEF4E7002013F01EFE25
:10BFD000F0E7002013F04AFEECE7002013F036FEF5
:10BFE000E8E7044814F0D9FEE4E70820E4E7042079
:10BFF000E2E700BF0C1AFF1F0248DBB2D0F8A00234
:10C0000012F028B80C1AFF1F012214F0B1B870B555
:10C010000122534E534C1146072014F04DF8F56899
:10C020006B6803F59472C4F8882203F5A472C4F80F
:10C030008C2203F1C802C4F8902203F1E80203F154
:10C040006800C4F8942203F18802A833C4F89C3233
:10C050002B68C4F89822DB68C4F8840298472B68E0
:10C06000D4F88802DB6898472B68D4F88C02DB6828
:10C0700098472B68D4F89002DB6898472B68D4F86F
:10C080009402DB6898472B68D4F898021B6998479C
:10C090002B68D4F89C021B699847F36AC4F8A03255
:10C0A00000251D705B6898472F4B3049D3F89020CE
:10C0B000C2F804122E49C2F8081201262D49168032
:10C0C000C3F89C102C49C3F898102C49C3F894105D
:10C0D0002B49C3F8A0102B49C3F8B4102A49C3F860
:10C0E000B0102A49C3F8A4102949C3F8A810294957
:10C0F000C3F8C4102849C3F8C0102849C3F8CC10AD
:10C100002749C3F8DC102749C3F8D81032204FF470
:10C11000C371C3E921102449C3F8D410234983F81B
:10C120008C60C3F8D01020462946214B14F0AEFD98
:10C130004FF4003013F0F8FDD4E9A2122B46284644
:10C1400013F048FC28464FF4484113F0FBFC284606
:10C150004FF4484113F0A5FE3046BDE8704081E63B
:10C16000D89D02000C1AFF1F885EFF1F3DBE000015
:10C1700033BE000017BE000031BE00002DBE00001F
:10C1800029BE000099BF000045BF000005BE0000A9
:10C1900025BF0000CDBD0000D9BD0000EDBD0000F1
:10C1A00065BE0000BDBD0000A9BE00000DBF0000BF
:10C1B00094850200024B0022C3F88020704700BF24
:10C1C000885EFF1F014814F0EBBD00BFBC1CFF1FC1
:10C1D00010B50348144614F01AFE206010BD00BFCD
:10C1E000BC1CFF1F08B50146034814F073FE002075
:10C1F000BDE8084013F080BBBC1CFF1F10B50B4608
:10C20000144606286AD8DFE800F004090F131B283B
:10C210004A00084613F0B6FB206003E0217830485E
:10C2200014F0C6FE002010BD2D4814F0BEFEF3E74A
:10C230002C4B0220DB6898475023B0FBF3F0EBE770
:10C2400023684FF4FA5159436423B1FBF3F1254BB2
:10C2500089B29B6802209847E4E72168204A013BA5
:10C2600001F00301D2F88802042B06D8DFE803F0BE
:10C27000030B0E111400D2F88C021B4BDB681B68F9
:10C28000DB699847CEE7D2F89802F6E7D2F89C022D
:10C29000F3E7D2F8A802F0E7D2F8AC02EDE71049D4
:10C2A000013BD1F88802042B06D8DFE803F0030B2A
:10C2B0000E111400D1F88C020B4BDB681B681B6A53
:10C2C0009847A9E7D1F89802F6E7D1F89C02F3E77E
:10C2D000D1F8A802F0E7D1F8AC02EDE70420A2E71C
:10C2E000BC1CFF1FE00AFF1FD89D020010B50446CA
:10C2F00018B913F0E9FA204610BD0820FCE710B584
:10C30000044618B913F0BAFA204610BD0820FCE71D
:10C310000021F4E74942F2E7F1E770B504461D4613
:10C320000E46002940F03783A62A00F0E48162D847
:10C33000082A00F021811CD8032A00F0DB800BD8EA
:10C34000012A00F0C98040F2BB80002840F0CD8077
:10C35000002013F06BFCB7E0052A00F0DE80C0F08F
:10C36000CF80062A00F0E280072A00F0F58004243E
:10C3700060E1322A00F045811AD81C2A00F01581AC
:10C380001D2A00F02481172AF1D1B949B94A0028A1
:10C3900040F0FC80D1F8B012002900F0F5804FF099
:10C3A000807393FBF1F39342A8BF13462B6091E097
:10C3B0008C2A00F0348107D8332AD8D1002840F0E5
:10C3C000298113F07FFC7FE0A22A00F07581A52A65
:10C3D000CDD10028CBD16C21A54814F018FD10F464
:10C3E000804F4FF06C01A24800F0778114F00FFDF0
:10C3F000C0F3C31068E0B42A00F0258226D8AA2A28
:10C4000000F0E1810ED8A82A00F0C28140F2B0818C
:10C4100042219748002C40F0CD8114F0F8FCC0F385
:10C42000413051E0AC2A00F0F081C0F0DD81AE2A4D
:10C4300000F0F781B32A9AD16C218D48002C40F08E
:10C44000F98114F0E4FCC0F340403DE0BB2A00F069
:10C450004A8219D8B62A00F01882C0F0FE81BA2AA2
:10C4600085D1844E002840F030821321804814F09A
:10C47000CEFC002800F027824FF0807393FBF0F091
:10C48000B042A8BF3046BAE0C02A00F05D820CD8A6
:10C49000BF2A7FF46CAF002840F0458270217448B9
:10C4A00014F0B5FCC0F301400EE0CC2A00F062822B
:10C4B000CE2A7FF45CAF00287FF459AF4121B2E16E
:10C4C00020B9002013F092FB2860B3E01968002027
:10C4D00013F0FAF90024ADE010B913F077FBF3E79D
:10C4E0001968304613F012FBF4E71968002013F0C6
:10C4F000C5F9EFE700287FF43AAF13F087FBE3E7D5
:10C5000018B9002013F0B2FBDEE719680029B8BFA4
:10C510004942002013F016FBDCE710B913F096FB3C
:10C52000D2E71968304613F0BCFCD3E7102150481D
:10C5300024B914F06CFCC0F30420C5E714F067FCC8
:10C540002B681B0203F4F85320F4F8521A4310210D
:10C55000474814F025FCBDE71021454824B914F0E4
:10C5600056FC00F01F00AFE714F051FC2B6820F0E0
:10C570001F0203F01F03E9E700287FF4F8AE13F071
:10C5800001FAC0F300109FE713460FE7186850B197
:10C590004FF0807393FBF0F39342A8BF13462B60D8
:10C5A000C1F8B03296E71346F9E7314824B914F0E0
:10C5B0002EFCC0F3400087E714F029FC2B685B00D9
:10C5C00003F0020320F002021A433146C0E70028BC
:10C5D0007FF4CDAE002013F075FB122104462448F1
:10C5E00014F015FCC0F313027A20D317A4FB00014A
:10C5F0001BF0D8F900F11303262B98BF0020286008
:10C6000068E710B913F050FB5EE71978304613F075
:10C61000B5FA5FE71968002013F0C0FA5AE758B975
:10C620006C21134814F0F3FB4FF48073C0F30360E4
:10C6300003412B60204670BD1B68102B36D00FDCE9
:10C64000022B2FD006DC012B1DD04FF0FF332B60C7
:10C650001024EFE7042B27D0082BF6D1052313E095
:10C66000402B25D008DC202BEFD103230CE000BFAA
:10C67000BC1CFF1FFFFF0F00802B1BD0B3F5807F7A
:10C68000E3D1002300E008232B606C21B24814F0B2
:10C69000BEFB2B681B0603F0706320F070621A4328
:10C6A0006C2155E70723EFE70623EDE70423EBE7CB
:10C6B0000223E9E70123E7E76C21A74824B914F036
:10C6C000A6FBC0F3C130FFE614F0A1FB2B68DB032F
:10C6D00003F4C03320F4C032E1E714F098FB6C217E
:10C6E00006469D4814F093FB3205C0F3021086D530
:10C6F00040F00800E8E66C219748D4B914F087FBB5
:10C7000010F480464FF06C01934804D014F07FFB86
:10C71000C0F30210D8E614F07AFB6C2104468E4870
:10C7200014F075FB2305C0F3C31048BF40F00800A8
:10C7300065E714F06CFB10F480444FF06C01864800
:10C7400008D014F064FB2B681B0103F0700320F089
:10C750007002A4E714F05BFB2B68DB0103F4F063C9
:10C7600020F4F0621A436C217B4814F019FB61E756
:10C770006C21794824B914F04AFB00F00F00A3E6BD
:10C7800014F045FB2B6820F00F0203F00F0386E73F
:10C790004221714824B914F03AFBC0F3C03093E64B
:10C7A00014F035FB2B68DB039BB220F400421A43E4
:10C7B0004221CDE614F02BFB2B685B0303F4C0434E
:10C7C00020F4C042F3E74221634824B914F01FFB70
:10C7D000C0F3032078E614F01AFB2B681B0203F465
:10C7E000706320F47062E2E742215B4824B914F0E0
:10C7F0000EFBC0F3411067E614F009FB2B685B01E8
:10C8000003F0600320F06002D1E742215248002C7F
:10C81000B1D014F0FCFA2B6820F00F0203F00F03E4
:10C82000C5E720B940214C4814F0F1FA4CE61A68EB
:10C8300040218DE614F0EBFA2B685B0403F400331F
:10C8400020F400322BE700287FF491AD6F2142489D
:10C8500014F0DDFAC0F3044036E618B9002013F0F6
:10C8600015FA31E61968002013F07AF92B683B4974
:10C87000B3EBE30325D04FF0807292FBF3F28A42D0
:10C88000A8BF0A462A60142162E678B9142132480A
:10C8900014F0BDFA40B14FF0807393FBF0F02F4BD2
:10C8A0009842A8BF1846AAE62C48A8E61B6843B1E0
:10C8B0004FF0807292FBF3F2284B9A42A8BF1A46BF
:10C8C000E0E7264ADEE7304699E61B684BB14FF0B9
:10C8D000807292FBF3F2B242A8BF32462A60132163
:10C8E00036E63246FAE770211B4824B914F08FFA75
:10C8F000C0F30720E8E514F08AFA2A68120220F44F
:10C900007F4092B202437021134814F049FA314635
:10C91000114814F07CFA2B68002B20F00402D4BFDD
:10C920000423002350E61B68032B3FF691AE7021D1
:10C93000094814F06CFA2B681B0403F4403320F40C
:10C9400040321A43702103E67021034844B914F0C1
:10C950005EFAC0F38040B7E5BC1CFF1FFFFF0F006D
:10C9600014F055FA2B68002B20F4802218BF4FF4E6
:10C970008023E6E77021094824B914F048FAC0F38F
:10C980000150A1E514F043FA2B681B0503F4401392
:10C9900020F44012D5E708244CE600BFBC1CFF1F62
:10C9A00007B5019201AB02460120FFF7B6FC03B0C8
:10C9B0005DF804FB134602460020AEE4014814F083
:10C9C000EBBA00BFBC1CFF1F10B5084C4FF4003081
:10C9D00013F0AAF9D4F8A032D4E9A412002012F07E
:10C9E000F9FF2046BDE8104014F0BFBABC1CFF1F81
:10C9F000022804BF0C4B93F8F00038B90B4BDB68EE
:10CA00001B685B690A4AD2F888021847012809D1D5
:10CA1000054B93F8F030012B04D1044BDB681B6805
:10CA20009B69EFE7704700BF885EFF1FD89D02003B
:10CA3000BC1CFF1F70B50020FFF7DAFF1D4B1E4C1A
:10CA4000DD68D4F888022B689B6898472B68D4F877
:10CA50008C029B6898472B68D4F890029B68984793
:10CA60002B68D4F894029B6898472B68D4F89802F6
:10CA70009B6898472B68D4F89C029B6898472B6862
:10CA8000D4F8A0029B6898472B68D4F8A4029B684E
:10CA900098472B68D4F8AC029B6898472B68D4F869
:10CAA000A8029B68984713F0B7F9044BBDE87040A3
:10CAB0005B681847D89D0200BC1CFF1FE00AFF1FDF
:10CAC00038B50D46044648B913F080F82B68C118F4
:10CAD0002960204612F0F8FE204638BD0820FCE709
:10CAE0000248DBB2D0F8B40211F0B4BABC1CFF1F8C
:10CAF000012213F03DBBF7B501226B4F6B4C114681
:10CB0000072013F0D9FAFD686B6803F5B472C4F816
:10CB10008C2203F59472C4F8902203F5A472C4F831
:10CB2000942203F1C802C4F8982203F1E802C4F881
:10CB30009C2203F1880203F16800C4F8A02203F1EB
:10CB4000A80203F5C473C4E9AA302B68C4F8A42270
:10CB50000026DB68C4F8B062C4F8880298472B68E6
:10CB6000D4F88C02DB6898472B68D4F89002DB6815
:10CB700098472B68D4F89402DB6898472B68D4F860
:10CB80009802DB6898472B68D4F89C02DB689847CA
:10CB90002B68D4F8A0021B6998472B68D4F8A4022C
:10CBA0001B6998472B68D4F898029B6998472B68B3
:10CBB000D4F89C029B699847FB6AC4F8B4320127F9
:10CBC0001F705B6898473A4A3A49D2F8903082F829
:10CBD0008C70C3F804123849C3F808123749C2F8F8
:10CBE0009C103749C2F898103649C2F8941036495B
:10CBF000C2F8A0103549C2F8B4103549C2F8B010D7
:10CC00003449C2F8A4103449C2F8A8103349C2F814
:10CC1000C4103349C2F8C0103249C2F8CC103249AE
:10CC2000C2F8DC103149C2F8D81032204FF4C37179
:10CC3000C2E921102E49C2F8D4102E49C2F8D010F2
:10CC40002D4A009231463246204614F023F94FF423
:10CC5000003013F069F8D4E9A412D4F8A0323046B9
:10CC600012F0B8FE30464FF4484112F06BFF4FF41B
:10CC70004841304613F015F92B68D4F8A802DB6858
:10CC80009847D4F8A8021D4C042343752B681B68F1
:10CC9000984723689847A36831460220984738464A
:10CCA00003B0BDE8F040A3E6D89D0200BC1CFF1F06
:10CCB000885EFF1FC9C90000BDC90000FFC2000097
:10CCC00019C3000015C3000011C30000B5C900005E
:10CCD000A1C90000EDC20000C1CA0000C5C100002A
:10CCE000D1C10000FDC10000F1C90000B5C10000C4
:10CCF00035CA0000E5C1000094870200E00AFF1F6A
:10CD0000024B0022C3F88020704700BF885EFF1FDF
:10CD1000074870B550F8044B0D46164614F0A9F9B3
:10CD200033462A4601462046BDE8704011F0FDB961
:10CD3000801FFF1F074870B550F8044B0D4616467C
:10CD400014F097F933462A4601462046BDE8704064
:10CD500011F0A4B9801FFF1F38B51546044628B945
:10CD6000084612F00FFE2860204638BD0420FCE77C
:10CD700010B5044618B912F0A7FD204610BD0820D2
:10CD8000FCE710B5044618B912F078FD204610BD36
:10CD90000820FCE70021F4E74942F2E7F1E7024B03
:10CDA000D3F8940214F05DB9801FFF1F10B54FF443
:10CDB0000030074C12F0B8FF0023D4E9A712184640
:10CDC00012F008FED4F89402BDE8104014F041B906
:10CDD000801FFF1F022804BF0C4B93F8F00038B9E6
:10CDE0000B4BDB681B685B690A4AD2F8980218474C
:10CDF000012809D1054B93F8F030012B04D1044BE5
:10CE0000DB681B689B69EFE7704700BF885EFF1F08
:10CE1000D89D0200801FFF1F38B50020FFF7DAFF02
:10CE2000164B174CDD68D4F898022B689B6898471E
:10CE30002B68D4F89C029B6898472B68D4F8A00212
:10CE40009B6898472B68D4F8A4029B6898472B6886
:10CE5000D4F8A8029B6898472B68D4F8AC029B686A
:10CE600098472B68D4F8B0029B68984723689B6862
:10CE70009847BDE8384012F0CFBF00BFD89D0200F0
:10CE8000801FFF1F08B5064A0146D2F894320020E1
:10CE9000043214F0CFF80020BDE8084012F02CBD99
:10CEA000801FFF1F38B50D46044648B912F08EFEAC
:10CEB0002B68C1182960204612F006FD204638BDB7
:10CEC0000820FCE708B549BB062829D8DFE800F0B0
:10CED000040A0F28141C21001146002012F0F4FC53
:10CEE000002008BD1146002012F010FEF8E71146A0
:10CEF000002012F0C3FCF3E782EAE271A1EBE271D9
:10CF0000002012F01FFEEBE71146002012F0C9FFCF
:10CF1000E6E7D1B2034814F0AFF8E1E70820E0E714
:10CF20000420DEE7841FFF1F10B5144629BB062826
:10CF300025D8DFE800F0040A0E12161A1E000020A1
:10CF400012F054FE2060002010BD002012F03EFEC2
:10CF5000F8E7002012F06AFEF4E7002012F056FE17
:10CF6000F0E7002012F082FEECE7002012F06EFEE7
:10CF7000E8E7044814F07DF8E4E70820E4E704203B
:10CF8000E2E700BF841FFF1F70B50122514C524ED3
:10CF90001146072013F090F8201D14F00DF8F568E5
:10CFA0006B6803F59472C4F89C2203F5A472C4F86C
:10CFB000A02203F1C802C4F8A42203F1E80203F19D
:10CFC0006800C4F8A82203F18802A833C4F8B0327C
:10CFD0002B68C4F8AC22DB68C4F8980298472B6829
:10CFE000D4F89C02DB6898472B68D4F8A002DB6871
:10CFF00098472B68D4F8A402DB6898472B68D4F8CC
:10D00000A802DB6898472B68D4F8AC021B699847E4
:10D010002B68D4F8B0021B699847F36A23605B68F9
:10D0200098472E4B2E49D3F89020C4F8942201251E
:10D03000C2F804122B491580C2F808122A4AC3F814
:10D040009C202A4AC3F89820294AC3F89420294AE8
:10D05000C3F8A020284AC3F8B420284AC3F8B02057
:10D06000274AC3F8A420274AC3F8A820264AC3F8B1
:10D07000C420264AC3F8C020254AC3F8CC20254A3C
:10D08000C3F8DC20244AC3F8D82032214FF4C372FD
:10D09000C3E92121214AC3F8D4204FF40030204AAB
:10D0A00083F88C50C3F8D02012F03EFE0023D4E960
:10D0B000A712184612F08EFC4FF44841002012F0DF
:10D0C00041FD00204FF4484112F0EBFE2846BDE838
:10D0D00070407FE6801FFF1FD89D0200885EFF1F03
:10D0E000ADCD00009FCD000083CD00009DCD0000A0
:10D0F00099CD000095CD000029CF0000C5CE0000DD
:10D1000071CD0000A5CE000011CD000035CD00008E
:10D1100059CD0000D5CD000001CD000019CE000092
:10D1200085CE0000024B0022C3F88020704700BF6C
:10D13000885EFF1F014813F0A3BF00BF4022FF1FFE
:10D1400010B50348144613F0CEFF206010BD00BF99
:10D150004022FF1F10B5044618B912F0B5FB204657
:10D1600010BD0820FCE710B5044618B912F086FB84
:10D17000204610BD0820FCE70021F4E74942F2E711
:10D18000F1E7F8B506461D460C46002940F06E82D0
:10D19000332A00F0228140D8052A00F0C08017D839
:10D1A000022A00F0A58007D8002A00F08C80012A0E
:10D1B00000F09480042624E1032A00F0A280042ACF
:10D1C000F8D1002840F0A380002012F04FFD7DE050
:10D1D000082A00F0CB800ED8062A00F0A980072A82
:10D1E000E8D11021BA48002E40F0B88013F07BFF40
:10D1F00000F01F006AE01D2A00F0CD80322A00F006
:10D20000E2801C2AD6D1002840F0B8800146B04800
:10D2100013F069FFC0F3400058E0B42A00F0AE817B
:10D2200023D8A52A00F033810ED88C2A00F0DE80A6
:10D23000A22ABFD16C21A648002E40F01F8113F016
:10D2400052FFC0F3C13041E0A72A00F07E81C0F058
:10D250004381B32AAED16C219D48002E40F08581D8
:10D2600013F041FFC0F3404030E0BB2A00F0AA8138
:10D2700017D8B52A00F08C81BA2A9BD1002840F03B
:10D2800092811321924813F02EFF002800F089812B
:10D290004FF0807393FBF0F08E4B9842A8BF184676
:10D2A00014E1C02A00F0BF81CC2A00F0CE81BF2A51
:10D2B00080D1002840F0A6817021854813F013FF2B
:10D2C000C0F3014002E018B912F090FC286098E029
:10D2D0001968104612F0F8FA002692E018B90020FA
:10D2E00012F074FCF2E71968002012F00FFCF3E76B
:10D2F00010B912F09BFCE9E71968204612F0BEFA5B
:10D30000EAE700287FF456AF12F080FCDEE71968E8
:10D310000029B8BF4942002012F014FCDCE710B924
:10D3200012F094FCD2E71968204612F0BAFDD3E758
:10D330001021674826B913F0D6FEC0F30420C5E7D4
:10D3400013F0D1FE2B681B0203F4F85320F4F852BB
:10D350001A4310215E4813F093FEBDE713F0C3FE9D
:10D360002B6820F01F0203F01F03F1E700287FF471
:10D3700021AF12F007FBC0F30010A7E700215448CB
:10D3800013F0B1FE2B685B0003F0020320F00202F1
:10D390001A430021DEE700287FF40CAF12F092FC64
:10D3A000122104464A4813F09EFEC0F313027A206D
:10D3B000D317A4FB00011AF0F5FA00F11303262B92
:10D3C00098BF002082E718B9002012F06DFC7DE7BD
:10D3D0001978002012F0D2FB7EE710B912F072FC2F
:10D3E00074E71968204612F0D9FB75E758B96C212B
:10D3F000374813F078FE4FF48073C0F303600341A5
:10D400002B603046F8BD1B68102B31D00FDC022B8F
:10D410002AD006DC012B18D04FF0FF332B601026EA
:10D42000EFE7042B22D0082BF6D105230EE0402B8A
:10D4300020D003DC202BEFD1032307E0802B1BD06F
:10D44000B3F5807FE8D1002300E008232B606C2136
:10D450001F4813F048FE2B681B0603F0706320F092
:10D4600070621A436C2175E70723EFE70623EDE7A7
:10D470000423EBE70223E9E70123E7E713F033FE98
:10D480002B68DB0303F4C03320F4C032E9E7002843
:10D490007FF490AE6C210E4813F025FE10F480440A
:10D4A0004FF06C010A4804D013F01DFEC0F3C31006
:10D4B0000CE713F018FE6C210646054813F013FE26
:10D4C000C0F30210330548BF40F00800286003E7AE
:10D4D0004022FF1FFFFF0F006C216548B6B913F013
:10D4E00002FE10F480444FF06C01614804D013F048
:10D4F000FAFDC0F30210E9E613F0F5FD6C210646D3
:10D500005B4813F0F0FDC0F3C310DBE713F0EBFD55
:10D5100010F480464FF06C01554808D013F0E3FD3D
:10D520002B681B0103F0700320F0700299E713F0E1
:10D53000DAFD2B68DB0103F4F06320F4F0621A4398
:10D540006C214B4813F09CFD5BE76C21484826B9E1
:10D5500013F0C9FD00F00F00B8E613F0C4FD2B680E
:10D5600020F00F0203F00F037BE713F0BCFD2B68E4
:10D570005B0403F4003320F4003272E700287FF4E8
:10D5800019AE6F213A4813F0AEFDC0F304409DE69A
:10D5900010B912F07BFB99E61968204612F0E0FA08
:10D5A0009AE6344892E71B6853B14FF0807292FBC1
:10D5B000F3F2304B9A42A8BF1A462A601321C9E6FB
:10D5C0002C4AFAE770212A4826B913F08CFDC0F3E3
:10D5D00007207BE613F087FD2A68120220F47F40C3
:10D5E00092B202437021224813F04AFD214620489E
:10D5F00013F079FD2B68002B20F00402D4BF042324
:10D600000023C5E61B68032B3FF609AF70211848BD
:10D6100013F069FD2B681B0403F4403320F44032FF
:10D620001A43702196E67021114826B913F05BFD6C
:10D63000C0F380404AE613F056FD2B68002B20F41F
:10D64000802218BF4FF48023EAE77021084826B9EA
:10D6500013F049FDC0F3015038E613F044FD2B6888
:10D660001B0503F4401320F44012D9E70826C8E64E
:10D670004022FF1FFFFF0F0007B5019201AB0246DA
:10D680000120FFF77EFD03B05DF804FB1346024660
:10D69000002076E5014813F0E3BD00BF4022FF1FE4
:10D6A00010B54FF40030074C12F03EFB0023D4E9D4
:10D6B000A312184612F08EF92046BDE8104013F070
:10D6C000B8BD00BF4022FF1F022804BF0C4B93F8D7
:10D6D000F00038B90B4BDB681B685B690A4AD2F86B
:10D6E00088021847012809D1054B93F8F030012B27
:10D6F00004D1044BDB681B689B69EFE7704700BFF0
:10D70000885EFF1FD89D02004022FF1F38B5002011
:10D71000FFF7DAFF144B154CDD68D4F888022B684C
:10D720009B6898472B68D4F88C029B6898472B68B5
:10D73000D4F890029B6898472B68D4F894029B68B1
:10D7400098472B68D4F898029B6898472B68D4F8C0
:10D750009C029B6898472B68D4F8A0029B68984766
:10D76000BDE8384012F058BBD89D02004022FF1F90
:10D7700008B50146034813F011FD0020BDE808403C
:10D7800012F0BAB84022FF1F10B51446042828D85A
:10D79000DFE800F003080E121A00084612F0F2F853
:10D7A000206003E01178104813F063FD002010BDE5
:10D7B0000D4813F061FDF3E70C4B0220DB6898473E
:10D7C0005023B0FBF3F0EBE713684FF4FA515943E1
:10D7D0006423B1FBF3F1054B89B29B6802209847A3
:10D7E000E4E70420E3E700BF4022FF1FE00AFF1F39
:10D7F00038B50D46044648B912F0E8F92B68C1184F
:10D800002960204612F060F8204638BD0820FCE769
:10D810000248DBB2D0F8A80210F01CBC4022FF1F67
:10D82000012212F0A5BC70B501225F4E5F4C11467B
:10D83000072012F041FCF5686B6803F59472C4F898
:10D840008C2203F5A472C4F8902203F1C802C4F834
:10D85000942203F1E802C4F8982203F1880203F14C
:10D860006800C4F89C2203F1A80203F5C473C4F84D
:10D87000A4322B68C4F8A022DB68C4F88802984759
:10D880002B68D4F88C02DB6898472B68D4F8900298
:10D89000DB6898472B68D4F89402DB6898472B68BC
:10D8A000D4F89802DB6898472B68D4F89C021B696F
:10D8B00098472B68D4F8A0021B699847F36AC4F80C
:10D8C000A83201261E705B689847394B3949D3F856
:10D8D0009020C2F804123849C2F80812374916805D
:10D8E000C3F89C103649C3F898103649C3F8941011
:10D8F0003549C3F8A0103549C3F8B4103449C3F80A
:10D90000B0103449C3F8A4103349C3F8A810334900
:10D91000C3F8C4103249C3F8C0103249C3F8CC1060
:10D920003149C3F8DC103149C3F8D81032204FF424
:10D93000C371C3E921102E49C3F8D4102D4983F8CF
:10D940008C60C3F8D01020462B4B002113F00AFC4A
:10D950004FF4003012F0E8F90023D4E9A31218467E
:10D9600012F038F84FF44841002012F0EBF84FF471
:10D970004841002012F095FA2B68D4F8A402DB6825
:10D980009847D4F8A4021D4C042343752B681B68E8
:10D99000984723689847A368022041F2707198471E
:10D9A0003046BDE870408FE6D89D02004022FF1F40
:10D9B000885EFF1FA1D6000095D6000067D1000049
:10D9C00081D100007DD1000079D100008DD600000A
:10D9D00079D6000055D10000F1D7000035D1000004
:10D9E00041D1000089D70000C9D6000025D1000030
:10D9F0000DD7000071D7000094890200E00AFF1FD4
:10DA0000012810B514460DD043B21BB1022810D026
:10DA1000042010BD12680949B2FA82F252090A7153
:10DA20000020F6E71368064AB3FA83F35B09136034
:10DA3000F6E7084611F0A6FF2060F1E7F824FF1F83
:10DA40006C00FF1F10B50348144613F061FC206002
:10DA500010BD00BFF824FF1F70B5164C01462046CC
:10DA600013F0A0FC002011F047FF002012F0CEF8C8
:10DA7000A36894F840200028B8BF4042984234BFC1
:10DA800000260126B24213D098424FF00501094802
:10DA90002CBFA579657913F03BFC05F00F0520F04C
:10DAA0000F022A430521034813F020FC84F840604C
:10DAB00070BD00BFF824FF1F014813F017BC00BF62
:10DAC000F824FF1F10B5044618B911F0FDFE2046DA
:10DAD00010BD0820FCE710B5044618B911F0CEFEC1
:10DAE000204610BD0820FCE70021F4E74942F2E798
:10DAF000F1E770B504461D460E46002940F032831A
:10DB0000A72A00F0148267D81D2A00F0028122D8CB
:10DB1000042A00F005810DD8012A00F0E880002ACF
:10DB200000F0D980022A00F0EB80032A00F0F18097
:10DB300004245EE1062A00F00981C0F0FD80072A76
:10DB400000F01A81082AF3D10028F1D111F01AFF50
:10DB5000C0F30010C3E0A12A00F086811AD8332A4E
:10DB600000F0278107D8322AE2D1002840F01C813A
:10DB700012F09AF8B3E08C2A00F02481A02AD7D1C1
:10DB8000002840F064810821B64813F0C1FBC0F3BF
:10DB90004020A4E0A42A00F099810ED8A22A00F027
:10DBA0007581A32AC4D1002840F085810C21AD489D
:10DBB00013F0AEFBC0F3803091E0A52A00F099810C
:10DBC000A62AB5D1002840F0A7810C21A54813F062
:10DBD0009FFBC0F3021082E0B22A00F0458241D8D8
:10DBE000AC2A00F0F48113D8A92A00F0C581C0F056
:10DBF000B081AA2A00F0D181AB2A99D10521994898
:10DC0000002C40F0DB8113F083FBC0F3411066E091
:10DC1000AF2A00F0FD8115D8AD2A00F0DF81AE2AD1
:10DC200086D106218F48002C40F0E98113F070FB6B
:10DC3000000A00F07F0310F0400018BF6FF07F0073
:10DC400018434CE0B02A00F0F581B12A7FF470AFA0
:10DC500007218448002C40F0FE8113F059FBC0F3EB
:10DC600080203CE0B72A00F0378210D8B42A00F0B8
:10DC70001D82C0F00A82B52A00F02282B62A7FF403
:10DC800057AF784B002840F024829B6861E0CE2A91
:10DC900000F0468213D8B82A00F02E82B92A7FF409
:10DCA00047AF07216F48002C00F09B8113F030FB39
:10DCB0002B681B0403F4803320F48032B7E1D02AB0
:10DCC00000F04482D62A7FF433AF664B002840F040
:10DCD00046821B693DE020B9002011F087FF2860D3
:10DCE00087E01968002011F0EFFD002481E010B9F1
:10DCF00011F06CFFF3E71968304611F007FFF4E705
:10DD000010B911F093FFEAE71968002011F0B6FD91
:10DD1000EBE7002C7FF40CAF204611F077FFDEE735
:10DD200010B911F0A3FFDAE719680029B8BF49421A
:10DD3000304611F007FFD8E718B9002011F086FF30
:10DD4000CDE71968002012F0ACF8CEE7454E10B9C7
:10DD5000737B2B604DE01B687373337B002BC4D146
:10DD60000621404813F0D4FA737B20F01F0203F021
:10DD70001F031A430621FDE03A4E08B9B37BE8E7DA
:10DD80001B68B373337B012BAFD10621304613F0F0
:10DD9000BFFAB37B20F01F0203F01F031A430621D2
:10DDA000304613F0A3FAA0E71978002011F0E6FE40
:10DDB0009BE710B911F086FF91E71968304611F022
:10DDC000EDFE92E740B90821264813F0A1FA00F0D1
:10DDD0000F00C0F1080082E71B68102B31D010DC67
:10DDE000022B2AD007DC012B19D04FF0FF332B6018
:10DDF0001024204670BD042B21D0082BF5D105231B
:10DE00000EE0402B1FD003DC202BEED1032307E0D4
:10DE1000802B1AD0B3F5807FE7D1002300E00823E0
:10DE20002B6000210F4813F073FA2B6820F00F02CB
:10DE300003F00F031A4300219CE00723F0E70623B9
:10DE4000EEE70423ECE70223EAE70123E8E70021F9
:10DE5000044813F05DFA2B685B0203F4007320F4AE
:10DE60000072E7E7F824FF1F30B90821AB4813F030
:10DE70004FFAC0F3002032E7A84813F049FA2B68A4
:10DE80001B0203F4807320F48072D3E730B90C21B5
:10DE9000A24813F03DFAC0F3C13020E704219F48A7
:10DEA00013F036FA2B68DB0303F4C03320F4C032DE
:10DEB0001A4304215EE00421984813F029FA2B68E4
:10DEC0009B0303F4804320F48042F1E730B90C2136
:10DED000924813F01DFAC0F3C12000E704218F48D7
:10DEE00013F016FA2B68DB0203F4C05320F4C0527F
:10DEF000DEE730B90C21894813F00AFAC0F3C310E9
:10DF0000EDE60421854813F003FA2B68DB0103F4E6
:10DF1000F06320F4F062CBE70421804813F0F8F9B5
:10DF20002B681B0103F0700320F07002C0E730B9CA
:10DF30000C217A4813F0ECF900F00F00CFE6042131
:10DF4000764813F0E5F92B6820F00F0203F00F0379
:10DF5000AEE70521714824B913F0DAF9C0F3C030F7
:10DF6000BDE613F0D5F92B68DB039BB220F4004229
:10DF70001A430521694814E70521684824B913F0BC
:10DF8000C7F9C0F34130AAE613F0C2F92B685B036E
:10DF900003F4C04320F4C042EAE705215F4824B9F6
:10DFA00013F0B6F9C0F3032099E613F0B1F92B682A
:10DFB0001B0203F4706320F47062D9E713F0A8F930
:10DFC0002B685B0103F0600320F06002D0E7534B45
:10DFD00008B99B79BDE62A689A7186E606214F4802
:10DFE00024B913F095F9C0F3004078E613F090F9E6
:10DFF0002B681B0403F4803320F48032B9E613F05D
:10E0000087F92B681B0203F4FE4320F4FE42B0E6BE
:10E010000721424824B913F07BF9C0F381305EE652
:10E0200013F076F92B689B039BB220F440421A430D
:10E0300007219FE70721394824B913F069F9C0F394
:10E0400001304CE613F064F92B681B0303F44053D2
:10E0500020F44052EBE713F05BF92B689B0203F4CA
:10E06000806320F48062E2E707212C4824B913F092
:10E070004FF9C0F3012032E613F04AF92B681B0276
:10E0800003F4407320F44072D1E70721234824B9F8
:10E0900013F03EF9C0F3801021E613F039F92B6834
:10E0A0009B0103F0400320F04002C0E700287FF40A
:10E0B0003FAD0221194813F02BF9C0F384200EE67E
:10E0C00010B911F0E3FD0AE61968002011F048FDCF
:10E0D0000BE62A689A6008E60721104824B913F075
:10E0E00017F9C0F3C010FAE513F012F92B68DB0141
:10E0F000DBB220F080029AE70421084824B913F02B
:10E1000007F9C0F34030EAE513F002F92B685B032E
:10E1100003F4005320F40052CAE600BFF824FF1FA6
:10E1200000287FF405AD104B1B6843B102210F4856
:10E1300013F0EEF8800A00F478702860D5E501212C
:10E140000A4813F0E5F8C0F38920F6E700287FF4C9
:10E15000EFAC0321054813F0DBF8C0B2BFE52A6835
:10E160001A61C2E5082444E66C00FF1FF824FF1F73
:10E1700007B5019201AB02460120FFF7BAFC03B0DC
:10E180005DF804FB134602460020B2E4014813F098
:10E190007BB900BFF824FF1F022804BF0B4B93F884
:10E1A000F00030B90A4BDB681B685B69094A106DE7
:10E1B0001847012809D1054B93F8F030012B04D101
:10E1C000034BDB681B689B69F0E77047885EFF1FA5
:10E1D000D89D0200F824FF1F38B50020FFF7DCFFB0
:10E1E0000F4B104CDD68206D2B685B6998472B68DE
:10E1F000606C9B6898472B68E06C9B6898472B681D
:10E20000206D9B6898472B68606D9B6898472B68CA
:10E21000A06C9B689847BDE8384011F0FDBD00BF79
:10E22000D89D0200F824FF1F0346052B10B50846B1
:10E2300014460BD006D8022B06D311F043FD206004
:10E24000002010BD182BF8D00420FAE711F056FD7D
:10E25000F5E738B50D46044620B911F0D7FC286023
:10E26000204638BD0820FCE770B5002011F0CEFC38
:10E270000646A8B90B4D284613F0EAF80A4B0124CC
:10E2800002201C60FFF788FF4FF4003011F04CFDB6
:10E2900030466B6DD5E9121211F09CFB204670BD23
:10E2A0000020FCE7F824FF1F6C00FF1F38B50D4667
:10E2B000044648B911F08AFC2B68C1182960204631
:10E2C00011F002FB204638BD0820FCE7022806D3E7
:10E2D000052801D9182802D10020106070470420B9
:10E2E0007047054BDB6E0846114603B11847034BD8
:10E2F000DB6DDB68FAE700BF885EFF1FF824FF1FB5
:10E300002DE9F041444B454C454DDFF86881D4F888
:10E310009020012700211F602846424B13F01DF872
:10E32000D8F80C60736803F168022A6503F188026B
:10E3300003F594706A6503F5A47203F502736B64C8
:10E340003368EA64DB68A86498473368E86CDB6884
:10E3500098473368286DDB6898473368686D1B6998
:10E3600098473368686CDB689847D8F8103003F139
:10E370001402EA656A6C9A614FF4003011F0D4FC23
:10E380006B6DD5E91212002011F024FBD4F8903007
:10E39000254AC3F80822254AC3F80422244BC4F8AE
:10E3A0009C30244BC4F89830234BC4F89430234B52
:10E3B000C4F8A030224BC4F8B430224BC4F8B030BB
:10E3C000214BC4F8A430214BC4F8A830204BC4F82A
:10E3D000C430204BC4F8C0301F4BC4F8D0301F4BA2
:10E3E000C4F8CC301E4BC4F8C8301E4BC4F8DC3027
:10E3F00032224FF41673C4E921321B4BC4F8D430D7
:10E400001A4BC4F8E8301A4B84F88C70C4F8EC301E
:10E410000220BDE8F041BFE66C00FF1F885EFF1FD1
:10E42000F824FF1F948B02008DE1000069E20000D8
:10E43000D7DA0000F1DA0000EDDA0000E9DA0000D6
:10E4400085E1000071E10000C5DA0000ADE20000E6
:10E45000B9DA000045DA000059DA000001DA0000FC
:10E4600053E2000099E10000D9E10000CDE2000094
:10E4700029E20000D89D0200012810B514460DD0F5
:10E4800043B21BB1022810D0042010BD1268094904
:10E49000B2FA82F252098A720020F6E71368064A3D
:10E4A000B3FA83F35B091360F6E7084611F06AFAE2
:10E4B0002060F1E76425FF1F7000FF1F10B50446C0
:10E4C00018B911F001FA204610BD0820FCE7024BF4
:10E4D000986C13F090B800BF6425FF1F022804BF9A
:10E4E0000B4B93F8F00030B90A4BDB681B685B6993
:10E4F000094A906D1847012809D1054B93F8F0306F
:10E50000012B04D1034BDB681B689B69F0E7704764
:10E51000885EFF1FD89D02006425FF1F38B50020CC
:10E52000FFF7DCFF0F4B104CDD68A06D2B685B69BB
:10E5300098472B68E06C9B6898472B68606D9B68D8
:10E5400098472B68A06D9B6898472B68E06D9B6887
:10E5500098472B68206D9B689847BDE8384011F0BC
:10E560005BBC00BFD89D02006425FF1F38B50D4677
:10E57000044620B911F04AFB2860204638BD082027
:10E58000FCE710B5044628B9034B188111F076F961
:10E59000204610BD0820FCE76425FF1F0021F0E79E
:10E5A0004942EEE7EDE770B5002011F02FFB06467B
:10E5B000B0B90C4DA96C284613F000F80A4B0124A1
:10E5C00002201C60FFF78AFF4FF4003011F0ACFB13
:10E5D0003046EB6DD5E9141211F0FCF9204670BD00
:10E5E0000020FCE76425FF1F7000FF1F38B50D46B3
:10E5F000044648B911F0EAFA2B68C1182960204690
:10E6000011F062F9204638BD0820FCE738B51F4CF0
:10E61000636E05469B680021C0F30740984794F855
:10E620006820A36C03EB820300025860636E002134
:10E630009B68C5F30720984794F86830A26C02EBFA
:10E640008302012153681843636E000250609B6887
:10E65000E8B29847A26C94F8681002EB81014B680D
:10E6600018430011AB0C486010610AD0C5F3424357
:10E67000072B03D1C5F3011184F8681043F0080398
:10E6800000E0082302EB83035D6038BD6425FF1FB3
:10E6900010B40A4C00F07702A36C42F0080203EBBE
:10E6A0008203C1F313015960A37A23B941EA4040C0
:10E6B00010BCFFF7ABBF10BC704700BF6425FF1F45
:10E6C00008461146E4E738B504460F2000F013F879
:10E6D0000323B4FBF3F303EB4303E41A0546E4B26C
:10E6E00020F0300040EA0410FFF790FF2846BDE814
:10E6F0003840FFF78BBF38B5084DA97A00F0080203
:10E7000051EA0203044601D1FFF7DDFFAB6C04F0D0
:10E710007F0403EB8404606838BD00BF6425FF1FDD
:10E7200070B504461D460E46002940F02E83A72AE8
:10E7300000F0028264D81D2A00F0F38022D8042A57
:10E7400000F0F6800DD8012A00F0D980002A00F0F0
:10E75000CA80022A00F0DC80032A00F0E280042450
:10E7600018E1062A00F0FA80C0F0EE80072A00F0D7
:10E770002081082AF3D10028F1D111F003F9C0F368
:10E780000010B4E0A12A00F0838119D8332A00F0E8
:10E790002B8107D8322AE2D1002840F0208111F0E5
:10E7A00083FAA4E08C2A00F02881A02AD7D108207F
:10E7B000002C40F06481FFF79EFFC0F3402096E0FC
:10E7C000A42A00F090810DD8A22A00F07181A32A1A
:10E7D000C5D10C20002C40F07D81FFF78CFFC0F3E9
:10E7E000803084E0A52A00F08E81A62AB7D10C20C3
:10E7F000002C40F09881FFF77EFFC0F3021076E016
:10E80000B22A00F041823ED8AC2A00F0E98112D849
:10E81000A92A00F0B981C0F0A381AA2A00F0C5811D
:10E82000AB2A9CD1002840F0D1810520FFF763FF7F
:10E83000C0F341105BE0AF2A00F0F98114D8AD2A93
:10E8400000F0DA81AE2A8AD1002840F0E681062065
:10E85000FFF751FF000A00F07F0310F0400018BFDF
:10E860006FF07F00184342E0B02A00F0F281B12A35
:10E870007FF475AF002840F0FD810720FFF73BFFD4
:10E88000C0F3802033E0B72A00F0358210D8B42AD4
:10E8900000F01C82C0F00982B52A00F02082B62A5E
:10E8A0007FF45DAFAC4B002840F022821B6958E03A
:10E8B000CE2A00F04B820AD8B82A00F02C82B92A5E
:10E8C0007FF44DAF002840F03782072096E1D02A30
:10E8D00000F05082D62A7FF442AF9F4B002840F0D0
:10E8E00051825B683DE020B9002011F07FF928607B
:10E8F00050E01968002010F0E7FF00244AE010B94A
:10E9000011F064F9F3E71968304611F0FFF8F4E705
:10E9100010B911F08BF9EAE71968002010F0AEFF8A
:10E92000EBE7002C7FF41BAF204611F06FF9DEE718
:10E9300010B911F09BF9DAE719680029B8BF49420C
:10E94000304611F0FFF8D8E718B9002011F07EF931
:10E95000CDE71968002011F0A4FACEE77E4E10B979
:10E96000F37A2B6016E01B68F3727C4BDB6E9BB96D
:10E970000020FFF7C0FE10F08004BED10E20FFF78C
:10E98000BAFEF37A20F01F0103F01F0319430E2093
:10E99000FFF77EFE204670BD2B6833700E20FFF718
:10E9A000AAFEF37A20F01F0103F01F0319430E2083
:10E9B000E7E0694E08B93378D3E71B683370674BDB
:10E9C000DC6E4CB92046FFF796FE030695D50E2067
:10E9D000FFF791FE3378D5E72B68F3728DE719784E
:10E9E000002011F0CBF888E710B911F06BF97EE741
:10E9F0001968304611F0D2F87FE738B90820FFF7E0
:10EA00007AFE00F00F00C0F1080070E71B68102BC1
:10EA10002FD00FDC022B28D006DC012B18D04FF0B2
:10EA2000FF332B601024B5E7042B20D0082BF6D140
:10EA300005230EE0402B1ED003DC202BEFD1032357
:10EA400007E0802B19D0B3F5807FE8D1002300E0E8
:10EA500008232B600820FFF74EFE2B6820F00F01E3
:10EA600003F00F03194308208BE00723F1E7062387
:10EA7000EFE70423EDE70223EBE70123E9E7FFF7E4
:10EA80003AFE2B685B0203F4007320F40071E9E79F
:10EA9000082024B9FFF72FFEC0F3002027E7FFF777
:10EAA0002AFE2B681B0203F4807320F48071D9E7DF
:10EAB0000C2024B9FFF71FFEC0F3C13017E7FFF7A2
:10EAC0001AFE2B68DB0303F4C03320F4C031194372
:10EAD0000C2056E0FFF70FFE2B689B0303F48043E6
:10EAE00020F48041F3E70C2024B9FFF704FEC0F3C3
:10EAF000C120FCE6FFF7FFFD2B68DB0203F4C053E7
:10EB000020F4C051E3E70C2024B9FFF7F4FDC0F373
:10EB1000C310ECE6FFF7EFFD2B68DB0103F4F063B5
:10EB200020F4F061D3E7FFF7E6FD2B681B0103F04B
:10EB3000700320F07001CAE70C2024B9FFF7DBFD59
:10EB400000F00F00D3E6FFF7D6FD2B6820F00F0191
:10EB500003F00F03BBE700BF6425FF1F885EFF1FA4
:10EB600028B90520FFF7C7FDC0F3C030BFE60D2070
:10EB7000FFF7C1FD2B68DB039BB220F40041194372
:10EB80000D20FFF785FDB8E628B90520FFF7B3FD96
:10EB9000C0F34130ABE60D20FFF7ADFD2B685B0302
:10EBA00003F4C04320F4C041E9E728B90520FFF78A
:10EBB000A2FDC0F303209AE60D20FFF79CFD2B6811
:10EBC0001B0203F4706320F47061D8E70D20FFF797
:10EBD00092FD2B685B0103F0600320F06001CEE73B
:10EBE00008B90520AAE70D20FFF785FD2B6820F066
:10EBF0000F0103F00F03C2E728B90620FFF77BFDE2
:10EC0000C0F3004073E60E20FFF775FD2B681B0470
:10EC100003F4803320F48031C8E60E20FFF76BFD4B
:10EC20002B681B0203F4FE4320F4FE41BEE628B924
:10EC30000720FFF760FDC0F3813058E60F20FFF793
:10EC40005AFD2B689B039BB220F4404119430F20CF
:10EC500097E728B90720FFF74EFDC0F3013046E6DD
:10EC60000F20FFF748FD2B681B0303F4405320F4EB
:10EC70004051EBE70F20FFF73EFD2B689B0203F4AA
:10EC8000806320F48061E1E728B90720FFF733FDB6
:10EC9000C0F301202BE60F20FFF72DFD2B681B0290
:10ECA00003F4407320F44071D0E728B90720FFF740
:10ECB00022FDC0F380101AE60F20FFF71CFD2B6821
:10ECC0009B0103F0400320F04001BFE700287FF4E0
:10ECD00046AD0220FFF70FFDC0F3842007E610B910
:10ECE00010F0D4FF03E61968002010F039FF04E6A5
:10ECF0002A681A6101E628B90720FFF7FCFCC0F377
:10ED0000C010F4E50F20FFF7F6FC2B68DB01DBB247
:10ED100020F080019AE728B90420FFF7ECFCC0F34B
:10ED20004030E4E50C20FFF7E6FC2B685B0303F4BE
:10ED3000005320F40051CAE60F20FFF7DCFC2B68DB
:10ED40001B0403F4803320F480317FE700287FF434
:10ED500006AD0F4B1B683BB10220FFF7CCFC800ACD
:10ED600000F478702860C8E50120FFF7C4FCC0F308
:10ED70008920F7E700287FF4F2AC0320FFF7BBFC03
:10ED8000C0B2B4E52A685A60B7E5082402E600BFBD
:10ED90007000FF1F07B5019201AB02460120FFF78B
:10EDA000BFFC03B05DF804FB134602460020B7E445
:10EDB00010B508461446FFF79EFC206010BDF8B55C
:10EDC000364D374C0646E86EE8B9FFF794FC94F8E8
:10EDD0006930C0F3C017BB4215D00E20002F4CD0B5
:10EDE000FFF789FC00F01F00E0720E20FFF783FCA4
:10EDF000237803F01F0320F01F0119430E20FFF7B3
:10EE000047FC84F86970227AD5F88030002A3ED019
:10EE100043F00103627A002A3CD043F00203002051
:10EE2000C5F8803010F0F2FE236994F86A200028BB
:10EE3000B8BF4042984234BF00270127BA4211D0E0
:10EE400098424FF00D002CBF657B257BFFF753FCEC
:10EE500005F00F0520F00F0129430D20FFF718FCE6
:10EE600084F86A70A36C0E4A3146002012F051FB00
:10EE70000020BDE8F84010F03FBDFFF73CFC00F07B
:10EE80001F0020700E20FFF736FCE37AB1E723F075
:10EE90000103BFE723F00203C1E700BF885EFF1F45
:10EEA0006425FF1F0A4810B4836C01F0770444F016
:10EEB000080403EB8403C2F313025A60837A23B974
:10EEC00042EA414010BCFFF7A1BB10BC704700BF35
:10EED0006425FF1F38B5094D01F008020C46A97AD8
:10EEE00051EA020302D12046FFF7EDFBA96C04F0C2
:10EEF0007F0401EB8404606838BD00BF6425FF1FF8
:10EF000038B51F4C636E0D469B680021C5F3074062
:10EF1000984794F86B20A36C03EB820300025860BF
:10EF2000636E00219B68C5F30720984794F86B3007
:10EF3000A26C02EB8302012153681843636E000246
:10EF400050609B68E8B29847A26C94F86B1002EB93
:10EF500081014B6818430011AB0C486010610AD066
:10EF6000C5F34243072B03D1C5F3011184F86B109D
:10EF700043F0080300E0082302EB83035D6038BD23
:10EF80006425FF1FF8B5434C434B444F01262046F0
:10EF90001E6012F09BFAFD686B6803F16802A265BF
:10EFA00003F1880203F59470E26503F5A47203F59A
:10EFB0000273E3642B686265DB68206598472B6801
:10EFC000606DDB6898472B68A06DDB6898472B68FD
:10EFD000E06D1B6998472B68E06CDB6898473B69DC
:10EFE00003F114026266E26C9A61052323704FF408
:10EFF00000304FF47A73636010F096FED4E9141277
:10F00000E36D002010F0E6FC254B2649D3F8902054
:10F01000A264C2F808122449C2F804120021118027
:10F02000224AC3F89C20224AC3F89820214AC3F8F8
:10F030009420214AC3F8A020204AC3F8B420204AD3
:10F04000C3F8B0201F4AC3F8A4201F4AC3F8A82061
:10F050001E4AC3F8C4201E4AC3F8C0201D4AC3F884
:10F06000D0201D4AC3F8CC201C4AC3F8C8201C4A33
:10F07000C3F8DC2032214FF41672C3E9212183F852
:10F080008C60184AC3F8D4200220BDE8F840FFF78E
:10F0900025BA00BF6425FF1F7000FF1FD89D020026
:10F0A000885EFF1FCFE40000A7E5000083E50000B5
:10F0B000A5E50000A1E500009DE50000A9ED000028
:10F0C00095ED0000BDE40000EDE50000C1E60000A4
:10F0D000B1ED0000BFED000079E400006DE5000037
:10F0E000DDE400001DE50000014B00229A6070473E
:10F0F000885EFF1F70B5184E184CF56860682B6865
:10F100009B6998472B68A0699B6898472B68606942
:10F110009B6898472B6820699B6898472B68E06834
:10F120009B6898472B68A0689B6898472B68206A63
:10F130009B6898472B68E0699B6898472B68206814
:10F140009B6898472B6860689B6898473369BDE85F
:10F1500070405B6A184700BFD89D0200DC25FF1F86
:10F16000022870B5144648D005D898B1012835D08A
:10F170000424204670BD03284DD0FF28F8D12A4C26
:10F18000D4F89030D3F804329847A369D3F8043206
:10F19000984714E0126832F0030310D1234B244D3A
:10F1A000DE6868693368D2070BD51B699847246805
:10F1B0003268A86914F0020409D013699847002442
:10F1C000D7E7DB689847336868699B69EEE7D368DF
:10F1D00098473368A8699B699847CAE7134B144D51
:10F1E000DE681468286933680CB11B69E6E7DB68E0
:10F1F0009847336828699B69EEE70C4B0C4DDE6835
:10F2000014683368A868002CEFD1DB68984733682E
:10F21000A8689B69E0E70121064812F01FFB206007
:10F220000028CCD12024A4E7885EFF1FD89D0200CF
:10F23000DC25FF1F0026FF1F0146014812F0CCBB52
:10F240000026FF1F10B50348144612F036FA20605E
:10F2500010BD00BF0026FF1F014812F020BA00BFFA
:10F260000026FF1F08B50448D0F8B822243012F059
:10F27000E5FA002008BD00BFDC25FF1F08B50448E3
:10F28000D0F8B822243012F0BDFA002008BD00BF2B
:10F29000DC25FF1F70B504461D460E46002940F0D0
:10F2A000CA836E2A00F02C825CD8122A00F0718189
:10F2B0002CD8052A00F0058114D8022A00F0CA8053
:10F2C00008D8002A00F0AA80012A00F0B5800424A2
:10F2D000204670BD032A00F0CF80042A00F0D580BC
:10F2E0000424F5E70F2A00F01E8107D8082A00F051
:10F2F000FC800E2A00F004810424E9E7102A00F0C3
:10F300002081112A00F031810424E1E7182A00F05D
:10F310009F8113D8152A00F06C8107D8132A00F0BA
:10F320004681142A00F057810424D1E7162A00F000
:10F330007381172A00F07E810424C9E71B2A00F09C
:10F34000B58107D8192A00F091811A2A00F09C8112
:10F350000424BDE76C2A00F0B7816D2A00F0C28159
:10F360000424B5E77E2A00F0A2822BD8742A00F08C
:10F37000398213D8712A00F0FC8107D86F2A00F077
:10F38000D481702A00F0E7810424A1E7722A00F0FA
:10F390000482732A00F01882042499E7772A00F087
:10F3A0005C8207D8752A00F02B82762A00F03F8213
:10F3B00004248DE77C2A00F05E827D2A00F06982B9
:10F3C000042485E7892A00F0DF8213D8852A00F01B
:10F3D000A78207D8812A00F08282842A00F09782CF
:10F3E000042475E7862A00F0AD82882A00F0B882EE
:10F3F00004246DE7D12A00F0F38207D88A2A00F0AE
:10F40000D982C82A00F0B581042461E7D42A00F02B
:10F41000F582D62A00F0FF82042459E728B9372163
:10F42000A04812F04AF9286052E71A689D4837212F
:10F4300012F035F900244BE728B92121994812F040
:10F440003CF9286044E71A689648212112F027F910
:10F4500000243DE730B92421924812F02EF9001221
:10F46000286035E7186812F09CF9242102468D487F
:10F4700012F015F934462BE7002840F0DE822221F5
:10F48000884812F01AF9286022E7874E18B9D6F892
:10F49000B8322B601CE71B68C6F8B832202106F191
:10F4A000240012F00AF9420740F12482D6F8B8028B
:10F4B00012F077F924210246701812F0F0F80024B7
:10F4C00006E730B92821774812F0F7F88010286055
:10F4D000FEE61A68940DA405002C40F0B08292005C
:10F4E0002821704812F0DBF8F2E6002840F0A982EB
:10F4F0000F216C4812F0E1F800F001002860E7E607
:10F5000030B92021674812F0D8F840002860DFE6C3
:10F510001B686448002B14BF02220122202112F034
:10F52000BEF80024D4E628B925215E4812F0C5F8BB
:10F530002860CDE61A685B48252112F0B0F8344601
:10F54000C6E630B92A21574812F0B7F88010286073
:10F55000BEE61A68940DA405002C40F07482920057
:10F560002A21504812F09BF8B2E630B929214D48C3
:10F5700012F0A3F880102860AAE61A68940DA4057A
:10F58000002C40F0628292002921464812F087F850
:10F590009EE628B92721434812F08FF8286097E6A5
:10F5A0001A684048272112F07AF8344690E630B9BC
:10F5B0002B213C4812F081F88010286088E61A68F8
:10F5C000940DA405002C40F0428292002B21354876
:10F5D00012F065F87CE628B92621324812F06DF861
:10F5E000286075E61A682F48262112F058F8002482
:10F5F0006EE628B92C212B4812F05FF8286067E6E8
:10F600001A68930D9B05002B40F023822C2125487E
:10F6100012F045F800245BE628B92D21214812F0AC
:10F620004CF8286054E61A681E482D2112F037F86D
:10F6300000244DE628B92E211A4812F03EF8286021
:10F6400046E61A6817482E2112F029F800243FE6F2
:10F6500028B92F21134812F030F8286038E61A68CC
:10F6600010482F2112F01BF8344631E628B930211A
:10F670000C4812F022F828602AE61A68094830215E
:10F6800012F00DF8002423E628B93321054812F0C2
:10F6900014F828601CE61A680248332111F0FFFFB5
:10F6A000002415E60026FF1FDC25FF1F28B93421A2
:10F6B000A24812F002F828600AE61A689F4834212E
:10F6C00011F0EDFF344603E628B960219B4811F0A4
:10F6D000F4FF2860FCE51A689848602111F0DFFF0C
:10F6E0000024F5E528B96121944811F0E6FF28606F
:10F6F000EEE51A689148612111F0D1FF0024E7E599
:10F700001C218E4824B911F0D8FF00142860DFE5D1
:10F7100011F0D3FF2A68C0F3080040EA02421C211E
:10F72000864811F0BCFF3446D2E51C21834824B939
:10F7300011F0C3FFC0B22860CAE511F0BEFF2B680C
:10F7400000F47F02C3F308031A431C217B4811F025
:10F75000A6FF0024BCE528B95921784811F0ADFF77
:10F760002860B5E51A687548592111F098FF002402
:10F77000AEE50521714824B911F09FFFC0B22860A1
:10F78000A6E511F09AFF2A7820F0FF000243052138
:10F790006A4811F084FF00249AE5052167482CB9D6
:10F7A00011F08BFFC0F30720286091E511F085FF71
:10F7B0002B681B0220F47F429BB21A4305215F484D
:10F7C00011F06DFF002483E528B95D4B5B6AD3F827
:10F7D0006C312B607CE51A6858485A2111F05FFFA4
:10F7E000002475E528B9564B5B6AD3F870312B605D
:10F7F0006EE51A6851485B2111F051FF344667E508
:10F800004F48436AD3F870311CB9C3F30E032B6021
:10F810005EE52A6823F4FF4323F07F03C2F30E0260
:10F820001A435B21243011F03AFF002450E544488C
:10F83000436AD3F870211CB9C2F307422A6047E536
:10F840002B681B0403F47F0322F47F021A435B211D
:10F85000243011F024FF00243AE528B95E2137480E
:10F8600011F02BFF286033E51A6834485E2111F04F
:10F8700016FF34462CE528B95C21304811F01DFFF5
:10F88000286025E51A682D485C2111F008FF002446
:10F890001EE528B95F21294811F00FFF286017E500
:10F8A0001A6826485F2111F0FAFE002410E50521B0
:10F8B00022482CB911F001FFC0F30740286007E58A
:10F8C00011F0FBFE2B681B0420F47F0203F47F037E
:10F8D0001A430521194811F0E2FE3446F8E448B114
:10F8E0001C684CB10121154811F0B8FF28600028B0
:10F8F00000F0B1800024EBE40721104811F0DDFE98
:10F90000072120F480020D4811F0C9FEE0E4002830
:10F9100040F0A3806521094811F0CFFE2860D7E4AC
:10F920000028E7D10721054811F0C7FEC0F3815038
:10F93000431E584258412860CAE400BF0026FF1FFA
:10F94000DC25FF1F28B95221454811F0B6FE28607A
:10F95000BEE41A684248522111F0A1FE0024B7E427
:10F960004048436AD3F8902114B9D2B22A60AFE478
:10F970002B6822F0FF0203F00F031A4363212430A7
:10F9800011F08DFE0024A3E43648436AD3F8902199
:10F990001CB9C2F303222A609AE42B681B0203F409
:10F9A000706322F470621A436321243011F077FEF1
:10F9B00034468DE42B48436AD3F890211CB9C2F336
:10F9C00007422A6084E42B681B0403F47F0322F4BB
:10F9D0007F021A436321243011F061FE002477E492
:10F9E00028B950211E4811F068FE286070E41A689A
:10F9F0001B48502111F053FE344669E420B9194BDD
:10FA00005B6A9B692B6063E41A681548532111F007
:10FA100046FE00245CE428B91521114811F04DFE82
:10FA2000286055E41B68104A0D485A43152111F00F
:10FA300036FE00244CE408244AE4042448E410245C
:10FA400046E4042444E4102442E4102440E4102456
:10FA50003EE410243CE420243AE4042438E400BFCB
:10FA60000026FF1FDC25FF1F0071020007B5019271
:10FA700001AB02460120FFF70DFC03B05DF804FB6B
:10FA800013460246002005E408B50021024811F0A3
:10FA90009BFE002008BD00BF0026FF1F08B549429D
:10FAA000024811F091FE002008BD00BF0026FF1F94
:10FAB00008B5024811F088FE002008BD0026FF1F8F
:10FAC00038B50A4B0A4CDD6860682B689B6998471B
:10FAD00001200CF001FE2B6860685B69984704F117
:10FAE000240011F046FE012038BD00BFD89D020061
:10FAF000DC25FF1F38B50A4B0A4CDD6860682B68AF
:10FB00009B69984701200CF0E7FD2B6860685B69F2
:10FB1000984704F1240011F019FE012038BD00BF00
:10FB2000D89D0200DC25FF1F08B5024811F04CFEED
:10FB3000002008BD0026FF1F034BD3F8BC32084647
:10FB4000DB681146184700BFDC25FF1FF8B5484C9D
:10FB5000484D494F494BAA69002104F1240011F096
:10FB6000D4FDFE68736803F1E802226203F5847233
:10FB7000E26103F55272A26103F55A72626103F504
:10FB80006272226103F56A7203F57A70E26003F52E
:10FB9000727203F5816323603368A260DB68606082
:10FBA00098473368A069DB68984733686069DB6809
:10FBB000984733682069DB6898473368E068DB68FA
:10FBC00098473368A068DB689847336860685B696A
:10FBD00098473368A0695B699847336860695B69D7
:10FBE0009847336820695B6998473368E0685B69C8
:10FBF00098473368A0685B6998473368206A1B6937
:10FC000098473368E0691B699847336820681B6927
:10FC1000984773683A691A49C4F8BC2203F53273ED
:10FC20005360AB690122C3F8041216491A80C3F865
:10FC30000812154B6B62154B2B62154BEB61154B84
:10FC4000AB62154BEB63154BAB63154BEB62154B7E
:10FC50002B63154BEB64154BAB64154BAB65154B28
:10FC60006B65154B2B66154B2A75EB65F8BD00BF10
:10FC7000DC25FF1F885EFF1FD89D0200B48B0200A9
:10FC8000F5FA0000C1FA000029FB0000B1FA0000FB
:10FC90009DFA000089FA000081FA00006DFA000068
:10FCA0007DF2000065F2000059F2000045F200000C
:10FCB00039F2000061F10000E9F00000F5F0000009
:10FCC000014B00229A607047885EFF1F022870B5C2
:10FCD000144646D004D890B1012833D0042070BD1A
:10FCE00003284CD0FF28F9D1264CD4F89030D3F813
:10FCF00004329847A369D3F80432984714E0126895
:10FD000032F00303EBD1204B204DDE686869336885
:10FD1000D2070BD51B69984724683268A86914F08C
:10FD2000020409D0136998470020D8E7DB68984798
:10FD3000336868699B69EEE7D36898473368A869B8
:10FD40009B69F0E7104B114DDE6814682869336831
:10FD50000CB11B69E7E7DB689847336828699B6942
:10FD6000E1E7094B094DDE6814683368A868002C88
:10FD7000EFD1DB6898473368A8689B69D3E72020F8
:10FD8000ADE700BF885EFF1FD89D0200A828FF1FB7
:10FD900070B5184E184CF56860682B689B699847D9
:10FDA0002B68A0699B6898472B6860699B68984797
:10FDB0002B6820699B6898472B68E0689B68984788
:10FDC0002B68A0689B6898472B68206A9B689847B7
:10FDD0002B68E0699B6898472B6820689B68984768
:10FDE0002B6860689B6898473369BDE870405B6A20
:10FDF000184700BFD89D0200A828FF1F0A460146E9
:10FE0000014811F09CBE00BFCC28FF1F01460148ED
:10FE100011F045BFCC28FF1F10B50348144611F060
:10FE200066FE206010BD00BFCC28FF1F6C2970B596
:10FE30000D46144623D06D2917D0062918D1214B21
:10FE400093F87C20032A2DD00B2A11D19E6F10210C
:10FE5000304610F0DCFDC4F3046220F01F000243C2
:10FE60001021304610F0C5FD02E0174BC3F8B82250
:10FE7000224629461548BDE8704011F02ABE1149B6
:10FE8000D1F8C43091F87C10012919BF0E49D1F87E
:10FE9000B812C2F31302C4F3025118BF01F07F017C
:10FEA0009847E5E79E6F1021304610F094FCC4F3AC
:10FEB000046220F01F0002431021304610F07DFC48
:10FEC000D6E700BF885EFF1FA828FF1FCC28FF1FB2
:10FED00008B50448D0F8BC22243011F06FFF002090
:10FEE00008BD00BFA828FF1F08B50448D0F8BC22F1
:10FEF000243011F047FF002008BD00BFA828FF1FD5
:10FF0000F8B504461D46002940F01E81112A00F074
:10FF1000D08029D8042A7DD00AD8012A62D057B2CD
:10FF2000002F55D0022A63D0032A6FD0042476E034
:10FF30000E2A00F09B800DD8052A00F08880082A40
:10FF4000F4D10028F2D10F21814811F0D0FD00F04A
:10FF5000010053E00F2A00F09B80102AE6D1002810
:10FF600040F09C802A2174E0172A00F0CD8017D839
:10FF7000142A00F0B78009D8122A00F0A580132AAD
:10FF8000D4D1002840F0A6802B2162E0152A00F091
:10FF9000AF80162ACAD1002840F0B3802D2119E085
:10FFA0001A2A00F0C08009D8182A00F0B380192A54
:10FFB000BCD1002840F0B48030210BE01B2A00F0B7
:10FFC000B880D62AB2D1002840F0B980152101E0CE
:10FFD00020B937215E4811F08AFD0FE01A683721F9
:10FFE0005B4830E008B92121F4E71A682121F7E7DE
:10FFF00030B92421564811F07AFD001228600EE035
:020000021000EC
:100000001A68002AB8BF52422421E9E700288DD19E
:100010002221DFE74F4F20B9D7F8BC322B602046B2
:10002000F8BD1B68C7F8BC32202107F1240011F08D
:100030005EFD10F00404F2D0D7F8BC0211F071FE9E
:1000400024210246781811F044FD0024E7E728B97E
:1000500028213F4811F04BFD8010CFE71A68930D1F
:100060009B05002B72D192002821B9E748B92021C5
:10007000374811F03CFD00F00300831E5842584100
:10008000BCE71B68002B14BF022201222021A7E736
:1000900008B925219EE71A682521A1E71A68940D61
:1000A000A405002C52D192002A21294811F011FDFB
:1000B000B5E708B92921CCE71A68940DA405002CEE
:1000C00044D192002921F0E708B9272182E71A6874
:1000D000272185E71A68940DA405002C36D19200DB
:1000E0002B21E2E708B9262174E71A68262177E771
:1000F00008B92C216EE71A68930D9B0533BB2C21A0
:100100006EE71A682D216BE708B92E2162E71A689D
:100110002E2165E708B92F215CE71A682F215FE7D8
:100120001A6830215CE708B9332153E71A68332194
:1001300056E708B934214DE71A68342150E71B68A7
:10014000054A15215A434BE7082468E7102466E75F
:10015000CC28FF1FA828FF1F0071020007B50192DD
:1001600001AB02460120FFF7CBFE03B05DF804FBB4
:10017000134602460020C3E608B50021024811F0EC
:10018000E3FD002008BD00BFCC28FF1F08B5494291
:10019000024811F0D9FD002008BD00BFCC28FF1F88
:1001A00008B5024811F0D0FD002008BDCC28FF1F83
:1001B00038B50A4B0A4CDD6860682B689B69984724
:1001C00001200CF089FA2B6860685B69984704F19C
:1001D000240011F04CFD012038BD00BFD89D020065
:1001E000A828FF1F38B50A4B0A4CDD6860682B68E9
:1001F0009B69984701200CF06FFA2B6860685B6977
:10020000984704F1240011F01FFD012038BD00BF04
:10021000D89D0200A828FF1F70B5114C94F87C30BF
:10022000012B0D4619D0032B0BBF002328230C22D2
:100230000F2242EA433242F0884242F04012042147
:1002400011F047FCD4F89030012D0CBFD3F80432E4
:10025000D3F80832BDE87040184700230B22E8E7C6
:10026000885EFF1FF8B5334CD4E9B032120240EA81
:10027000032042EA1362C4E9B002D4E9B46094F8FE
:10028000C832050E0133000240EA1660DBB23602C6
:1002900084F8C832C4E9B460002949D0042B04D9D9
:1002A0006D2104F1240011F014FCD4F8C02222487E
:1002B0006C2111F00EFC01200CF00EFAD4F8C022D3
:1002C0001D486C2111F005FC00230022C4E9B42371
:1002D00094F8C832042B08D96F21174811F007FC95
:1002E000D4F8D4321843C4F8D4026E21124811F065
:1002F000FEFBD4E9B423C717104394F8C822C2F117
:100300000802D200A2F120063B43C2F12001934033
:1003100000FA06F620FA01F133430B439040C4E99A
:10032000B40300220023C4E9B023002384F8C832B8
:100330002846F8BDA828FF1FCC28FF1F08B5024893
:1003400011F002FD002008BDCC28FF1F034BD3F89D
:10035000D8320846DB681146184700BFA828FF1F9F
:10036000F8B54C4C4C4D4D4BAA694D4F04F1240649
:100370003046002111F047FC4A49304611F08BFC11
:10038000FE68736803F1E802226203F58472E26199
:1003900003F55272A26103F55A72626103F562724B
:1003A000226103F56A7203F57A70E26003F57272F6
:1003B00003F5816323603368A260DB68606098475F
:1003C0003368A069DB68984733686069DB689847E1
:1003D00033682069DB6898473368E068DB689847D2
:1003E0003368A068DB689847336860685B69984742
:1003F0003368A0695B699847336860695B699847AF
:10040000336820695B6998473368E0685B6998479F
:100410003368A0685B6998473368206A1B6998470E
:100420003368E0691B699847336820681B699847FF
:1004300073683A691C49C4F8D82203F532735360D3
:10044000AB690122C3F8041218491A80C3F80812D4
:10045000174BAB66174B6B62174B2B62174BEB615D
:10046000174BAB62174BEB63174BAB63174BEB624E
:10047000174B2B63174BEB64174BAB64174BAB65F8
:10048000174B6B65174B2B66174BEB65174B2A7594
:10049000EB66F8BDA828FF1F885EFF1FB48D020021
:1004A000D89D020019020100E5010100B10101001F
:1004B000650201003D030100A10101008D01010061
:1004C00079010100710101005D010100E9FE0000F8
:1004D000D1FE00002DFE000019FE00000DFE000000
:1004E000CDFC0000C1FC000091FD0000FDFD0000FE
:1004F000014B00229A607047885EFF1F70B5184E4E
:10050000184CF56860682B689B6998472B68A06950
:100510009B6898472B6860699B6898472B6820699F
:100520009B6898472B68E0689B6898472B68A06891
:100530009B6898472B68206A9B6898472B68E069FE
:100540009B6898472B6820689B6898472B68606871
:100550009B6898473369BDE870405B6A184700BFE5
:10056000D89D0200902BFF1F0A460146014811F05A
:10057000A2BC00BFB42BFF1F022870B5144648D0A0
:1005800005D898B1012835D00424204670BD032831
:100590004DD0FF28F8D12A4CD4F89030D3F804324B
:1005A0009847A369D3F80432984714E0126832F0F0
:1005B000030310D1234B244DDE6868693368D207EA
:1005C0000BD51B69984724683268A86914F00204A7
:1005D00009D0136998470024D7E7DB689847336848
:1005E00068699B69EEE7D36898473368A8699B6997
:1005F0009847CAE7134B144DDE68146828693368BE
:100600000CB11B69E6E7DB689847336828699B698A
:10061000EEE70C4B0C4DDE6814683368A868002CBC
:10062000EFD1DB6898473368A8689B69E0E7012150
:10063000064811F04FFD20600028CCD12024A4E70B
:10064000885EFF1FD89D0200902BFF1FB42BFF1F59
:100650000146014811F0FCBDB42BFF1F10B5034843
:10066000144611F000FC206010BD00BFB42BFF1F2A
:100670006C2970B50D46144623D06D2917D0062974
:1006800018D1214B93F87C20032A2DD00B2A11D1AD
:100690009E6F1021304610F0BAF9C4F3046220F0C6
:1006A0001F0002431021304610F0A3F902E0174B5F
:1006B000C3F8B822224629461548BDE8704011F01B
:1006C000C4BB1149D1F8C43091F87C10012919BF7D
:1006D0000E49D1F8B812C2F31302C4F3025118BF85
:1006E00001F07F019847E5E79E6F1021304610F03A
:1006F00072F8C4F3046220F01F0002431021304658
:1007000010F05BF8D6E700BF885EFF1F902BFF1F3D
:10071000B42BFF1F08B50448D0F8BC22243011F0D8
:10072000C9FC002008BD00BF902BFF1F08B504487E
:10073000D0F8BC22243011F0A1FC002008BD00BF7D
:10074000902BFF1F70B504461D460E46002940F051
:10075000EB836F2A00F047825ED8122A00F0768180
:100760002CD8052A00F00A8114D8022A00F0CF8084
:1007700008D8002A00F0AF80012A00F0BA800424D3
:10078000204670BD032A00F0D480042A00F0DA80ED
:100790000424F5E70F2A00F0238107D8082A00F087
:1007A00001810E2A00F009810424E9E7102A00F0F3
:1007B0002581112A00F036810424E1E7182A00F08F
:1007C000A48113D8152A00F0718107D8132A00F0EC
:1007D0004B81142A00F05C810424D1E7162A00F032
:1007E0007881172A00F083810424C9E71B2A00F0CE
:1007F000BB8107D8192A00F096811A2A00F0A1813E
:100800000424BDE76D2A00F0CB8100F2D7816C2A69
:1008100000F0B8810424B3E77D2A00F0B4822BD81D
:10082000752A00F04B8213D8722A00F0148207D880
:10083000702A00F0EE81712A00F0F98104249FE70C
:10084000732A00F01F82742A00F02A82042497E79A
:10085000782A00F06E8207D8762A00F04682772A3E
:1008600000F0598204248BE7792A00F070827C2AF8
:1008700000F07B82042483E7882A00F0EA8213D800
:10088000842A00F0C28207D87E2A00F08A82812A58
:1008900000F09F82042473E7852A00F0BF82862A35
:1008A00000F0C98204246BE7C82A00F0C08107D891
:1008B000892A00F0E2828A2A00F0F58204245FE7A8
:1008C000D42A00F01483D62A00F01E83D12A00F027
:1008D0000083042454E728B93721A14811F0C3FA52
:1008E00028604DE71A689E48372111F0AEFA0024BF
:1008F00046E728B921219A4811F0B5FA28603FE768
:100900001A689748212111F0A0FA002438E730B97D
:100910002421934811F0A7FA0012286030E71868E4
:1009200011F07BFB242102468D4811F08EFA3446EB
:1009300026E7002840F0FA822221894811F093FA34
:1009400028601DE7874E18B9D6F8BC322B6017E730
:100950001B68C6F8BC32202106F1240011F083FA8E
:10096000420740F14182D6F8BC0211F056FB242127
:100970000246701811F069FA002401E730B9282105
:10098000774811F070FA80102860F9E61A68940D23
:10099000A405002C40F0CC8292002821704811F070
:1009A00054FAEDE6002840F0C5820F216C4811F0A2
:1009B0005AFA00F001002860E2E630B920216848C8
:1009C00011F051FA40002860DAE61B686448002BF9
:1009D00014BF02220122202111F037FA0024CFE6B1
:1009E00028B925215E4811F03EFA2860C8E61A6849
:1009F0005B48252111F029FA3446C1E630B92A2195
:100A0000574811F030FA80102860B9E61A68940D42
:100A1000A405002C40F0908292002A21504811F049
:100A200014FAADE630B929214D4811F01CFA8010B6
:100A30002860A5E61A68940DA405002C40F07E827B
:100A400092002921464811F000FA99E628B9272199
:100A5000434811F008FA286092E61A6840482721B6
:100A600011F0F3F934468BE630B92B213C4811F0F4
:100A7000FAF98010286083E61A68940DA405002C0A
:100A800040F05E8292002B21354811F0DEF977E6C6
:100A900028B92621324811F0E6F9286070E61A6874
:100AA0002F48262111F0D1F9002469E628B92C211C
:100AB0002B4811F0D8F9286062E61A68930D9B055F
:100AC000002B40F03F822C21254811F0BEF9002474
:100AD00056E628B92D21224811F0C5F928604FE6C5
:100AE0001A681F482D2111F0B0F9002448E628B9F2
:100AF0002E211B4811F0B7F9286041E61A68184802
:100B00002E2111F0A2F900243AE628B92F21144829
:100B100011F0A9F9286033E61A6811482F2111F065
:100B200094F934462CE628B930210D4811F09BF990
:100B3000286025E61A680A48302111F086F9002459
:100B40001EE628B93321064811F08DF9286017E612
:100B50001A680348332111F078F9002410E600BF29
:100B6000B42BFF1F902BFF1F28B934219F4811F091
:100B70007AF9286004E61A689C48342111F065F976
:100B80003446FDE528B96021984811F06CF92860D9
:100B9000F6E51A689548602111F057F90024EFE551
:100BA00028B96121914811F05EF92860E8E51A68DA
:100BB0008E48612111F049F90024E1E51C218B48A0
:100BC00024B911F050F900142860D9E511F04BF95F
:100BD0002A68C0F3080040EA02421C21834811F051
:100BE00034F90024CCE51C21804824B911F03BF9EC
:100BF000C0B22860C4E511F036F92B6800F47F021A
:100C0000C3F308031A431C21784811F01EF9344637
:100C1000B6E528B95921754811F025F92860AFE5E6
:100C20001A687248592111F010F90024A8E506212C
:100C30006E4824B911F017F9C0B22860A0E511F090
:100C400012F92A7820F0FF0002430621674811F0CC
:100C5000FCF8002494E5062164482CB911F003F94E
:100C6000C0F3072028608BE511F0FDF82B681B020C
:100C700020F47F429BB21A4306215C4811F0E5F84C
:100C800034467DE528B95A4B5B6AD3F86C312B604A
:100C900076E51A6855485A2111F0D7F800246FE517
:100CA00028B9534B5B6AD3F870312B6068E51A683A
:100CB0004E485B2111F0C9F8002461E54C48436AB5
:100CC000D3F870311CB9C3F30E032B6058E52A68C2
:100CD00023F4FF4323F07F03C2F30E021A435B2188
:100CE000243011F0B2F834464AE54148436AD3F85B
:100CF00070211CB9C2F307422A6041E52B681B042E
:100D000003F47F0322F47F021A435B21243011F0A5
:100D10009CF8002434E528B95E21344811F0A3F88A
:100D200028602DE51A6831485E2111F08EF8002404
:100D300026E528B918212D4811F095F828601FE5FF
:100D40001A682A48182111F080F8344618E528B9A5
:100D50001921264811F087F8286011E51A68234800
:100D6000192111F072F800240AE528B95C211F4806
:100D700011F079F8286003E51A681C485C2111F02D
:100D800064F80024FCE428B95F21184811F06BF8DE
:100D90002860F5E41A6815485F2111F056F83446CA
:100DA000EEE4062111482CB911F05DF8C0F30740BC
:100DB0002860E5E411F057F82B681B0420F47F024B
:100DC00003F47F031A430621084811F03EF800247B
:100DD000D6E448B11C686CB10121044811F07AF9DD
:100DE0002860002800F0B0800024C9E4B42BFF1F65
:100DF000902BFF1F0721564811F035F8072120F4EA
:100E00008002534811F021F8BAE4002840F09E8097
:100E100065214F4811F027F82860B1E40028E3D19C
:100E200007214B4811F01FF8C0F38150431E584270
:100E300058412860A4E428B95221454811F013F81C
:100E400028609DE41A684248522110F0FEFF0024F9
:100E500096E44048436AD3F8902114B9D2B22A608C
:100E60008EE42B6822F0FF0203F00F031A43632184
:100E7000243010F0EAFF344682E43648436AD3F85F
:100E800090211CB9C2F303222A6079E42B681B026B
:100E900003F4706322F470621A436321243010F06B
:100EA000D4FF00246CE42B48436AD3F890211CB98A
:100EB000C2F307422A6063E42B681B0403F47F0338
:100EC00022F47F021A436321243010F0BEFF002475
:100ED00056E428B950211E4810F0C5FF28604FE4A1
:100EE0001A681B48502110F0B0FF002448E420B9D4
:100EF000184B5B6ADB692B6042E41A681448532183
:100F000010F0A3FF00243BE428B91521104810F08D
:100F1000AAFF286034E41B680F4A0D485A43152184
:100F200010F093FF00242BE4082429E4042427E490
:100F3000102425E4042423E4102421E410241FE4D5
:100F400010241DE410241BE4202419E4042417E4D5
:100F5000B42BFF1F902BFF1F0071020007B50192F9
:100F600001AB02460120FFF7EDFB03B05DF804FB87
:100F7000134602460020FFF7E5BB08B500210248F2
:100F800011F05EF8002008BDB42BFF1F08B54942E0
:100F9000024811F055F8002008BD00BFB42BFF1F18
:100FA00008B5024811F04CF8002008BDB42BFF1F13
:100FB00038B50A4B0A4CDD6860682B689B69984716
:100FC00001200BF089FB2B6860685B69984704F18E
:100FD000240011F00AF8012038BD00BFD89D02009E
:100FE000902BFF1F38B50A4B0A4CDD6860682B68F0
:100FF0009B69984701200BF06FFB2B6860685B6969
:10100000984704F1240010F0DDFF012038BD00BF37
:10101000D89D0200902BFF1F70B5114C94F87C30C6
:10102000012B0D4619D0032B0BBF002328230C22C4
:101030000F2242EA433242F0884242F04012042139
:1010400010F003FFD4F89030012D0CBFD3F8043218
:10105000D3F80832BDE87040184700230B22E8E7B8
:10106000885EFF1FF8B5334CD4E9B032120240EA73
:10107000032042EA1362C4E9B002D4E9B46094F8F0
:10108000C832050E0133000240EA1660DBB23602B8
:1010900084F8C832C4E9B460002949D0042B04D9CB
:1010A0006D2104F1240010F0D0FED4F8C0222248B3
:1010B0006C2110F0CAFE01200BF00EFBD4F8C02208
:1010C0001D486C2110F0C1FE00230022C4E9B423A6
:1010D00094F8C832042B08D96F21174810F0C3FECA
:1010E000D4F8D4321843C4F8D4026E21124810F058
:1010F000BAFED4E9B423C717104394F8C822C2F14A
:101100000802D200A2F120063B43C2F12001934025
:1011100000FA06F620FA01F133430B439040C4E98C
:10112000B40300220023C4E9B023002384F8C832AA
:101130002846F8BD902BFF1FB42BFF1F08B50248AF
:1011400010F07EFF002008BDB42BFF1F034BD3F827
:10115000D8320846DB681146184700BF902BFF1FA6
:10116000F8B54C4C4C4D4D4BAA694D4F04F124063B
:101170003046002110F003FF4A49304610F049FF85
:10118000FE68736803F1E802226203F58472E2618B
:1011900003F55272A26103F55A72626103F562723D
:1011A000226103F56A7203F57A70E26003F57272E8
:1011B00003F5816323603368A260DB686060984751
:1011C0003368A069DB68984733686069DB689847D3
:1011D00033682069DB6898473368E068DB689847C4
:1011E0003368A068DB689847336860685B69984734
:1011F0003368A0695B699847336860695B699847A1
:10120000336820695B6998473368E0685B69984791
:101210003368A0685B6998473368206A1B69984700
:101220003368E0691B699847336820681B699847F1
:1012300073683A691C49C4F8D82203F532735360C5
:10124000AB690122C3F8041218491A80C3F80812C6
:10125000174BAB66174B6B62174B2B62174BEB614F
:10126000174BAB62174BEB63174BAB63174BEB6240
:10127000174B2B63174BEB64174BAB64174BAB65EA
:10128000174B6B65174B2B66174BEB65174B2A7586
:10129000EB66F8BD902BFF1F885EFF1FB48F020026
:1012A000D89D020019100100E50F0100B10F0100E7
:1012B000651001003D110100A10F01008D0F01001B
:1012C0007B0F0100710F01005D0F01002D07010070
:1012D00015070100710601005D06010051060100BD
:1012E00079050100F1040100FD0401006905010018
:1012F000014B00229A607047885EFF1F70B5184E40
:10130000184CF56860682B689B6998472B68A06942
:101310009B6898472B6860699B6898472B68206991
:101320009B6898472B68E0689B6898472B68A06883
:101330009B6898472B68206A9B6898472B68E069F0
:101340009B6898472B6820689B6898472B68606863
:101350009B6898473369BDE870405B6A184700BFD7
:10136000D89D0200782EFF1F0A460146014811F061
:1013700022B800BF9C2EFF1F022870B5144648D02B
:1013800005D898B1012835D00424204670BD032823
:101390004DD0FF28F8D12A4CD4F89030D3F804323D
:1013A0009847A369D3F80432984714E0126832F0E2
:1013B000030310D1234B244DDE6868693368D207DC
:1013C0000BD51B69984724683268A86914F0020499
:1013D00009D0136998470024D7E7DB68984733683A
:1013E00068699B69EEE7D36898473368A8699B6989
:1013F0009847CAE7134B144DDE68146828693368B0
:101400000CB11B69E6E7DB689847336828699B697C
:10141000EEE70C4B0C4DDE6814683368A868002CAE
:10142000EFD1DB6898473368A8689B69E0E7012142
:10143000064811F0F5F820600028CCD12024A4E75C
:10144000885EFF1FD89D0200782EFF1F9C2EFF1F75
:101450000146014811F0A2B99C2EFF1F10B50348A8
:10146000144610F080FF206010BD00BF9C2EFF1FAF
:101470006C2970B50D46144623D06D2917D0062966
:1014800018D1214B93F87C20032A2DD00B2A11D19F
:101490009E6F102130460FF0BAFAC4F3046220F0B8
:1014A0001F000243102130460FF0A3FA02E0174B51
:1014B000C3F8BC22224629461548BDE8704010F00A
:1014C00044BF1149D1F8C43091F87C10012919BFEB
:1014D0000E49D1F8BC12C2F31302C4F3025118BF73
:1014E00001F07F019847E5E79E6F102130460FF02D
:1014F00072F9C4F3046220F01F0002431021304649
:101500000FF05BF9D6E700BF885EFF1F782EFF1F44
:101510009C2EFF1F08B50448D0F8C022243011F0DB
:101520006FF8002008BD00BF782EFF1F08B50448E3
:10153000D0F8C022243011F047F8002008BD00BFC9
:10154000782EFF1F70B504461D460E46002940F058
:10155000EB836F2A00F047825ED8122A00F0768172
:101560002CD8052A00F00A8114D8022A00F0CF8076
:1015700008D8002A00F0AF80012A00F0BA800424C5
:10158000204670BD032A00F0D480042A00F0DA80DF
:101590000424F5E70F2A00F0238107D8082A00F079
:1015A00001810E2A00F009810424E9E7102A00F0E5
:1015B0002581112A00F036810424E1E7182A00F081
:1015C000A48113D8152A00F0718107D8132A00F0DE
:1015D0004B81142A00F05C810424D1E7162A00F024
:1015E0007881172A00F083810424C9E71B2A00F0C0
:1015F000BB8107D8192A00F096811A2A00F0A18130
:101600000424BDE76D2A00F0CB8100F2D7816C2A5B
:1016100000F0B8810424B3E77D2A00F0B4822BD80F
:10162000752A00F04B8213D8722A00F0148207D872
:10163000702A00F0EE81712A00F0F98104249FE7FE
:10164000732A00F01F82742A00F02A82042497E78C
:10165000782A00F06E8207D8762A00F04682772A30
:1016600000F0598204248BE7792A00F070827C2AEA
:1016700000F07B82042483E7882A00F0EA8213D8F2
:10168000842A00F0C28207D87E2A00F08A82812A4A
:1016900000F09F82042473E7852A00F0BF82862A27
:1016A00000F0C98204246BE7C82A00F0C08107D883
:1016B000892A00F0E2828A2A00F0F58204245FE79A
:1016C000D42A00F01483D62A00F01E83D12A00F019
:1016D0000083042454E728B93721A14810F043FEC1
:1016E00028604DE71A689E48372110F02EFE00242E
:1016F00046E728B921219A4810F035FE28603FE7D7
:101700001A689748212110F020FE002438E730B9EC
:101710002421934810F027FE0012286030E7186853
:1017200010F021FF242102468D4810F00EFE3446B1
:1017300026E7002840F0FA822221894810F013FEA3
:1017400028601DE7874E18B9D6F8C0322B6017E71E
:101750001B68C6F8C032202106F1240010F003FEF9
:10176000420740F14182D6F8C00210F0FCFE24216D
:101770000246701810F0E9FD002401E730B9282175
:10178000774810F0F0FD80102860F9E61A68940D93
:10179000A405002C40F0CC8292002821704810F063
:1017A000D4FDEDE6002840F0C5820F216C4810F012
:1017B000DAFD00F001002860E2E630B92021684837
:1017C00010F0D1FD40002860DAE61B686448002B69
:1017D00014BF02220122202110F0B7FD0024CFE621
:1017E00028B925215E4810F0BEFD2860C8E61A68B9
:1017F0005B48252110F0A9FD3446C1E630B92A2105
:10180000574810F0B0FD80102860B9E61A68940DB2
:10181000A405002C40F0908292002A21504810F03C
:1018200094FDADE630B929214D4810F09CFD8010A3
:101830002860A5E61A68940DA405002C40F07E826D
:1018400092002921464810F080FD99E628B9272109
:10185000434810F088FD286092E61A684048272126
:1018600010F073FD34468BE630B92B213C4810F064
:101870007AFD8010286083E61A68940DA405002C78
:1018800040F05E8292002B21354810F05EFD77E635
:1018900028B92621324810F066FD286070E61A68E3
:1018A0002F48262110F051FD002469E628B92C218B
:1018B0002B4810F058FD286062E61A68930D9B05CE
:1018C000002B40F03F822C21254810F03EFD0024E3
:1018D00056E628B92D21224810F045FD28604FE634
:1018E0001A681F482D2110F030FD002448E628B961
:1018F0002E211B4810F037FD286041E61A68184871
:101900002E2110F022FD00243AE628B92F21144898
:1019100010F029FD286033E61A6811482F2110F0D5
:1019200014FD34462CE628B930210D4810F01BFD7B
:10193000286025E61A680A48302110F006FD0024C8
:101940001EE628B93321064810F00DFD286017E681
:101950001A680348332110F0F8FC002410E600BF99
:101960009C2EFF1F782EFF1F28B934219F4810F0AE
:10197000FAFC286004E61A689C48342110F0E5FC63
:101980003446FDE528B96021984810F0ECFC286049
:10199000F6E51A689548602110F0D7FC0024EFE5C1
:1019A00028B96121914810F0DEFC2860E8E51A684A
:1019B0008E48612110F0C9FC0024E1E51C218B4810
:1019C00024B910F0D0FC00142860D9E510F0CBFC4D
:1019D0002A68C0F3080040EA02421C21834810F044
:1019E000B4FC0024CCE51C21804824B910F0BBFCD9
:1019F000C0B22860C4E510F0B6FC2B6800F47F028A
:101A0000C3F308031A431C21784810F09EFC3446A7
:101A1000B6E528B95921754810F0A5FC2860AFE556
:101A20001A687248592110F090FC0024A8E506219C
:101A30006E4824B910F097FCC0B22860A0E510F001
:101A400092FC2A7820F0FF0002430621674810F03C
:101A50007CFC002494E5062164482CB910F083FC3A
:101A6000C0F3072028608BE510F07DFC2B681B027B
:101A700020F47F429BB21A4306215C4810F065FCBB
:101A800034467DE528B95A4B5B6AD3F86C312B603C
:101A900076E51A6855485A2110F057FC00246FE586
:101AA00028B9534B5B6AD3F870312B6068E51A682C
:101AB0004E485B2110F049FC002461E54C48436A24
:101AC000D3F870311CB9C3F30E032B6058E52A68B4
:101AD00023F4FF4323F07F03C2F30E021A435B217A
:101AE000243010F032FC34464AE54148436AD3F8CA
:101AF00070211CB9C2F307422A6041E52B681B0420
:101B000003F47F0322F47F021A435B21243010F098
:101B10001CFC002434E528B95E21344810F023FC75
:101B200028602DE51A6831485E2110F00EFC002473
:101B300026E528B918212D4810F015FC28601FE56E
:101B40001A682A48182110F000FC344618E528B914
:101B50001921264810F007FC286011E51A6823486F
:101B6000192110F0F2FB00240AE528B95C211F4876
:101B700010F0F9FB286003E51A681C485C2110F09E
:101B8000E4FB0024FCE428B95F21184810F0EBFBCB
:101B90002860F5E41A6815485F2110F0D6FB34463A
:101BA000EEE4062111482CB910F0DDFBC0F307402C
:101BB0002860E5E410F0D7FB2B681B0420F47F02BB
:101BC00003F47F031A430621084810F0BEFB0024EB
:101BD000D6E448B11C686CB10121044810F020FD26
:101BE0002860002800F0B0800024C9E49C2EFF1F6C
:101BF000782EFF1F0721564810F0B5FB072120F46F
:101C00008002534810F0A1FBBAE4002840F09E8007
:101C100065214F4810F0A7FB2860B1E40028E3D10C
:101C200007214B4810F09FFBC0F38150431E5842E0
:101C300058412860A4E428B95221454810F093FB8C
:101C400028609DE41A684248522110F07EFB00246F
:101C500096E44048436AD3F8902114B9D2B22A607E
:101C60008EE42B6822F0FF0203F00F031A43632176
:101C7000243010F06AFB344682E43648436AD3F8D5
:101C800090211CB9C2F303222A6079E42B681B025D
:101C900003F4706322F470621A436321243010F05D
:101CA00054FB00246CE42B48436AD3F890211CB900
:101CB000C2F307422A6063E42B681B0403F47F032A
:101CC00022F47F021A436321243010F03EFB0024EB
:101CD00056E428B950211E4810F045FB28604FE417
:101CE0001A681B48502110F030FB002448E420B94A
:101CF000184B5B6ADB692B6042E41A681448532175
:101D000010F023FB00243BE428B91521104810F003
:101D10002AFB286034E41B680F4A0D485A431521FA
:101D200010F013FB00242BE4082429E4042427E406
:101D3000102425E4042423E4102421E410241FE4C7
:101D400010241DE410241BE4202419E4042417E4C7
:101D50009C2EFF1F782EFF1F0071020007B5019215
:101D600001AB02460120FFF7EDFB03B05DF804FB79
:101D7000134602460020FFF7E5BB08B500210248E4
:101D800010F004FC002008BD9C2EFF1F08B549423E
:101D9000024810F0FBFB002008BD00BF9C2EFF1F77
:101DA00008B5024810F0F2FB002008BD9C2EFF1F72
:101DB00038B50A4B0A4CDD6860682B689B69984708
:101DC00001200AF089FC2B6860685B69984704F180
:101DD000240010F0B0FB012038BD00BFD89D0200E8
:101DE000782EFF1F38B50A4B0A4CDD6860682B68F7
:101DF0009B69984701200AF06FFC2B6860685B695B
:101E0000984704F1240010F083FB012038BD00BF87
:101E1000D89D0200782EFF1FF8B5334CD4E9B232BA
:101E2000120240EA032042EA1362C4E9B202D4E992
:101E3000B66094F8D032050E0133000240EA166015
:101E4000DBB2360284F8D032C4E9B660002949D04A
:101E5000042B04D96D2104F1240010F076FAD4F893
:101E6000C82222486C2110F070FA01200AF034FCDC
:101E7000D4F8C8221D486C2110F067FA0023002214
:101E8000C4E9B62394F8D032042B08D96F2117483F
:101E900010F069FAD4F8DC321843C4F8DC026E2181
:101EA000124810F060FAD4E9B623C717104394F82B
:101EB000D022C2F10802D200A2F120063B43C2F1B7
:101EC0002001934000FA06F620FA01F133430B4358
:101ED0009040C4E9B60300220023C4E9B2230023E2
:101EE00084F8D0322846F8BD782EFF1F9C2EFF1FA5
:101EF00070B51A4C94F87C30012B05460E4625D05F
:101F0000032B0BBF002328230C220F2242EA43326B
:101F100042F0884242F040120421284610F015FA9F
:101F2000012E16D103220521284610F00EFA0022B8
:101F30000621284610F009FA284610F0C1FAD4F814
:101F40009030D3F80432BDE87040184700230B22CC
:101F5000DCE7D4F89030D3F80832F4E7885EFF1F4E
:101F600008B5024810F012FB002008BD9C2EFF1F90
:101F7000034BD3F8E0320846DB681146184700BF30
:101F8000782EFF1FF8B54C4C4C4D4D4BAA694D4F68
:101F900004F124063046002110F071FA4A49304617
:101FA00010F0DDFAFE68736803F1E802226203F5BF
:101FB0008472E26103F55272A26103F55A726261A2
:101FC00003F56272226103F56A7203F57A70E260CA
:101FD00003F5727203F5816323603368A260DB68E6
:101FE000606098473368A069DB6898473368606928
:101FF000DB68984733682069DB6898473368E06896
:10200000DB6898473368A068DB6898473368606886
:102010005B6998473368A0695B6998473368606972
:102020005B699847336820695B6998473368E06863
:102030005B6998473368A0685B6998473368206A92
:102040001B6998473368E0691B69984733682068C3
:102050001B69984773683A691C49C4F8E02203F584
:1020600032735360AB690122C3F8041218491A8015
:10207000C3F80812174BAB66174B6B62174B2B62FA
:10208000174BEB61174BAB62174BEB63174BAB6313
:10209000174BEB62174B2B63174BEB64174BAB647F
:1020A000174BAB65174B6B65174B2B66174BEB65E7
:1020B000174B2A75EB66F8BD782EFF1F885EFF1F51
:1020C000B4910200D89D0200F11E0100E51D01003F
:1020D000B11D0100191E0100611F0100A11D0100B9
:1020E0008D1D01007B1D0100711D01005D1D0100A2
:1020F0002D15010015150100711401005D1401007A
:102100005114010079130100F1120100FD120100C8
:10211000691301000020704701207047014B002225
:102120009A607047885EFF1F10B50020144610F0BB
:102130007BFB206010BD002010F098BB10B504465A
:1021400018B910F08FFC204610BD0820FCE710B530
:10215000044618B910F068FC204610BD0820FCE7C2
:102160000021F4E74942F2E7F1E738B504461D469D
:10217000002940F03C87043AFA2A00F23B87DFE866
:1021800012F0FB00390739073907390739073907D2
:10219000390739073907390739073907390739073F
:1021A000390739073907390739073907390739072F
:1021B000390739073907390739073907390739071F
:1021C000390739073907390739073907390739070F
:1021D0003907390739073907390739073907090135
:1021E0001901390729013901390739073907390731
:1021F00039073907390739073907390739073907DF
:1022000039073907390739073907390739073907CE
:1022100039073907390739073907390739073907BE
:1022200039073907390739073907390739073907AE
:10223000390739073907390739073907390739079E
:102240003907490157016501730181018F019D0122
:10225000AB01B901C701D501E301F101FF010D0295
:102260001B02290233023D023907470251025B0279
:1022700065026F027E028D029C02A50239073907B2
:102280003907AE02B602BE02C802D20239073907C8
:102290003907DA02E202EA02390739073907390752
:1022A000390739073907F402FE0208031203390718
:1022B000390739073907390739071C032603300363
:1022C0003A034403390739073907390739074E03F9
:1022D00058036803780380038C0396039F03A903C4
:1022E000B003BB03C803D503E203EF03FC030904F7
:1022F0001604390723042E043B04480453046004E5
:102300006D047A0487049404A304B204C104D004C5
:10231000DF04EE04FD040D051F052F053F054F05E5
:102320005F056F057F058F059F05AF05BF05CE05CE
:10233000390739073907390739073907390739079D
:10234000390739073907DD05ED05FD050D061D06C1
:102350002D063D064D065D066C067B068A0699062F
:10236000A806B706C606D506E306F106FF06390736
:102370000D07180726072E0728B9602110F054FA18
:102380002860204638BD2A686021002010F06EFACF
:102390000024F6E730B90246082110F087FA00B2AF
:1023A0002860EEE700222B880821104610F08BFAF7
:1023B0000024E6E730B90246092110F077FA00B2AE
:1023C0002860DEE700222B880921104610F07BFAF6
:1023D0000024D6E730B90122082110F067FA00B2D4
:1023E0002860CEE72B8801220821002010F06BFA2C
:1023F0000024C6E730B90122092110F057FA00B2D3
:102400002860BEE72B8801220921002010F05BFA2A
:102410000024B6E7002840F0F0850122032110F0E7
:1024200025FA22460221204610F040FA2860A8E74B
:10243000002840F0E5850122032110F017FA01225F
:102440000221204610F032FA28609AE7002840F076
:10245000DA850222032110F009FA224602212046E1
:1024600010F024FA28608CE7002840F0CF8502465F
:10247000032110F0FBF922460221204610F016FA43
:1024800028607EE7002840F0C4850246032110F052
:10249000EDF901220221204610F008FA286070E7C9
:1024A000002840F0B9850322114610F0DFF92246DA
:1024B0000221204610F0FAF9286062E7002840F077
:1024C000AE850422032110F0D1F9224602212046D4
:1024D00010F0ECF9286054E7002840F0A3850422AE
:1024E000032110F0C3F901220221204610F0DEF989
:1024F000286046E7002840F098850522032110F067
:10250000B5F922460221204610F0D0F9286038E7BC
:10251000002840F08D850522032110F0A7F9012243
:102520000221204610F0C2F928602AE7002840F076
:1025300082850622032110F099F9224602212046C5
:1025400010F0B4F928601CE7002840F077850722D6
:10255000032110F08BF922460221204610F0A6F943
:1025600028600EE7002840F06C850722032110F058
:102570007DF901220221204610F098F9286000E739
:10258000002840F061850822032110F06FF92246EF
:102590000221204610F08AF92860F2E6002840F077
:1025A00056850822032110F061F9012202212046FC
:1025B00010F07CF92860E4E6002840F04B85092201
:1025C000032110F053F922460221204610F06EF943
:1025D0002860D6E6002840F040850246122110F01F
:1025E00065F900B22860CCE6002840F03985012268
:1025F000122110F05BF900B22860C2E6002840F01A
:1026000032850246132110F051F900B22860B8E675
:10261000002840F02B850246152110F047F900B242
:102620002860AEE6002840F024850122152110F034
:102630003DF900B22860A4E6002840F01D8502465E
:10264000162110F033F900B228609AE6002840F015
:1026500016850122162110F029F900B2286090E6B3
:10266000002840F00F850A22032110F0FFF82246CF
:102670000221204610F01AF900B2286081E60028F5
:1026800040F003850A22032110F0F0F80122022114
:10269000204610F00BF900B2286072E6002840F0E6
:1026A000F7840B22032110F0E1F822460221204694
:1026B00010F0FCF800B2286063E6002840F0EB84DC
:1026C0000246062110F0F2F828605AE6002840F091
:1026D000E5840122062110F0E9F8286051E600287F
:1026E00040F0DF84412110F09FF8286049E600287F
:1026F00040F0DA84422110F097F8286041E6002883
:1027000040F0D5840122462110F0D0F800B22860B4
:1027100037E6002840F0CE840246462110F0C6F885
:1027200000B228602DE6002840F0C784472110F051
:102730007BF8286025E6002840F0C284212110F0B3
:1027400073F828601DE6002840F0BD84222110F0B7
:102750006BF8286015E6002840F0B8840246232173
:1027600010F0A4F800B228600BE6002840F0B18415
:10277000272110F059F820F07F40286001E600285A
:1027800040F0AA84282110F04FF820F07F40286004
:10279000F7E5002840F0A38401222A2110F086F8F2
:1027A00000B22860EDE5002840F09C8402462A2112
:1027B00010F07CF800B22860E3E5002840F0958432
:1027C0000246392110F072F800B22860D9E50028DD
:1027D00040F08E840122392110F068F800B22860A0
:1027E000CFE5002840F0878402463D2110F05EF8D6
:1027F00000B22860C5E5002840F0808402463F21F1
:1028000010F054F800B22860BBE5002840F079844D
:1028100002463A2110F04AF800B22860B1E50028DB
:1028200040F072840246532110F040F800B2286054
:10283000A7E530B90122642110F038F800B2286011
:102840009FE52B8801226421002010F03CF8002431
:1028500097E530B90246642110F028F800B22860EC
:102860008FE500222B886421104610F02CF80024FC
:1028700087E5002840F04B8466210FF0D5FF2860E3
:102880007FE520B968210FF0CFFF286079E529683E
:10289000002010F0E7F8002473E5002840F03A84A7
:1028A0000122692110F002F800B2286069E50028D1
:1028B00040F03384C14B598910F069F8286060E515
:1028C000002840F02D84024669210FF0EFFF00B28E
:1028D000286056E5002840F0268410F0BEF82860F5
:1028E0004FE518B910F0E3F828604AE529680020A0
:1028F00010F0D9F8002444E5002840F0178402467F
:102900006D210FF0B3FF6C2120460FF08DFF286082
:1029100037E5002840F00D8401226D210FF0A6FF5D
:102920006C2120460FF080FF28602AE5002840F047
:10293000038402226D210FF099FF6C2120460FF0D5
:1029400073FF28601DE5002840F0F98303226D2104
:102950000FF08CFF6C2120460FF066FF286010E519
:10296000002840F0EF8304226D210FF07FFF6C21DF
:1029700020460FF059FF286003E5002840F0E5836A
:1029800005226D210FF072FF6C2120460FF04CFFE5
:102990002860F6E4002840F0DB8306226D210FF06A
:1029A00065FF6C2120460FF03FFF2860E9E4002816
:1029B00040F0D18307226D210FF058FF6C21204693
:1029C0000FF032FF2860DCE418B90FF0B1FF286087
:1029D000D7E4296800200FF09DFF0024D1E4774B55
:1029E000598918B90FF0CAFF2860CAE42A68002084
:1029F0000FF0B2FF0024C4E4002840F0AF830122AE
:102A00006F210FF033FF6E2120460FF00DFF28607D
:102A1000B7E418B910F015F82860B2E4296800206E
:102A200010F002F80024ACE4002840F09A8303225E
:102A30006F210FF01BFF6E2120460FF0F5FE28607E
:102A40009FE4002840F0908304226F210FF00EFFD6
:102A50006E2120460FF0E8FE286092E4002840F046
:102A6000868305226F210FF001FF6E2120460FF0B3
:102A7000DBFE286085E4002840F07C8306226F217D
:102A80000FF0F4FE6E2120460FF0CEFE286078E4B1
:102A9000002840F0728307226F210FF0E7FE6E21BD
:102AA00020460FF0C1FE28606BE4002840F06883E8
:102AB00008226F210FF0DAFE22466E2120460FF029
:102AC000F5FE00B228605CE4002840F05C83082238
:102AD0006F210FF0CBFE01226E2120460FF0E6FEA3
:102AE00000B228604DE4002840F0508309226F2195
:102AF0000FF0BCFE22466E2120460FF0D7FE00B23A
:102B000028603EE4002840F044830A226F210FF041
:102B1000ADFE22466E2120460FF0C8FE00B22860AE
:102B20002FE4002840F038830A226F210FF09EFE28
:102B300001226E2120460FF0B9FE00B2286020E489
:102B4000002840F02C830B226F210FF08FFE2246CD
:102B50006E2120460FF0AAFE00B2286011E4002882
:102B600040F020830B226F210FF080FE01226E21A6
:102B700020460FF09BFE00B2286002E4002840F0DF
:102B800014830C226F210FF071FE22466E21204625
:102B90000FF08CFE00B22860FFF7F3BB002840F076
:102BA00007830C226F210FF061FE01226E21204667
:102BB0000FF07CFE00B22860FFF7E3BB0065FF1F4B
:102BC000002840F0F8820D226F210FF04FFE2246C0
:102BD0006E2120460FF06AFE00B22860FFF7D1BBDD
:102BE000002840F0EB820D226F210FF03FFE012202
:102BF0006E2120460FF05AFE00B22860FFF7C1BBDD
:102C0000002840F0DE820E226F210FF02FFE2246B8
:102C10006E2120460FF04AFE00B22860FFF7B1BBDC
:102C2000002840F0D1820E226F210FF01FFE0122FA
:102C30006E2120460FF03AFE00B22860FFF7A1BBDC
:102C4000002840F0C4820F226F210FF00FFE2246B1
:102C50006E2120460FF02AFE00B22860FFF791BBDC
:102C6000002840F0B7820F226F210FF0FFFD0122F4
:102C70006E2120460FF01AFE00B22860FFF781BBDC
:102C8000002840F0AA8210226F210FF0EFFD2246AB
:102C90006E2120460FF00AFE00B22860FFF771BBDC
:102CA000002840F09D8211226F210FF0DFFD2246A7
:102CB0006E2120460FF0FAFD00B22860FFF761BBDD
:102CC000002840F0908211226F210FF0CFFD0122E9
:102CD0006E2120460FF0EAFD00B22860FFF751BBDD
:102CE000002840F0838212226F210FF0BFFD2246A0
:102CF0006E2120460FF0DAFD00B22860FFF741BBDD
:102D0000002840F0768213226F210FF0AFFD22469B
:102D10006E2120460FF0CAFD2860FFF732BB002865
:102D200040F06A8213226F210FF0A0FD01226E2174
:102D300020460FF0BBFD2860FFF723BB002840F0C2
:102D40005E82C0226F210FF091FD22466E21204647
:102D50000FF0ACFD00B22860FFF713BB002840F075
:102D60005182C0226F210FF081FD01226E21204689
:102D70000FF09CFD00B22860FFF703BB002840F075
:102D80004482C1226F210FF071FD22466E21204640
:102D90000FF08CFD00B22860FFF7F3BA002840F076
:102DA0003782C1226F210FF061FD01226E21204682
:102DB0000FF07CFD00B22860FFF7E3BA002840F076
:102DC0002A82C2226F210FF051FD22466E21204639
:102DD0000FF06CFD00B22860FFF7D3BA002840F076
:102DE0001D82C2226F210FF041FD01226E2120467B
:102DF0000FF05CFD00B22860FFF7C3BA002840F076
:102E00001082C3226F210FF031FD22466E21204631
:102E10000FF04CFD00B22860FFF7B3BA002840F075
:102E20000382C3226F210FF021FD01226E21204673
:102E30000FF03CFD00B22860FFF7A3BA002840F075
:102E4000F681C4226F210FF011FD22466E2120462B
:102E50000FF02CFD2860FFF794BA002840F0EA81BB
:102E6000C4226F210FF002FD01226E2120460FF0D7
:102E70001DFD2860FFF785BA002840F0DE81C522DD
:102E80006F210FF0F3FC22466E2120460FF00EFD5D
:102E90002860FFF776BA002840F0D281C5226F2162
:102EA0000FF0E4FC01226E2120460FF0FFFC2860A9
:102EB000FFF767BA002840F0C681C6226F210FF0E5
:102EC000D5FC22466E2120460FF0F0FC2860FFF76B
:102ED00058BA002840F0BA81C6226F210FF0C6FC14
:102EE00001226E2120460FF0E1FC2860FFF749BA6D
:102EF000002840F0AE81C7226F210FF0B7FC2246B8
:102F00006E2120460FF0D2FC2860FFF73ABA002865
:102F100040F0A281C7226F210FF0A8FC01226E2190
:102F200020460FF0C3FC2860FFF72BBA002840F0C2
:102F30009681C8226F210FF099FC6E2120460FF078
:102F400073FC2860FFF71DBA002840F08B81C9226E
:102F50006F210FF08BFC6E2120460FF065FC28607E
:102F6000FFF70FBA002840F08081CA226F210FF0CE
:102F70007DFC6E2120460FF057FC2860FFF701BA58
:102F8000002840F07581CB226F210FF06FFC6E217D
:102F900020460FF049FC2860FFF7F3B9B94B18B988
:102FA0005B892B60FFF7EDB92A685A810024FFF78F
:102FB000E8B920B9B34B5B7A2B60FFF7E2B9B24AAC
:102FC0002878511C0FF06AFE0024FFF7DAB90028B8
:102FD00040F05181AB4B1B7A2B60FFF7D2B9002830
:102FE00040F04C81A74BDB882B60FFF7CAB908245F
:102FF000FFF7C7B90424FFF7C4B90424FFF7C1B928
:103000000424FFF7BEB90424FFF7BBB90424FFF77B
:10301000B8B90424FFF7B5B90424FFF7B2B9042402
:10302000FFF7AFB90424FFF7ACB90424FFF7A9B93F
:103030000424FFF7A6B90424FFF7A3B90424FFF77B
:10304000A0B90424FFF79DB90424FFF79AB904241A
:10305000FFF797B90424FFF794B90424FFF791B957
:103060000424FFF78EB90424FFF78BB90424FFF77B
:1030700088B90424FFF785B90424FFF782B9042432
:10308000FFF77FB90424FFF77CB90424FFF779B96F
:103090000424FFF776B90424FFF773B90424FFF77B
:1030A00070B90424FFF76DB90424FFF76AB904244A
:1030B000FFF767B90424FFF764B90424FFF761B987
:1030C0000424FFF75EB90424FFF75BB90424FFF77B
:1030D00058B90424FFF755B90424FFF752B9042462
:1030E000FFF74FB90424FFF74CB90424FFF749B99F
:1030F0000424FFF746B90424FFF743B90424FFF77B
:1031000040B90424FFF73DB90424FFF73AB9042479
:10311000FFF737B90424FFF734B90424FFF731B9B6
:103120000424FFF72EB90424FFF72BB90424FFF77A
:1031300028B90424FFF725B90424FFF722B9042491
:10314000FFF71FB90424FFF71CB90424FFF719B9CE
:103150000424FFF716B90424FFF713B90424FFF77A
:1031600010B90424FFF70DB90424FFF70AB90424A9
:10317000FFF707B90424FFF704B90424FFF701B9E6
:103180000424FFF7FEB80424FFF7FBB80424FFF77C
:10319000F8B80424FFF7F5B80424FFF7F2B80424C4
:1031A000FFF7EFB80424FFF7ECB80424FFF7E9B801
:1031B0000424FFF7E6B80424FFF7E3B80424FFF77C
:1031C000E0B80424FFF7DDB80424FFF7DAB80424DC
:1031D000FFF7D7B80424FFF7D4B80424FFF7D1B819
:1031E0000424FFF7CEB80424FFF7CBB80424FFF77C
:1031F000C8B80424FFF7C5B80424FFF7C2B80424F4
:10320000FFF7BFB80424FFF7BCB80424FFF7B9B830
:103210000424FFF7B6B80424FFF7B3B80424FFF77B
:10322000B0B80424FFF7ADB80424FFF7AAB804240B
:10323000FFF7A7B80424FFF7A4B80424FFF7A1B848
:103240000424FFF79EB80424FFF79BB80424FFF77B
:1032500098B80424FFF795B80424FFF792B8042423
:10326000FFF78FB80424FFF78CB80424FFF789B860
:103270000424FFF786B80424FFF783B80424FFF77B
:1032800080B800BF0065FF1F0865FF1F07B50192EA
:1032900001AB02460120FEF768FF03B05DF804FBB6
:1032A000134602460020FEF760BF022804BF0C4B05
:1032B00093F8F00030B90B4BDB681B689B690A4A36
:1032C00010681847012809D1054B93F8F030012BFD
:1032D00004D1044BDB681B685B69F0E7704700BFF3
:1032E000885EFF1FD89D02006831FF1F10B50020C7
:1032F000FFF7DBFF044B054ADB6810681B68BDE87D
:1033000010409B69184700BFD89D02006831FF1F1D
:103310001FB5084B33F8081C0291991E019133F830
:10332000041C00915A78014600200FF0ADFC05B056
:103330005DF804FB0865FF1F10B5044620B9096855
:103340000FF09DFB204610BD0820FCE738B50D4668
:10335000044620B90FF081FB2860204638BD0820C4
:10336000FCE70120704710B40C4630B9044B5B6891
:1033700020469B6810BC11461847002010BC7047BF
:103380006831FF1F70B5274E274DF46860682368C9
:103390006830DB68286098470120FFF786FF636884
:1033A00032696A6003F532735360204B20499A6991
:1033B000C2F804121F49C2F80812002111801E4AE7
:1033C0005A621E4A1A621E4ADA611E4A9A621E4AEE
:1033D0001A651E4ADA631E4A9A631E4ADA621E4A58
:1033E0001A631E4ADA641E4A9A641E4A9A651E4A85
:1033F0005A651E4A5A661E4A1A6601221A751D4AE5
:10340000DA65322040F28A22C3E903201A4B4FF4D6
:103410007A729A8041F270721A6059724FF4807217
:103420005A8170BDD89D02006831FF1F885EFF1F62
:1034300019210100633301004F21010069210100BE
:1034400065210100612101004D330100A13201001D
:103450008D3201003D210100393301003721010087
:10346000292101001133010015210100AB320100B7
:103470001D210100ED3201000065FF1F0020704793
:10348000014B00229A607047885EFF1F00200FF0FA
:1034900035BC10B5002014460FF00EFC206010BDA6
:1034A000022804BF0B4B93F8F00030B90A4BDB68DD
:1034B0001B689B69094A10681847012809D1054B08
:1034C00093F8F030012B04D1034BDB681B685B6978
:1034D000F0E77047885EFF1FD89D02007C31FF1F18
:1034E00010B50020FFF7DCFF044B054ADB681068CD
:1034F0001B68BDE810409B69184700BFD89D0200BB
:103500007C31FF1F08B50022104617210FF0F6FB93
:10351000002210461A210FF0F1FB41F61912192171
:103520000020BDE808400FF0E9BB08B5FFF7EAFF4F
:10353000012008BD08B5FFF7E5FF012008BD38B53B
:103540000D46044620B90FF012FD2860204638BD14
:103550000820FCE7F0B53D4B3D4D33F8062C85B017
:103560009C1F0292221D019262880092064601462B
:10357000E27900200FF012FE6B68B34224D105B04F
:10358000F0BD022B15D1334F20460CF04BFE2269C3
:103590003B689A4258D0662100200FF0AFFB2369A8
:1035A0003B606B2100200FF087FB0023A0602362AB
:1035B0004AE0012B48D1F4E76B2138460FF07CFB41
:1035C0002761A06027623FE000200FF0D0FC0823B5
:1035D000009301460323E26804F110000CF036FD6D
:1035E0000122E060692100200FF0A8FB00F5F943FB
:1035F0007F339BB24FF6FE1293420ED82389B4F963
:10360000182001B2594348BFFF3108230093091223
:10361000042311480CF01AFD2083104C94F82470F8
:10362000002FC9D00E4B1B78032BAAD10D4F20467B
:103630000CF02AFEA2683B689A4205D0682100205F
:103640000FF05CFBA3683B606E6098E70665FF1FA8
:103650007C31FF1F2C65FF1F2065FF1FD864FF1FF3
:103660002865FF1F3065FF1F70B50E46E0B90F4D8E
:1036700095F82440A4B10E4C2278012A02D10FF013
:1036800076FC28610321002021700FF07BFB6B2169
:1036900000200FF011FB336818446860002070BDF3
:1036A00009680FF076FCF9E70820F8E7D864FF1FF7
:1036B0002865FF1F70B50E46A8B90C4D95F824403B
:1036C00074B10B4C2278012A02D10FF050FC286112
:1036D0000321002021700FF055FB6E60002070BDAB
:1036E0000FF04AFCFAE70820F9E700BFD864FF1F93
:1036F0002865FF1F70B50E46A8B90C4D95F82440FB
:1037000074B10B4C2278012A02D10FF030FC2861F1
:103710000221002021700FF035FBEE60002070BD0B
:103720000FF015FCFAE70820F9E700BFD864FF1F87
:103730002865FF1F0021DDE74942DBE7DAE738B5FE
:1037400015460C4600295FD1AC283DD014D80C2872
:1037500036D006D8042825D00B282AD004242046A9
:1037600038BD0D28FBD0AB28F8D193B201226421DB
:1037700020460FF0F0FAF2E7BE2839D008D8B32877
:1037800025D0BD28EAD1114620460FF00BFBE6E715
:10379000FB2836D0FC28E1D11C4AE8B2511C0FF0BE
:1037A00007FDDCE7602120460FF0A8FA184B1D60EA
:1037B000D5E75F2120460FF0A1FA154B5D61CEE7FA
:1037C000134B83F82420CAE793B20A46CFE76B2154
:1037D00020460FF093FA0F4B1B78032BBFD10C4BF5
:1037E0002A46C3E90155682120460FF087FAB6E75B
:1037F000094B204619890FF002FB064B01221A7073
:10380000ADE7054B1A81AAE70824A8E70665FF1F64
:10381000D864FF1F2865FF1F0065FF1F38B51546D8
:103820000C46002940F08D80B22875D022D8AB28F4
:1038300061D014D80B284BD004D8042840D00424DD
:10384000204638BD0C284BD00D28F8D13E4B93F8BC
:103850002420002A49D01B692B600024F0E7AD2802
:1038600053D050D3AE2855D0B028E8D1374BB3F958
:10387000183038E0C0285CD013D8BD284FD005D808
:10388000B328DCD108460FF09CFB3AE0BE284AD0B2
:10389000BF28D4D101226F2120460FF02FFA6E21CC
:1038A00034E0FC2847D004D8FB28C8D1274B1B891B
:1038B00019E0FD2842D0FE28C1D1244B9B8812E09C
:1038C000602120460FF0F8F91F4B28601860B7E719
:1038D0005F2120460FF0F0F91B4B28605861AFE7DD
:1038E000194B93F824302B60AAE7662100200FF0D3
:1038F000E3F92860B1E70122642120460FF01EFAA7
:1039000000B228609CE70A46F6E7662120460FF0E1
:10391000D3F9F6E76821F9E70C4BDB68E3E70846E3
:103920000FF04EFAEDE7094B204619890FF079FAAE
:10393000E7E70222AFE7054BDB79D4E7034B9B793E
:10394000D1E708247CE700BFD864FF1F0065FF1F94
:1039500010B40C4630B9054B9B6820469B6810BCE0
:1039600011461847002010BC704700BF7C31FF1F74
:1039700070B5444E444DF468606823686830DB6875
:10398000286098470120FFF78BFD63683269AA60C1
:1039900003F5327353603D4B3D499A693D4DC2F882
:1039A00004123D49C2F80812012111803B4A5A62B3
:1039B0003B4A1A623B4ADA613B4A9A623B4A1A65C1
:1039C0003B4ADA633B4A9A633B4ADA623B4A1A63F0
:1039D0003B4ADA643B4A9A643B4A9A653B4A5A65D9
:1039E0003B4A5A663B4A1A663B4A1975DA654621D4
:1039F00040F28A22C3E90321384B394A1A60002475
:103A0000002000214FF48072C3E904011A81DC71A7
:103A1000DC6022461C83C3E90801172120460FF011
:103A20006DF922461A2120460FF068F941F6191265
:103A3000192120460FF062F92246062120460FF098
:103A40005DF94FF4FA625F2120460FF057F94FF409
:103A50007A62602120460FF051F928460CF0D4FB21
:103A6000204B1C70204B1C60204B602120461C60AA
:103A70000FF022F95F21286020460FF01DF96861E0
:103A800070BD00BFD89D02007C31FF1F885EFF1F04
:103A900035350100D864FF1F2B350100F5360100D4
:103AA0003D37010039370100353701003F3501004E
:103AB0001D3801003F370100B536010069360100AD
:103AC0008D34010093340100553501007D3401002F
:103AD000A134010081340100E13401000065FF1FC1
:103AE0007017E8032865FF1F3065FF1F2C65FF1F57
:103AF00001280BD8064B1A682023834043F00203A9
:103B000002EB830300205B680B607047082070475E
:103B10009431FF1F014B00229A607047885EFF1F9F
:103B200070B5094E3446054654F8043B014622461A
:103B300000200FF033FC3368224629460120BDE8FF
:103B400070400FF02BBC00BF9431FF1F014B186871
:103B50000FF085BC9431FF1F012838B5144613D0EF
:103B600045B21DB102281CD0042038BD114B124AA9
:103B7000DB6824681B68D2F8A8021CB15B6998470F
:103B80000020F2E79B69FAE70A4B0B4ADB68D2F8A0
:103B9000A0021B685B6A9847003018BF01202060B4
:103BA000EEE7044B044ADB68D2F8A4021B685B6AA8
:103BB000F1E700BFD89D02009431FF1F022804BF27
:103BC0000C4B93F8F00038B90B4BDB681B685B6952
:103BD0000A4AD2F89C021847012809D1054B93F8EC
:103BE000F030012B04D1044BDB681B689B69EFE7C5
:103BF000704700BF885EFF1FD89D02009431FF1FF1
:103C000070B50020FFF7DAFF134B144CDD68D4F8D1
:103C10009C022B689B6898472B68D4F8A0029B688D
:103C200098472B68D4F8A4029B6898472B68D4F86F
:103C3000B4029B6898472B68D4F8AC029B689847FD
:103C40002B68D4F8B0029B6898472B68D4F8A80278
:103C50009B68BDE870401847D89D02009431FF1F53
:103C60002DE9F8431A4C9DF820609DF824509846A1
:103C7000D4F8B8320F469B68002147F08000914687
:103C80009847D4F8B83200219B6848469847D4F842
:103C9000B83200219B6840469847D4F8B8320021DA
:103CA0009B6830469847D4F8B83228469B68012173
:103CB0009847236848EA092807F07F0746EA08265C
:103CC00003EB870745EA06257D60BDE8F88300BF62
:103CD0009431FF1F07B5D3B20193C2F307230093BA
:103CE000C2F30743120EFFF7BBFF03B05DF804FBFE
:103CF0000020FFF7EFBF01282DE9F34105460F46ED
:103D000028D8DFF85880202618F80030864074B292
:103D100063B1114B03EB800344F00701D3F8BC22DD
:103D2000C9B2FFF7D7FF002308F8053044F00D01B2
:103D30003A460024C9B22846FFF7CCFF2846CDE911
:103D4000004423462246F1B2FFF78AFF204602B024
:103D5000BDE8F0810820FAE79431FF1F7400FF1FCF
:103D6000012873B505460E461CD82024844044F033
:103D7000070186EAE672A2EBE672C9B2FFF7AAFF74
:103D8000094A0123002E5355E1B2B8BF0223002493
:103D9000CDE90043284623462246FFF761FF20462F
:103DA00002B070BD0820FBE77400FF1F0021D7E7B9
:103DB0004942D5E7D4E738B5274D01F07F042B19E8
:103DC00093F81832DB0704D42B6803EB8404606893
:103DD00038BDD5F8B83200219B6820469847D5F801
:103DE000B83200219B6808469847D5F8B8320021C0
:103DF0009B6808469847D5F8B83200219B6808466A
:103E00009847D5F8B83201219B6800209847D5F82B
:103E1000B83200219B6820469847D5F8B832002177
:103E20009B6808469847D5F8B832002104029B6881
:103E300008469847D5F8B832002104439B680846E5
:103E40009847D5F8B832240204439B68012100202A
:103E5000984724022043BBE79431FF1F10B5002090
:103E60001446FFF7A8FF206010BD38B50D4620218D
:103E7000814041F00101C9B20446FFF79CFF296867
:103E8000014429602046BDE8384034E701292DE986
:103E9000F84304460D461E4600F22F861C2A00F009
:103EA000B3825FD80C2A00F0B4812DD8052A00F027
:103EB000358115D8022A00F0E38009D8002A00F0E5
:103EC000BD80012A00F0CB8004242046BDE8F883A1
:103ED000032A00F0EC80042A00F0FC800424F4E7BC
:103EE000082A00F0658107D8062A00F02881072AF1
:103EF00000F042810424E8E70A2A00F068810B2AD6
:103F000000F077810424E0E7122A00F0028213D83F
:103F10000F2A00F0CB8107D80D2A00F098810E2AD5
:103F200000F0B3810424D0E7102A00F0D081112AD8
:103F300000F0DE810424C8E7152A00F0218207D8AA
:103F4000132A00F0F781142A00F005820424BCE74C
:103F5000172A00F03782C0F02482182A00F043822A
:103F60000424B2E7AC2A00F03A8438D8A52A00F03D
:103F70002C8313D8A22A00F0D48207D81D2A00F07F
:103F80005F828C2A00F06B8204249EE7A32A00F053
:103F9000E482A42A00F0FD82042496E7A82A00F017
:103FA000B58307D8A62A00F05683A72A00F091838C
:103FB00004248AE7AA2A4FEA011700F0E38340F2BB
:103FC000C28347F06D07FFB239462846002C40F007
:103FD000F683FFF7F0FEC0F34110306075E7B62AB4
:103FE00000F0BE8413D8B32A00F0598407D8AD2A54
:103FF00000F01284AE2A00F02D84042465E7B42A70
:1040000000F06B84B52A00F0778404245DE7CE2AA3
:1040100000F0F58407D8B82A00F0B584B92A00F07A
:10402000D084042451E7D22A00F00B85D32A00F073
:104030001B85D12A00F0F284042446E72021A94000
:1040400041F00D01C9B220B92846FFF7B4FE306037
:104050003BE71A682846FFF73DFE002435E720219C
:10406000A94041F00101C9B220B92846FFF7A3FEDB
:1040700030602AE71A682846FFF72CFE002424E760
:104080002021A94041F00701C9B220B92846FFF715
:1040900092FE306019E7B54B01225A553268002A6A
:1040A000B8BF52422846FFF715FE00240DE700284E
:1040B00040F026852021A94041F00201C9B22846DE
:1040C000FFF779FE10F4000318BF4FF07F43184349
:1040D0003060FAE6A64B8A00134418B9D3F8BC3214
:1040E0003360F2E632682027002A07FA01F7B8BFEA
:1040F0005242F9B22846C3F8BC22FFF75CFE0446E0
:1041000008B10024E1E6326847F00701002AB8BF91
:104110005242C9B22846FFF7DDFDD6E62021A9406C
:1041200041F00601C9B220B92846FFF744FE3060CD
:10413000CBE61A682846FFF7CDFD0024C5E6202708
:104140008F4047F01007FFB2394628462CB9FFF7D9
:1041500032FEC0F304203060B7E6FFF72CFE336870
:104160001B0203F4F85320F4F8521A433946284648
:10417000FFF7B0FD0024A8E620278F4047F0100786
:10418000FFB2394628462CB9FFF715FE00F01F0094
:1041900030609AE6FFF70FFE336820F01F0203F04D
:1041A0001F031A4339462846FFF794FD00248CE686
:1041B000002840F0A8842021A94041F01501C9B28F
:1041C0002846FFF7F8FDC0F3402030607DE6002868
:1041D00040F09C842021A94041F01501C9B2284635
:1041E000FFF7E9FD10F0020F0CBF0123002333603D
:1041F0006BE6002840F08D842021A94041F0150194
:10420000C9B22846FFF7D7FDC04300F00100306077
:104210005BE620278F4047F01407FFB23946284657
:104220002CB9FFF7C8FDC0F3400030604DE6FFF742
:10423000C2FD3368002B20F002020CBF02230023D2
:104240001A4339462846FFF745FD00243DE620275E
:104250008F4047F01407FFB2394628462CB9FFF7C4
:10426000AAFD00F0010030602FE6FFF7A4FD3268E0
:1042700020F00100002A14BF024640F00102394636
:104280002846FFF727FD00241FE62021A94041F022
:104290001401C9B220B92846FFF78DFD306014E63D
:1042A0001A682846FFF716FD00240EE62021A940D3
:1042B00041F00401C9B220B92846FFF77CFD306007
:1042C00003E61A682846FFF705FD0024FDE52021D6
:1042D000A94041F00501C9B220B92846FFF76BFD9E
:1042E0003060F2E51A682846FFF7F4FC0024ECE59C
:1042F0002021A94041F00801C9B220B92846FFF7A2
:104300005AFD3060E1E51A682846FFF7E3FC002417
:10431000DBE52021A94041F00A01C9B220B92846B5
:10432000FFF749FD3060D0E51A682846FFF7D2FC58
:104330000024CAE52021A94041F00301C9B220B9F7
:104340002846FFF738FD3060BFE51A682846FFF7BA
:10435000C1FC0024B9E52021A94041F00B01C9B2FC
:1043600040B92846FFF727FD3060AEE57400FF1F17
:104370009431FF1F1A682846FFF7ACFC0024A4E51F
:104380002021A94041F00C01C9B220B92846FFF70D
:1043900012FD306099E51A682846FFF79BFC00245F
:1043A00093E52021A94041F01101C9B220B9284666
:1043B000FFF701FD306088E51A682846FFF78AFCA0
:1043C000002482E52021A94041F01201C9B220B9A0
:1043D0002846FFF7F0FC306077E51A682846FFF7BB
:1043E00079FC002471E52021A94041F01301C9B2F4
:1043F00020B92846FFF7DFFC306066E51A682846DA
:10440000FFF768FC002460E50F0147F06C07FFB27E
:10441000394628462CB9FFF7CEFCC0F38040306007
:1044200053E5FFF7C8FC33689B0403F4802320F4B2
:1044300080221A4339462846FFF74CFC002444E505
:10444000002840F06983C64B1A68202303FA01F55F
:1044500045F0020502EB85056B68336035E570B900
:10446000090141F06C0101F0FC012846FFF7A3FCB3
:104470004FF48073C0F303600341336025E51B688C
:10448000102B48D00FDC022B41D006DC012B18D0BA
:104490004FF0FF333360002417E5042B39D0082B8D
:1044A000F6D105230EE0402B37D003DC202BEFD1D3
:1044B000032307E0802B32D0B3F5807FE8D10023BF
:1044C00000E008232C0144F06C04E4B22146336080
:1044D0002846FFF770FC33681B0603F0706320F07A
:1044E00070621A4321462846FFF7F4FB214628460E
:1044F000FFF761FC33681B0603F0706320F0706205
:1045000021461A432846FFF7E5FB0024DDE4072394
:10451000D8E70623D6E70423D4E70223D2E7012312
:10452000D0E70F0147F06C07FFB2394628462CB997
:10453000FFF741FCC0F3C1303060C6E4FFF73BFC3D
:104540003368DB0303F4C03320F4C0321A43394626
:104550002846FFF7BFFB0024B7E40F0147F06C07C4
:10456000FFB2394628462CB9FFF725FCC0F380304E
:104570003060AAE4FFF71FFC33689B0303F4804319
:1045800020F480421A4339462846FFF7A3FB002453
:104590009BE40F0147F06C07FFB2394628462CB95F
:1045A000FFF709FCC0F3003030608EE4FFF703FC36
:1045B00033681B0303F4805320F480521A433946B6
:1045C0002846FFF787FB00247FE40F0147F06C07C4
:1045D000FFB239462846FFF7EEFB3946814600F424
:1045E00080482846B4B9B8F1000F05D0FFF7E3FBC7
:1045F000C0F3C310306068E4FFF7DDFB19F4006F0F
:10460000C0F3021001D130607BE540F0080030605B
:1046100044465AE4B8F1000F0ED0FFF7CCFB3368E4
:10462000DB0103F4F06320F4F0621A4339462846B4
:10463000FFF750FB002448E4FFF7BDFB33681B0184
:1046400003F0700320F070021A4339462846FFF742
:1046500041FB444639E40F0147F06C07FFB239468D
:104660002846FFF7A8FB394600F48048284674B96D
:10467000B8F1000F05D0FFF79EFBC0F302103060C9
:1046800023E4FFF798FBC0F3C31030601DE4B8F1DA
:10469000000F0ED0FFF78FFB33681B0103F0700390
:1046A00020F070021A4339462846FFF713FB002416
:1046B0000BE4FFF780FB3368DB0103F4F06320F4C5
:1046C000F0621A4339462846FFF704FB4446FFF7D9
:1046D000FCBB0F0147F06C07FFB23946284634B9DE
:1046E000FFF769FB00F00F003060FFF7EEBBFFF74C
:1046F00062FB336820F00F0203F00F031A433946C0
:104700002846FFF7E7FA0024FFF7DFBB0F0147F069
:104710006D07FFB23946284634B9FFF74CFBC0F3AA
:10472000C0303060FFF7D1BBFFF745FB3368DB03D8
:104730009BB220F400421A4339462846FFF7CAFAD2
:104740000024FFF7C2BB47F06D07FFB23946284689
:1047500044B9FFF730FBC0F341303060FFF7B5BB21
:104760009431FF1FFFF727FB33685B0303F4C0435B
:1047700020F4C0421A4339462846FFF7ABFA00241A
:10478000FFF7A3BB47F06D07FFB23946284634B99F
:10479000FFF711FBC0F303203060FFF796BBFFF774
:1047A0000AFB33681B0203F4706320F470621A433F
:1047B00039462846FFF78EFA0024FFF786BBFFF73D
:1047C000FAFA33685B0103F0600320F060021A43D9
:1047D00039462846FFF77EFA0024FFF776BB0F0123
:1047E00047F06D07FFB23946284634B9FFF7E3FAC0
:1047F00000F00F003060FFF768BBFFF7DCFA3368AA
:1048000020F00F0203F00F031A4339462846FFF742
:1048100061FA0024FFF759BB0F0147F06D07FFB2A3
:104820003946284634B9FFF7C6FAC0F30060306055
:10483000FFF74BBBFFF7BFFA33681B0603F080732B
:1048400020F080721A4339462846FFF743FA0024C5
:10485000FFF73BBB0F0147F06D07FFB23946284613
:104860006CB9FFF7A8FA001400F07F0310F04000C5
:1048700018BF6FF07F0018433060FFF726BBFFF7CB
:104880009AFA33681B0403F4FE0320F4FE021A4371
:1048900039462846FFF71EFA0024FFF716BB0F0122
:1048A00047F06C07FFB23946284634B9FFF783FA60
:1048B000C0F340403060FFF708BBFFF77CFA336875
:1048C0005B0403F4003320F400321A4339462846CF
:1048D000FFF700FA0024FFF7F8BA002840F01F8124
:1048E000090141F06F01C9B22846FFF764FAC0F32D
:1048F00004403060FFF7E9BA20278F407FB247F0CD
:1049000014085FFA88F841462846FFF754FA6CB954
:10491000410508D547F01101C9B22846FFF74BFA07
:104920003060FFF7D2BA3460FFF7CFBA47F0110119
:104930003268C9B22846FFF7CDF941462846FFF74D
:104940003AFA3368002B20F4806218BF4FF480637A
:104950001A4341462846FFF7BDF90024FFF7B5BAD0
:104960002021A94041F01101C9B228B92846FFF71A
:1049700022FA3060FFF7A9BA1A682846FFF7AAF9A9
:104980000024FFF7A2BA0F0147F06C07FFB23946C7
:10499000284634B9FFF70FFAC0F340303060FFF714
:1049A00094BAFFF708FA33685B0303F4005320F46A
:1049B00000521A4339462846FFF78CF90024FFF7C6
:1049C00084BA0F0147F06C07FFB23946284634B964
:1049D000FFF7F1F9C0F303503060FFF776BAFFF745
:1049E000EAF933681B0503F4700320F470021A43DC
:1049F00039462846FFF76EF90024FFF766BA00280B
:104A000040F09080090141F06F01C9B22846FFF7DC
:104A1000D2F9C0F309003060FFF757BA2021A9404E
:104A200041F01901C9B228B92846FFF7C4F930602E
:104A3000FFF74BBA1A682846FFF74CF90024FFF736
:104A400044BA2021A94041F01A01C9B228B9284628
:104A5000FFF7B1F93060FFF738BA1A682846FFF758
:104A600039F90024FFF731BAC8B9012D01460AD03F
:104A7000FFF7A1F900F01800A0F1100250425041D8
:104A80003060FFF722BA2846FFF795F900F0600082
:104A9000A0F12003584258413060FFF716BA012DAB
:104AA0004FF0000114D00846FFF785F9336853B181
:104AB00020F0080242F0100200210846FFF70AF930
:104AC0000024FFF702BA20F0100242F00802F3E7D8
:104AD0002846FFF770F9336853B120F0400242F0E6
:104AE000200200210120FFF7F5F80024FFF7EDB9BF
:104AF00020F0200242F04002F3E70824FFF7E5B976
:104B00000424FFF7E2B90424FFF7DFB90424FFF718
:104B1000DCB90424FFF7D9B90424FFF7D6B904247B
:104B2000FFF7D3B90424FFF7D0B907B5019201AB61
:104B300002460120FFF7AAF903B05DF804FB134613
:104B400002460020FFF7A2B908B522210020FFF796
:104B500032F950B942210120FFF72DF928B9044B51
:104B60001868BDE808400EF073BC002008BD00BF07
:104B70009431FF1F70B5424C424E201D0EF0CEFB0B
:104B8000F5686B6803F58472C4F8A02203F594728B
:104B9000C4F8A42203F57272C4F8A82203F57A724D
:104BA00003F16800C4F8AC2203F5816203F5856364
:104BB000C4F8B4322B68C4F8B022DB68C4F89C0295
:104BC00098472B68D4F8A802DB6898472B68D4F87C
:104BD000A8029B6998472B68D4F8A0021B699847E4
:104BE0002B68D4F8A4021B6998472B68D4F8B40248
:104BF0001B6998472B68D4F8AC021B6998472B684F
:104C0000D4F8B0021B6998476B683269C4F8B822BF
:104C100003F5327353601C4B1C499A692260C2F839
:104C2000041201201A491080C2F80812194A5A6267
:104C3000194A1A62194ADA61194A9A62194ADA63F8
:104C4000194A9A63194ADA62194A1A63194ADA64E4
:104C5000194A9A64194A9A65194A5A65194A1A658D
:104C6000194A5A66194A1A6602221A753221B62260
:104C7000C3E90321BDE87040154ADA65FEF79EBF1F
:104C80009431FF1FD89D0200885EFF1F494B010031
:104C90004D3B0100613D0100B53D0100B13D01000A
:104CA000AD3D01003F4B01002B4B0100F73C0100E3
:104CB0006B3E0100F13C01005D3E0100213B010023
:104CC000593B0100F13A0100BD3B0100153B0100D9
:104CD000013C010001289FBF044B03EB800300202F
:104CE0005B6894BF0B600820704700BF6434FF1FEF
:104CF000014B00229A607047885EFF1F0146014801
:104D00000EF044BC6434FF1F10B5034814460EF087
:104D1000F0FB206010BD00BF6434FF1F01480EF09F
:104D2000DABB00BF6434FF1F0128F8B50D4625D853
:104D3000134B1F18202497F89822844066B27AB14A
:104D4000D3F89C2244F0070102EB810246F00701F0
:104D500018465268C9B20EF0BEFB002387F898329D
:104D600046F00D012A46C9B205480EF0B4FB0448CE
:104D70000022E1B20EF0AFFB0020F8BD0820FCE7F6
:104D80006434FF1F38B50D462021814041F00101F8
:104D90000446C9B204480EF0ACFB296801442960FE
:104DA0002046BDE83840BFE76434FF1F0129F8B54D
:104DB00004460D461E4600F2F8851C2A00F0C78204
:104DC0005ED80C2A00F0A8812CD8052A00F0278193
:104DD00014D8022A00F0D58008D8002A00F0AF804D
:104DE000012A00F0BD8004242046F8BD032A00F00B
:104DF000E080042A00F0F0800424F5E7082A00F09F
:104E00005A8107D8062A00F01B81072A00F0368154
:104E10000424E9E70A2A00F05D810B2A00F06C8186
:104E20000424E1E7122A00F01B8213D80F2A00F0B5
:104E3000E18107D80D2A00F09D810E2A00F0C9817A
:104E40000424D1E7102A00F0E981112A00F0F7814B
:104E50000424C9E7152A00F0368207D8132A00F087
:104E60001082142A00F01E820424BDE7172A00F0E5
:104E70004C82C0F03982182A00F058820424B3E72B
:104E8000AB2A00F039842BD8A52A00F02F8313D841
:104E9000A22A00F0D48207D81D2A00F074828C2A3E
:104EA00000F07A8204249FE7A32A00F0E482A42A77
:104EB00000F00083042497E7A82A00F0C48307D8F1
:104EC000A62A00F06383A72A00F0A68304248BE7B8
:104ED000A92A00F0D583AA2A00F0F083042483E7EE
:104EE000B52A00F0B78413D8AE2A00F0618407D841
:104EF000AC2A00F01F84AD2A00F03984042473E743
:104F0000B32A00F07A84B42A00F0958404246BE775
:104F1000CE2A00F0F88407D8B62A00F0C384B82A55
:104F200000F0D38404245FE7D12AC0F04185D22A5F
:104F300040F24185D32A00F0F484042454E7202170
:104F4000A94041F00D01C9B220B9B0480EF0D1FA24
:104F5000306049E71A68AD480EF0BDFA002443E717
:104F60002021A94041F00101C9B220B9A7480EF0A3
:104F7000C0FA306038E71A68A4480EF0ACFA002492
:104F800032E72021A94041F00701C9B29F481CB96E
:104F90000EF0AFFA306027E732680544002A4FF080
:104FA0000103B8BF524285F8983200240EF093FAFC
:104FB0001AE7002840F002852021A94041F00201B3
:104FC000C9B292480EF095FA10F4000318BF4FF0E2
:104FD0007F431843306007E78C4F2021A940D7F862
:104FE0009C3241F00705AA00134410B95B68336096
:104FF000FAE63268002AB8BF52425A60C9B238464F
:105000000EF077FA044608B10024EDE63268002A73
:10501000B8BF5242E9B238460EF05DFAE4E620210C
:10502000A94041F00601C9B220B978480EF061FAF2
:105030003060D9E61A6875480EF04DFA0024D3E6C0
:10504000202101FA05F545F01005EDB229466F481B
:105050002CB90EF04EFAC0F304203060C4E60EF016
:1050600048FA33681B0203F4F85320F4F8521A4349
:10507000294666480EF02FFA0024B5E6202101FAF1
:1050800005F545F01005EDB2294660482CB90EF043
:1050900030FA00F01F003060A6E60EF02AFA3368FE
:1050A00020F01F0203F01F031A43294657480EF051
:1050B00012FA002498E6002840F083842021A940B9
:1050C00041F01501C9B251480EF013FAC0F3402067
:1050D000306089E6002840F077842021A94041F023
:1050E0001501C9B249480EF004FA10F0020F0CBFC6
:1050F00001230023336077E6002840F068842021F4
:10510000A94041F01501C9B240480EF0F2F9C04380
:1051100000F00100306067E6202101FA05F545F056
:105120001405EDB2294639482CB90EF0E2F9C0F366
:105130004000306058E60EF0DCF93368002B18BFF1
:10514000022320F002021A43294630480EF0C3F928
:1051500029462E480EF0CDF93368022B20F00802C4
:105160000CBF082300231A43294628480EF0B3F940
:10517000002439E6202101FA05F545F01405EDB2C9
:10518000294622482CB90EF0B4F900F00100306035
:105190002AE60EF0AEF9326820F00100002A0CBFBA
:1051A000024640F00102294618480EF094F92946BB
:1051B00016480EF09EF93368022B20F004020CBF53
:1051C000042300231A43294610480EF084F90024D2
:1051D0000AE62021A94041F01401C9B220B90B48C8
:1051E0000EF087F93060FFE51A6808480EF073F991
:1051F0000024F9E52021A94041F00401C9B238B9E1
:1052000002480EF076F93060EEE500BF6434FF1F0F
:105210001A68A7480EF05FF90024E5E52021A940AF
:1052200041F00501C9B220B9A1480EF062F9306021
:10523000DAE51A689E480EF04EF90024D4E52021E4
:10524000A94041F00801C9B220B999480EF051F9BE
:105250003060C9E51A6896480EF03DF90024C3E5B0
:105260002021A94041F00A01C9B220B990480EF0AE
:1052700040F93060B8E51A688D480EF02CF900242A
:10528000B2E52021A94041F00301C9B220B9884804
:105290000EF02FF93060A7E51A6885480EF01BF96B
:1052A0000024A1E52021A94041F00B01C9B220B999
:1052B0007F480EF01EF9306096E51A687C480EF0C3
:1052C0000AF9002490E52021A94041F00C01C9B25F
:1052D00020B977480EF00DF9306085E51A687448FA
:1052E0000EF0F9F800247FE52021A94041F01101DA
:1052F000C9B220B96E480EF0FCF8306074E51A6847
:105300006B480EF0E8F800246EE52021A94041F03A
:105310001201C9B220B966480EF0EBF8306063E5BF
:105320001A6863480EF0D7F800245DE52021A940F3
:1053300041F01301C9B220B95D480EF0DAF83060CF
:1053400052E51A685A480EF0C6F800244CE50D01E3
:1053500045F06C05EDB2294655482CB90EF0C9F858
:10536000C0F3804030603FE50EF0C3F833689B0423
:1053700003F4802320F480221A4329464C480EF07F
:10538000AAF8002430E5002840F02483484901EBC6
:1053900085014B68336027E570B9090141F06C0164
:1053A00001F0FC0142480EF0A4F84FF48073C0F302
:1053B00003600341336017E51B68102B39D00FDC05
:1053C000022B32D006DC012B18D04FF0FF333360B4
:1053D000002409E5042B2AD0082BF6D105230EE082
:1053E000402B28D003DC202BEFD1032307E0802BB8
:1053F00023D0B3F5807FE8D1002300E008232D01FE
:1054000045F06C05EDB23360294629480EF071F87D
:1054100033681B0603F0706320F070621A4329465C
:1054200023480EF058F80024DEE40723E7E70623BC
:10543000E5E70423E3E70223E1E70123DFE70D01CA
:1054400045F06C05EDB2294619482CB90EF051F81B
:10545000C0F3C1303060C7E40EF04BF83368DB03B3
:1054600003F4C03320F4C0321A43294610480EF02A
:1054700032F80024B8E40D0145F06C05EDB2294680
:105480000B482CB90EF035F8C0F380303060ABE437
:105490000EF02FF833689B0303F4804320F480421E
:1054A0001A43294602480EF016F800249CE400BF77
:1054B0006434FF1F0D0145F06C05EDB22946BB4871
:1054C0002CB90EF016F8C0F3003030608CE40EF00A
:1054D00010F833681B0303F4805320F480521A43FE
:1054E0002946B2480DF0F7FF00247DE40D0145F098
:1054F0006C05EDB22946AD480DF0FBFF00F4804786
:10550000A4B93FB12946A9480DF0F3FFC0F3C31079
:10551000306069E40311020503F0700301D43360C5
:1055200072E543F0080333603C465DE429469F483A
:1055300077B10DF0DEFF3368DB0103F4F06320F494
:10554000F0621A43294699480DF0C5FF00244BE448
:105550000DF0CFFF3268120220F4006002F4006206
:105560000243294691480DF0B6FF29468F480DF0B9
:10557000C0FF33681B0103F0700320F070021A4370
:1055800029468A480DF0A7FF3C462DE40D0145F061
:105590006C05EDB2294685480DF0ABFF294607465C
:1055A00082489CB97D0405D50DF0A3FFC0F302101D
:1055B000306019E40DF09DFF3905C0F3C31001D42C
:1055C000306021E540F0080030600DE40DF091FFFF
:1055D00010F48044294675480FD00DF08AFF3368D7
:1055E0001B0103F0700320F070021A4329466F4834
:1055F0000DF071FF0024FFF7F7BB0DF07AFF336861
:10560000DB0103F4F06320F4F0621A432946674893
:105610000DF061FFFFF7E8BB0D0145F06C05EDB241
:105620002946624824B90DF064FF3460FFF7DCBB03
:105630000DF05FFF294620F00F025C480DF04BFF94
:105640000024FFF7D1BB0D0145F06D05EDB22946F1
:10565000564834B90DF04DFFC0F3C0303060FFF74D
:10566000C3BB0DF046FF3368DB039BB220F400425E
:105670001A4329464D480DF02EFF0024FFF7B4BB16
:105680000D0145F06D05EDB22946484834B90DF0DD
:1056900030FFC0F341303060FFF7A6BB0DF029FFAB
:1056A00033685B0303F4C04320F4C0421A43294625
:1056B0003E480DF010FF0024FFF796BB0D0145F0AA
:1056C0006D05EDB22946394834B90DF012FFC0F32B
:1056D00003203060FFF788BB0DF00BFF33681B021F
:1056E00003F4706320F470621A4329462F480DF0CA
:1056F000F2FE0024FFF778BB0D0145F06D05EDB219
:1057000029462A4834B90DF0F4FEC0F34110306048
:10571000FFF76ABB0DF0EDFE33685B0103F0600339
:1057200020F060021A43294620480DF0D4FE0024E0
:10573000FFF75ABB0D0145F06D05EDB229461B4838
:1057400034B90DF0D6FE00F00F003060FFF74CBB0F
:105750000DF0CFFE336820F00F0203F00F031A4361
:10576000294612480DF0B7FE0024FFF73DBB0D019E
:1057700045F06D05EDB229460C4834B90DF0B9FE7F
:10578000C0F300603060FFF72FBB0DF0B2FE33684E
:105790001B0603F0807320F080721A4329460348E9
:1057A0000DF099FE0024FFF71FBB00BF6434FF1FFC
:1057B0000D0145F06D05EDB229468B486CB90DF031
:1057C00098FE001400F07F0310F0400018BF6FF047
:1057D0007F0018433060FFF707BB0DF08AFE336887
:1057E0001B0403F4FE0320F4FE021A4329467E48FC
:1057F0000DF071FE0024FFF7F7BA0D0145F06C05BE
:10580000EDB22946784834B90DF073FEC0F340403C
:105810003060FFF7E9BA0DF06CFE33685B0403F407
:10582000003320F400321A4329466F480DF053FE2E
:105830000024FFF7D9BA002840F0CF80090141F0D9
:105840006F01C9B268480DF054FEC0F304403060E7
:10585000FFF7CABA202101FA05F56DB245F0110132
:10586000C9B228B960480DF044FE3060FFF7BCBAF9
:1058700045F014051A685C48EDB20DF02CFE29467F
:1058800059480DF036FE3368002B20F4806218BFB3
:105890004FF480631A43294653480DF01CFE002440
:1058A000FFF7A2BA2021A94041F01101C9B228B9DD
:1058B0004D480DF01EFE3060FFF796BA1A684A4850
:1058C0000DF009FE0024FFF78FBA0D0145F06C05BD
:1058D000EDB22946444834B90DF00BFEC0F3403018
:1058E0003060FFF781BA0DF004FE33685B0303F408
:1058F000005320F400521A4329463B480DF0EBFDBB
:105900000024FFF771BA00286AD1090141F06F0144
:10591000C9B235480DF0EDFDC0F309003060FFF766
:1059200063BAC8B9012D01462F480AD00DF0E1FD38
:1059300000F01800A0F11002504250413060FFF713
:1059400053BA0DF0D6FD00F06000A0F120035842DC
:1059500058413060FFF748BA012D4FF0000122484E
:1059600011D00DF0C6FD336820F0180243B142F0AB
:10597000100200211C480DF0AEFD0024FFF734BAE0
:1059800042F00802F5E70DF0B4FD336820F0600244
:1059900043B142F02002002113480DF09CFD002489
:1059A000FFF722BA42F04002F5E70824FFF71CBADD
:1059B0000424FFF719BA0024FFF716BA0424FFF7EE
:1059C00013BA0424FFF710BA0424FFF70DBA042415
:1059D000FFF70ABA0424FFF707BA0424FFF704BA52
:1059E0000424FFF701BA00BF6434FF1F07B501921A
:1059F00001AB02460120FFF7D9F903B05DF804FBC3
:105A0000134602460020FFF7D1B901480DF028BE29
:105A10006434FF1F012810B5144603D002280FD0AC
:105A2000042010BD0A4B0B4ADB68D2F8A4021B68A5
:105A30005B6A9847003018BF012020600020F0E723
:105A4000034B044ADB68D2F8A8021B685B6AF0E7E4
:105A5000D89D02006434FF1F022804BF0C4B93F84A
:105A6000F00038B90B4BDB681B685B690A4AD2F857
:105A7000A0021847012809D1054B93F8F030012BFB
:105A800004D1044BDB681B689B69EFE7704700BFDC
:105A9000885EFF1FD89D02006434FF1F70B5002090
:105AA000FFF7DAFF094B0A4CDD68D4F8A0022B6837
:105AB0009B6898472B68D4F8A4029B6898472B688A
:105AC000D4F8A8029B68BDE870401847D89D020032
:105AD0006434FF1F0128F8B504460F461AD8202564
:105AE00085400D4E45F0070187EAE772A2EBE772A9
:105AF000C9B230460DF0EFFC34440123002F30468C
:105B0000ACBF1A460222E9B284F898320DF0E3FCE9
:105B10000020F8BD0820FCE76434FF1F0021D9E70E
:105B20004942D7E7D6E708B5222108480DF0E1FC45
:105B300048B9422105480DF0DCFC20B90348BDE816
:105B400008400DF085BD002008BD00BF6434FF1F74
:105B5000034BD3F8AC320846DB681146184700BF48
:105B60006434FF1FF8B5304C304D314FA269314BD2
:105B7000002128460DF0E5FCFE68736803F5847289
:105B800003F1680003F59473C5F8A8323368C5F8CB
:105B9000A422DB68C5F8A00298473368D5F8A402B0
:105BA0001B6998473368D5F8A8021B699847736842
:105BB0003A69C5F8AC2203F532735360A3691E4AF3
:105BC000C3F804221D4AC3F8082201221A80C5F82E
:105BD0009C321B4B63621B4B23621B4BE3611B4BD1
:105BE000A3621B4BE3631B4BA3631B4BE3621B4B87
:105BF00023631B4BE3641B4BA3641B4BA3651B4B31
:105C000063651B4B23651B4B63661B4B236632226C
:105C10004FF48C73C4E903320220184B2075E365FE
:105C2000BDE8F84018E700BF885EFF1F6434FF1F1F
:105C3000D89D0200B4930200275B01000B5A0100BB
:105C4000D55A0100255B0100215B01001D5B0100AD
:105C5000015A0100ED590100294D0100854D010057
:105C60001D4D0100094D0100FD4C0100155A0100B8
:105C7000D54C0100595A0100F14C01009D5A010018
:105C800001289FBF044B03EB80030020DB6994BF16
:105C90000B600820704700BF2037FF1F014B002218
:105CA0009A607047885EFF1F014601480DF06DBE87
:105CB0002037FF1F0A46014601480DF007BD00BF0F
:105CC0002037FF1F10B500201446FFF7F3FF2060B8
:105CD00010BD38B514460A46014603481D460DF06E
:105CE000F5FC2040E84038BD2037FF1F13460A4628
:105CF000014601480DF0E6BC2037FF1F0020F5E704
:105D000001282DE9F041044688461FD8104F07EBC3
:105D100080072025D7F8A42285406EB23AB146F01C
:105D20000701C9B2FFF7E2FF0023C7F8A43246F02B
:105D30000D014246C9B22046FFF7D8FF2046002297
:105D4000E9B2FFF7D3FF0020BDE8F0810820FBE7B0
:105D50002037FF1F38B50D462021814041F0010159
:105D6000C9B20446FFF7A6FF29680144296020460E
:105D7000BDE83840C4E701282DE9F04104468846D3
:105D800023D8134F07EB800720258540D7F8A4328E
:105D900045F00706F6B223B93146FFF78BFFC7F887
:105DA000A40288EAE872A2EBE87231462046FFF7C7
:105DB0009DFFB8F1000F2046ACBF01220222E9B2DC
:105DC000FFF794FF0020BDE8F0810820FBE700BF4B
:105DD0002037FF1F0021CEE74942CCE7CBE72DE972
:105DE000F0470C4D089C06460F4690460A46014671
:105DF000284699460DF06AFC04FA09F2424002EA8C
:105E0000080282EA000331463A462846BDE8F047D8
:105E10000DF058BC2037FF1F01292DE9F34104463E
:105E20000D461E4600F2B0851C2A00F0958260D80F
:105E30000C2A00F0A8812ED8052A00F0318116D84E
:105E4000022A00F0E3800AD8002A00F0BD80012A6F
:105E500000F0CB800424204602B0BDE8F081032A84
:105E600000F0E880042A00F0F8800424F3E7082A10
:105E700000F0558107D8062A00F02381072A00F098
:105E800038810424E7E70A2A00F059810B2A00F040
:105E900068810424DFE7122A00F0E58113D80F2A75
:105EA00000F0AE8107D80D2A00F083810E2A00F0A1
:105EB00096810424CFE7102A00F0B381112A00F064
:105EC000C1810424C7E7152A00F0008207D8132AED
:105ED00000F0DA81142A00F0E8810424BBE7172AD5
:105EE00000F01882C0F00382182A00F024820424F3
:105EF000B1E7AC2A00F0E28337D8A52A00F0E182AE
:105F000013D8A22A00F0988207D81D2A00F03B82FD
:105F10008C2A00F0418204249DE7A32A00F0A3828A
:105F2000A42A00F0B782042495E7A82A00F072831F
:105F300007D8A62A00F01883A72A00F05683042465
:105F400089E7AA2A4FEA011100F0968340F279838B
:105F500041F06D01C9B2002840F0A68305236022FC
:105F60002846FFF7B6FE306075E7B62A00F04C848D
:105F700013D8B32A00F0F18307D8AD2A00F0B58317
:105F8000AE2A00F0CB83042465E7B42A00F0FE8338
:105F9000B52A00F00B8404245DE7CE2A00F0798452
:105FA00007D8B82A00F04384B92A00F059840424A1
:105FB00051E7D22A00F09084D32A00F0A084D12A9D
:105FC00000F07784042446E72021A94041F00D0128
:105FD000C9B220B92846FFF76DFE30603BE71A686A
:105FE0002846FFF783FE002435E72021A94041F031
:105FF0000101C9B220B92846FFF75CFE30602AE7EC
:106000001A682846FFF772FE002424E72021A940E1
:1060100041F00701C9B220B92846FFF74BFE3060B6
:1060200019E71A68002AB8BF52422846FFF75EFEF9
:10603000002410E7002840F0AA842021A94041F064
:106040000201C9B22846FFF735FE10F4000318BF5D
:106050004FF07F4318433060FDE6AD4B2021A9404F
:10606000D3F8AC3241F00707BA00134410B95B68AB
:106070003360F0E63268002AB8BF52425A60C9B2B3
:106080002846FFF717FE044608B10024E3E632680D
:10609000002AB8BF5242F9B22846FFF727FEDAE6D7
:1060A0002021A94041F00601C9B220B92846FFF7D6
:1060B00001FE3060CFE61A682846FFF717FE00247D
:1060C000C9E62021A94041F01001C9B238B908231E
:1060D0004FF4F8522846FFF7FCFD3060BBE61B6822
:1060E00000934FF4F85208232846FFF778FE002467
:1060F000B1E62021A94041F01001C9B230B90346F0
:106100001F222846FFF7E5FD3060A4E61B680093D8
:106110001F2200232846FFF762FE00249BE600288A
:1061200040F038842021A94041F0150109234FF4A3
:106130000072C9B22846FFF7CCFD30608BE600281C
:1061400040F02B842021A94041F0150101230222B7
:10615000C9B22846FFF7BDFDB0FA80F040093060B3
:1061600079E6002840F01C842021A94041F0150167
:1061700003460122C9B22846FFF7ABFDB0FA80F012
:106180004009306067E62021A94041F01401C9B2FE
:1061900030B9012302222846FFF79BFD30605AE602
:1061A0001B680093022201232846FFF718FE0024F3
:1061B00051E62021A94041F01401C9B230B903468B
:1061C00001222846FFF785FD306044E61B680093F6
:1061D000012200232846FFF702FE00243BE620218F
:1061E000A94041F01401C9B220B92846FFF762FD69
:1061F000306030E61A682846FFF778FD00242AE66A
:106200002021A94041F00401C9B220B92846FFF776
:1062100051FD30601FE61A682846FFF767FD00242D
:1062200019E62021A94041F00501C9B220B928464C
:10623000FFF740FD30600EE61A682846FFF756FD6E
:10624000002408E62021A94041F00801C9B220B984
:106250002846FFF72FFD3060FDE51A682846FFF756
:1062600045FD0024F7E52021A94041F00A01C9B20B
:1062700020B92846FFF71EFD3060ECE51A68284675
:10628000FFF734FD0024E6E52021A94041F0030199
:10629000C9B220B92846FFF70DFD3060DBE51A686A
:1062A0002846FFF723FD0024D5E52021A94041F031
:1062B0000B01C9B220B92846FFF7FCFC3060CAE5E3
:1062C0001A682846FFF712FD0024C4E52021A940E2
:1062D00041F00C01C9B220B92846FFF7EBFC306051
:1062E000B9E51A682846FFF701FD0024B3E520212F
:1062F000A94041F01101C9B220B92846FFF7DAFCE4
:106300003060A8E51A682846FFF7F0FC0024A2E5F3
:106310002037FF1F2021A94041F01201C9B220B946
:106320002846FFF7C7FC306095E51A682846FFF756
:10633000DDFC00248FE52021A94041F01301C9B202
:1063400020B92846FFF7B6FC306084E51A68284675
:10635000FFF7CCFC00247EE5090141F06C01C9B2D5
:1063600038B912234FF480222846FFF7B2FC306080
:1063700071E51B6800934FF4802212232846FFF733
:106380002EFD002467E5002840F00D83B94B03EB98
:106390008105EB6933605EE580B9090141F06C016C
:1063A00018234FF0706201F0FC012846FFF791FCC2
:1063B0004FF4807343FA00F030604CE51B68102BFB
:1063C00034D00DDC022B2DD004DC012B16D04FF085
:1063D000FF3314E0042B27D0082BF8D105230EE05F
:1063E000402B25D003DC202BF1D1032307E0802BA9
:1063F00020D0B3F5807FEAD1002300E0082333608A
:1064000033685C1C3FF441AE290141F06C010093FC
:106410004FF07062182301F0FC012846FFF7DFFC03
:10642000002418E50723EAE70623E8E70423E6E764
:106430000223E4E70123E2E7090141F06C01C9B25C
:1064400038B90F234FF4C0322846FFF742FC3060C2
:1064500001E51B6800934FF4C0320F232846FFF775
:10646000BEFC0024F7E4090141F06C01C9B238B95F
:106470000E234FF480422846FFF72BFC3060EAE4FD
:106480001B6800934FF480420E232846FFF7A7FCB9
:106490000024E0E4090141F06C01C9B238B90C23D1
:1064A0004FF480522846FFF714FC3060D3E41B6899
:1064B00000934FF480520C232846FFF790FC0024F1
:1064C000C9E40F0147F06C07FFB240BB0E234FF445
:1064D000804239462846FFF7FCFB804640B107233F
:1064E0004FF4F06239462846FFF7F3FB3060B2E420
:1064F0000423702239462846FFF7EBFB0B2330605C
:106500004FF4006239462846FFF7E3FB00283FF4CA
:10651000BCAD336843F00803336044469BE439461E
:106520002846FFF7C7FB10F48044336809D0009376
:106530004FF4F062072339462846FFF750FC002449
:1065400089E4C3F3C0030093394628460B234FF474
:106550000062FFF744FC336800937022042339463D
:106560002846FFF73CFC76E40F0147F06C07FFB2CA
:106570003946284614BBFFF79DFB400407D504238A
:10658000702239462846FFF7A4FB306063E40723F6
:106590004FF4F06239462846FFF79BFB0B2330602F
:1065A0004FF4006239462846FFF793FB00283FF47A
:1065B0006CAD336843F0080333604CE4FFF77AFBBB
:1065C0003368009310F4804407D0042370223946C6
:1065D0002846FFF704FC00243DE407234FF4F06253
:1065E00039462846FFF7FBFB35E4090141F06C0111
:1065F000C9B230B903460F222846FFF76AFB306064
:1066000029E41B6800930F2200232846FFF7E7FBCD
:10661000002420E4090141F06D01C9B238B90F230B
:106620004FF400422846FFF754FB306013E41B6828
:1066300000934FF400420F232846FFF7D0FB0024BD
:1066400009E441F06D01C9B240B90D234FF4C042D5
:106650002846FFF73EFB3060FFF7FDBB1B68009349
:106660004FF4C0420D232846FFF7B9FB0024FFF783
:10667000F2BB00BF2037FF1F41F06D01C9B240B926
:1066800008234FF470622846FFF723FB3060FFF7C2
:10669000E2BB1B6800934FF4706208232846FFF7A3
:1066A0009EFB0024FFF7D7BB1B68009360220523E5
:1066B0002846FFF794FB0024FFF7CDBB090141F00A
:1066C0006D01C9B238B903460F222846FFF701FB16
:1066D0003060FFF7C0BB1B6800930F2200232846E1
:1066E000FFF77DFB0024FFF7B6BB090141F06D0108
:1066F000C9B240B918234FF080722846FFF7E9FA73
:106700003060FFF7A8BB1B6800934FF0807218231E
:106710002846FFF764FB0024FFF79DBB090141F009
:106720006D01C9B270B910234FF4FE022846FFF77D
:10673000D0FA10F0400318BF6FF07F0318433060A9
:10674000FFF789BB1B6800934FF4FE021023284615
:10675000FFF745FB0024FFF77EBB090141F06C0108
:10676000C9B240B911234FF400322846FFF7B1FAFD
:106770003060FFF770BB1B6800934FF400321123A9
:106780002846FFF72CFB0024FFF765BB002840F0EC
:106790000D81090141F06F0110234FF4F812C9B2C5
:1067A0002846FFF796FA3060FFF755BB20278F4049
:1067B0007FB247F014085FFA88F878B94146284656
:1067C000FFF778FA41057FF560AC47F01101C9B2D7
:1067D0002846FFF76FFA3060FFF73DBB47F0110125
:1067E0001A68C9B22846FFF781FA3368003318BF28
:1067F000012300934FF480620A2341462846FFF7A5
:10680000EEFA0024FFF727BB2021A94041F0110137
:10681000C9B228B92846FFF74DFA3060FFF71BBB15
:106820001A682846FFF762FA0024FFF714BB090133
:1068300041F06C01C9B240B90D234FF40052284613
:10684000FFF747FA3060FFF706BB1B6800934FF471
:1068500000520D232846FFF7C2FA0024FFF7FBBAC7
:10686000090141F06C01C9B240B914234FF4700220
:106870002846FFF72EFA3060FFF7EDBA1B68009349
:106880004FF4700214232846FFF7A9FA0024FFF7FB
:10689000E2BA002840F08D80090141F06F01034603
:1068A00040F2FF32C9B22846FFF713FA3060FFF713
:1068B000D2BA2021A94041F01901C9B228B928460D
:1068C000FFF7F8F93060FFF7C6BA1A682846FFF7F5
:1068D0000DFA0024FFF7BFBA2021A94041F01A01A8
:1068E000C9B228B92846FFF7E5F93060FFF7B3BA17
:1068F0001A682846FFF7FAF90024FFF7ACBAC8B9BE
:10690000012D01460AD0FFF7D5F900F01800A0F1DB
:106910001002504250413060FFF79DBA2846FFF701
:10692000C9F900F06000A0F12003584258413060DE
:10693000FFF791BA012D4FF0000112D00846FFF782
:10694000B9F9336820F0180243B142F01002002177
:106950000846FFF7CBF90024FFF77DBA42F00802A2
:10696000F5E72846FFF7A6F9336820F0600243B147
:1069700042F0200200210120FFF7B8F90024FFF7C0
:106980006ABA42F04002F5E70824FFF764BA04242B
:10699000FFF761BA0424FFF75EBA0424FFF75BBA7D
:1069A0000424FFF758BA0424FFF755BA0424FFF76C
:1069B00052BA0424FFF74FBA07B5019201AB024661
:1069C0000120FFF729FA03B05DF804FB13460246E5
:1069D0000020FFF721BA01480CF038BF2037FF1F15
:1069E000012838B5144613D045B21DB102281CD079
:1069F000042038BD114B124ADB6824681B68D2F8AA
:106A0000BC021CB15B6998470020F2E79B69FAE77A
:106A10000A4B0B4ADB68D2F8B4021B685B6A9847E2
:106A2000003018BF01202060EEE7044B044ADB6809
:106A3000D2F8B8021B685B6AF1E700BFD89D02007C
:106A40002037FF1F022804BF0C4B93F8F00038B921
:106A50000B4BDB681B685B690A4AD2F8B002184727
:106A6000012809D1054B93F8F030012B04D1044BD8
:106A7000DB681B689B69EFE7704700BF885EFF1FFC
:106A8000D89D02002037FF1F70B50020FFF7DAFF06
:106A9000134B144CDD68D4F8B0022B689B68984700
:106AA0002B68D4F8B4029B6898472B68D4F8B802D6
:106AB0009B6898472B68D4F8C8029B6898472B6856
:106AC000D4F8C0029B6898472B68D4F8C4029B682E
:106AD00098472B68D4F8BC029B68BDE87040184703
:106AE000D89D02002037FF1F08B522210020FFF7A4
:106AF000E1F848B942210120FFF7DCF820B903484A
:106B0000BDE808400CF08BBE002008BD2037FF1FF9
:106B1000012938B505460C460FD1084B102200213B
:106B20000CF0D0FD2846054B214618220CF0CAFD7A
:106B30000348BDE838400CF03FBE38BDC80405002E
:106B40002037FF1F012810B40C4607D8054BD3F897
:106B5000CC3220469B6810BC11461847002010BC60
:106B6000704700BF2037FF1F2DE9F0415F4C604D9B
:106B7000604BA169C5F8AC128CB00127CDE9007358
:106B80005D4ADFF8DC81002328460CF0EBFD5B4911
:106B900028460CF040FED8F80C60736803F5847248
:106BA000C5F8B42203F59472C5F8B82203F57272E1
:106BB000C5F8BC2203F57A7203F16800C5F8C0225B
:106BC00003F5816203F58563C5F8C8323368C5F8FB
:106BD000C422DB68C5F8B00298473368D5F8BC0218
:106BE000DB6898473368D5F8BC029B6998473368DF
:106BF000D5F8B4021B6998473368D5F8B8021B6909
:106C000098473368D5F8C8021B6998473368D5F8A8
:106C1000C0021B6998473368D5F8C4021B699847BE
:106C20007368D8F81020C5F8CC2203F5327353608E
:106C3000334B029303F19F2303F56A035633039307
:106C4000304A314B3148CDE90423314B6FF080613C
:106C5000CDE90613A3F1D943A3F59113A3F227239A
:106C600008932C4B02AACDE9090300214FF4774386
:106C70002846ADF82C300CF022FF02AA39462846EF
:106C80000CF01DFFA369244AC3F80422234A1F8085
:106C9000C3F80822224B6362224B2362224BE3613A
:106CA000224BA362224BE363224BA363224BE3629A
:106CB000224B2363224BE364224BA364224BA36544
:106CC000224B6365224B2365224B6366224B23666E
:106CD000022323753225DE23C4E9033538461F4BD2
:106CE000E365FFF7AFFE0CB0BDE8F081885EFF1FE3
:106CF0002037FF1F0024F400B4950200116B01003F
:106D000054B5AAAA2929492422421010224240003F
:106D10007D77BBB580FFFF56E96A0100D7690100A6
:106D2000775D0100DD5D0100D95D0100D55D0100E9
:106D3000CD690100B9690100015D0100555D0100E7
:106D4000FD5C0100C55C0100A95C0100E169010076
:106D5000815C0100456A01009D5C0100896A0100B7
:106D6000D89D020001289FBF044B03EB8003002045
:106D7000DB6894BF0B600820704700BFFC39FF1F21
:106D8000014B00229A607047885EFF1F38B5064CA1
:106D90000546014620460DF02BF829462046BDE861
:106DA00038400DF025B800BFFC39FF1F10B503486F
:106DB00014460CF0AEFF206010BD00BFFC39FF1F71
:106DC00001480CF098BF00BFFC39FF1F0129F8B53E
:106DD00004461E4600F253861C2A00F0CD825ED87F
:106DE0000C2A00F0A5812CD8052A00F0268114D8A1
:106DF000022A00F0D78008D8002A00F0AF80012ACC
:106E000000F0BE8004242046F8BD032A00F0DF8095
:106E1000042A00F0F0800424F5E7082A00F05881E5
:106E200007D8062A00F01B81072A00F035810424C8
:106E3000E9E70A2A00F05C810B2A00F0698104244A
:106E4000E1E7122A00F01A8213D80F2A00F0DE813F
:106E500007D80D2A00F09A810E2A00F0C58104247B
:106E6000D1E7102A00F0E681112A00F0F581042410
:106E7000C9E7152A00F0388207D8132A00F01082DB
:106E8000142A00F01F820424BDE7172A00F0508264
:106E9000C0F03C82182A00F05D820424B3E7AB2ADC
:106EA00000F03D842BD8A52A00F0358313D8A22A00
:106EB00000F0DA8207D81D2A00F07A828C2A00F0CE
:106EC000808204249FE7A32A00F0EA82A42A00F02B
:106ED0000383042497E7A82A00F0C88307D8A62ACA
:106EE00000F06283A72A00F0A48304248BE7A92A78
:106EF00000F0D983AA2A00F0F483042483E7B52A9A
:106F000000F0BB8413D8AE2A00F0628407D8AC2A04
:106F100000F02384AD2A00F03D84042473E7B32AF3
:106F200000F07E84B42A00F0998404246BE7CE2A12
:106F300000F00B8507D8B62A00F0D584B82A00F0F7
:106F4000E68404245FE7D22A00F02585D32A00F0E6
:106F50003685D12A00F00885042454E7202303FA5B
:106F600001F141F00D01C9B220B9B1480CF0D1FED8
:106F7000306048E73268AE480CF0BDFE002442E7BE
:106F8000202303FA01F141F00101C9B220B9A84858
:106F90000CF0BFFE306036E73268A5480CF0ABFE5F
:106FA000002430E7202303FA01F141F00701C9B2C0
:106FB00020B99F480CF0ADFE306024E732689C4851
:106FC000002AB8BF52420CF096FE00241BE70028AE
:106FD00040F05885202303FA01F141F00201C9B2C3
:106FE00093480CF096FE10F4000318BF4FF07F4357
:106FF0001843306007E78E4F8D003D4418B9D5F82F
:1070000098323360FFE61B682026002B06FA01F653
:10701000B8BF5B42F1B23846C5F898320CF079FE41
:107020000446002840F0318546F00701D5F8982243
:10703000C9B238460CF05FFEE5E6202303FA01F101
:1070400041F00601C9B220B979480CF062FE306007
:10705000D9E6326876480CF04EFE0024D3E62025AF
:107060008D4045F01005EDB2294671482CB90CF061
:1070700050FEC0F304203060C5E60CF04AFE3368D1
:107080001B0203F4F85320F4F8521A4329466848C7
:107090000CF031FE0024B6E620258D4045F01005A9
:1070A000EDB2294662482CB90CF033FE00F01F0007
:1070B0003060A8E60CF02DFE336820F01F0203F0CC
:1070C0001F031A4329465A480CF015FE00249AE67D
:1070D000002840F0DD84202303FA01F141F015017E
:1070E000C9B253480CF015FEC0F3402030608AE668
:1070F000002840F0D084202303FA01F141F015016B
:10710000C9B24B480CF005FEC0F3400030607AE68F
:10711000002840F0C384202303FA01F141F0150157
:10712000C9B243480CF0F5FD00F0010030606AE69A
:1071300020258D4045F01405EDB229463C482CB978
:107140000CF0E7FDC0F3400030605CE60CF0E1FDC0
:107150003368002BCCBF0223002320F002021A4325
:10716000294633480CF0C7FD294631480CF0D1FDC3
:107170003368022B20F008020CBF082300231A43B7
:1071800029462B480CF0B7FD00243CE620258D4015
:1071900045F01405EDB2294625482CB90CF0B9FD8F
:1071A00000F0010030602EE60CF0B3FD326820F0F4
:1071B0000100002AD4BF024640F0010229461C48C3
:1071C0000CF099FD29461A480CF0A3FD3368022BF8
:1071D00020F004020CBF042300231A43294614485C
:1071E0000CF089FD00240EE6202303FA01F141F0A2
:1071F0001401C9B220B90E480CF08BFD306002E6D4
:1072000032680B480CF077FD0024FCE5202303FADC
:1072100001F141F00401C9B220B905480CF079FD33
:107220003060F0E5326802480CF065FD0024EAE5C4
:10723000FC39FF1F202303FA01F141F00501C9B217
:1072400020B9AC480CF065FD3060DCE53268A94837
:107250000CF051FD0024D6E5202303FA01F141F0A2
:107260000801C9B220B9A3480CF053FD3060CAE54B
:107270003268A0480CF03FFD0024C4E5202303FA47
:1072800001F141F00A01C9B220B99A480CF041FD60
:107290003060B8E5326897480CF02DFD0024B2E567
:1072A000202303FA01F141F00301C9B220B991484A
:1072B0000CF02FFD3060A6E532688E480CF01BFD07
:1072C0000024A0E5202303FA01F141F00B01C9B22B
:1072D00020B988480CF01DFD306094E5326885487F
:1072E0000CF009FD00248EE5202303FA01F141F0A2
:1072F0000C01C9B220B97F480CF00BFD306082E56B
:1073000032687C480CF0F7FC00247CE5202303FA6B
:1073100001F141F01101C9B220B976480CF0F9FC35
:10732000306070E5326873480CF0E5FC00246AE5D3
:10733000202303FA01F141F01201C9B220B96D48CE
:107340000CF0E7FC30605EE532686A480CF0D3FC74
:10735000002458E5202303FA01F141F01301C9B2DA
:1073600020B964480CF0D5FC30604CE532686148C7
:107370000CF0C1FC002446E5090141F06C05EDB2BA
:1073800029465C482CB90CF0C4FCC0F38040306046
:1073900039E50CF0BEFC33689B0403F4802320F431
:1073A00080221A43294653480CF0A5FC00242AE504
:1073B000002840F076834F4B03EB8101CB683360AC
:1073C00021E570B9090141F06C0101F0FC01494867
:1073D0000CF09FFC4FF4807300F00F00034133600A
:1073E00011E51B68102B39D00FDC022B32D006DCE4
:1073F000012B18D04FF0FF333360002403E5042B3A
:107400002AD0082BF6D105230EE0402B28D003DC30
:10741000202BEFD1032307E0802B23D0B3F5807F0F
:10742000E8D1002300E00823090141F06C04E4B234
:10743000214633602F480CF06CFC33681B0603F0C8
:10744000706320F0706221461A432A480CF053FC06
:107450000024D8E40723E7E70623E5E70423E3E76E
:107460000223E1E70123DFE7090141F06C05EDB2FA
:10747000294620482CB90CF04CFCC0F3C1303060D8
:10748000C1E40CF046FC3368DB0303F4C03320F4A2
:10749000C0321A43294617480CF02DFC0024B2E4F0
:1074A000090141F06C05EDB2294612482CB90CF0E7
:1074B00030FCC0F340303060A5E40CF02AFC3368A7
:1074C0005B0303F4005320F400521A432946094891
:1074D0000CF011FC002496E4090141F06C05EDB2BA
:1074E0002946044844B90CF014FCC0F30030306065
:1074F00089E400BFFC39FF1F0CF00BFC33681B0351
:1075000003F4805320F480521A432946C3480CF0F8
:10751000F2FB002477E4090141F06C05EDB2294645
:10752000BE480CF0F6FB2946C0F38037BB486CB967
:107530002FB10CF0EEFBC0F3C310306063E40CF02D
:10754000E8FBC0F3021030603C465CE477B10CF01D
:10755000E0FB3368DB0103F4F06320F4F0621A43CC
:107560002946AE480CF0C7FB00244CE40CF0D1FBDC
:107570003268120220F4006002F4006202432946DD
:10758000A6480CF0B8FB2946A4480CF0C2FB3368AF
:107590001B0103F0700320F070021A4329469F4834
:1075A0000CF0A9FB3C462EE4090141F06C05EDB25C
:1075B00029469A480CF0ADFB2946C0F3803797481E
:1075C000B4B92FB10CF0A5FBC0F3021030601AE47F
:1075D0000CF09FFBC0F3C310306029468F480CF0BD
:1075E00098FB3368000A00F00800034333600AE4A4
:1075F0007FB10CF08EFB33681B0103F0700320F0A9
:1076000070021A43294685480CF075FB0024FFF7E9
:10761000FABB0CF07EFB3368DB0103F4F06320F46B
:10762000F0621A4329467D480CF065FB3C46FFF7A3
:10763000EABB090141F06C05EDB22946774834B93F
:107640000CF067FB00F00F003060FFF7DCBB0CF0C4
:1076500060FB336820F00F0203F00F031A43294642
:107660006E480CF048FB0024FFF7CDBB090141F048
:107670006D05EDB22946694834B90CF04AFBC0F3F8
:10768000C0303060FFF7BFBB0CF043FB3368DB0357
:107690009BB220F400421A43294660480CF02BFBB1
:1076A0000024FFF7B0BB090141F06D05EDB229469A
:1076B0005A4834B90CF02DFBC0F341303060FFF76D
:1076C000A2BB0CF026FB33685B0303F4C04320F439
:1076D000C0421A43294651480CF00DFB0024FFF725
:1076E00092BB090141F06D05EDB229464B4834B912
:1076F0000CF00FFBC0F303203060FFF784BB0CF0ED
:1077000008FB33681B0203F4706320F470621A43B1
:10771000294642480CF0EFFA0024FFF774BB090138
:1077200041F06D05EDB229463C4834B90CF0F1FA50
:10773000C0F341103060FFF766BB0CF0EAFA336823
:107740005B0103F0600320F060021A4329463348CE
:107750000CF0D1FA0024FFF756BB090141F06D058A
:10776000EDB229462D4834B90CF0D3FA00F00F00E1
:107770003060FFF748BB0CF0CCFA336820F00F0202
:1077800003F00F031A43294624480CF0B4FA0024EE
:10779000FFF739BB090141F06D05EDB229461F48DD
:1077A00034B90CF0B6FAC0F300603060FFF72BBBC1
:1077B0000CF0AFFA33681B0603F0807320F0807280
:1077C0001A43294615480CF096FA0024FFF71BBB14
:1077D000090141F06D05EDB2294610486CB90CF075
:1077E00098FA001400F07F0310F0400018BF6FF00B
:1077F0007F0018433060FFF706BB0CF08AFA33684D
:107800001B0403F4FE0320F4FE021A432946034836
:107810000CF071FA0024FFF7F6BA00BFFC39FF1F25
:10782000090141F06C05EDB22946A24834B90CF0CB
:1078300070FAC0F340403060FFF7E5BA0CF069FA27
:1078400033685B0403F4003320F400321A43294602
:1078500098480CF050FA0024FFF7D5BA002840F001
:107860002381090141F06F01C9B292480CF051FA2D
:10787000C0F304403060FFF7C6BA202505FA01F1D5
:107880004DB245F01407FFB298B9394689480CF05B
:1078900040FA10F4806008D045F01101C9B2854863
:1078A0000CF037FA3060FFF7AEBA30600446FFF7ED
:1078B000AABA45F011011A687E48C9B20CF01BFA49
:1078C00039467C480CF025FA3368002B20F480629E
:1078D00018BF4FF480631A43394676480CF00BFA10
:1078E0000024FFF790BA202303FA01F141F01101BF
:1078F000C9B228B96F480CF00CFA3060FFF783BAB0
:1079000032686C480CF0F7F90024FFF77CBA0901E3
:1079100041F06C05EDB22946664834B90CF0F9F92E
:10792000C0F340303060FFF76EBA0CF0F2F9336804
:107930005B0303F4005320F400521A4329465D48C8
:107940000CF0D9F90024FFF75EBA002840F0AF80B0
:10795000090141F06F01C9B256480CF0DAF9C0F3E1
:1079600009003060FFF74FBA20258D4045F019051A
:10797000EDB229464F4824B90CF0CBF93060FFF73F
:1079800042BA0CF0C6F932684A4829460CF0B3F9FD
:107990000024FFF738BA202303FA01F141F01A015D
:1079A000C9B228B943480CF0B4F93060FFF72BBADC
:1079B000326840480CF09FF90024FFF724BAC8B998
:1079C000012901463B480AD00CF0A3F900F0180049
:1079D000A0F11002504250413060FFF714BA0CF091
:1079E00098F900F06000A0F120035842584130603F
:1079F000FFF709BA01292F484FF000011FD00CF002
:107A000088F93368002B0CBF0823002320F00802FC
:107A10001A43002127480CF06EF9002125480CF08C
:107A200078F93368002B20F0100218BF10231A4396
:107A3000002120480CF05FF90024FFF7E4B90CF0B6
:107A400068F93368002B18BF202320F020021A4366
:107A5000002118480CF04FF9002116480CF059F994
:107A60003368002B20F040020CBF402300231A4350
:107A7000002110480CF03FF90024FFF7C4B9082496
:107A8000FFF7C1B90424FFF7BEB90024FFF7BBB963
:107A90000424FFF7B8B90424FFF7B5B90424FFF7AD
:107AA000B2B90424FFF7AFB90424FFF7ACB904243A
:107AB000FFF7A9B9FC39FF1F07B5019201AB0246D8
:107AC0000120FFF783F903B05DF804FB134602467B
:107AD0000020FFF77BB910B50446054800EB84028F
:107AE0000B46D2F8982221460CF06FFA002010BD08
:107AF000FC39FF1F10B50446054800EB84030A4615
:107B0000D3F8983221460CF042FA002010BD00BF95
:107B1000FC39FF1F08B5014602480CF035FA002079
:107B200008BD00BFFC39FF1F08B50A4601460248E0
:107B30000CF027FA002008BDFC39FF1F08B50A46E3
:107B4000014602480CF01BFA002008BDFC39FF1F5B
:107B500008B50A46014602480CF0F3F9002008BDBA
:107B6000FC39FF1F01480CF0D4B900BFFC39FF1FDE
:107B7000012838B5144613D045B21DB102281CD0D7
:107B8000042038BD114B124ADB6824681B68D2F808
:107B9000AC021CB15B6998470020F2E79B69FAE7E9
:107BA0000A4B0B4ADB68D2F8A4021B685B6A984751
:107BB000003018BF01202060EEE7044B044ADB6868
:107BC000D2F8A8021B685B6AF1E700BFD89D0200EB
:107BD000FC39FF1F022804BF0C4B93F8F00038B9A2
:107BE0000B4BDB681B685B690A4AD2F8A002184796
:107BF000012809D1054B93F8F030012B04D1044B37
:107C0000DB681B689B69EFE7704700BF885EFF1F5A
:107C1000D89D0200FC39FF1F70B50020FFF7DAFF86
:107C2000134B144CDD68D4F8A0022B689B6898476E
:107C30002B68D4F8A4029B6898472B68D4F8A80254
:107C40009B6898472B68D4F8B8029B6898472B68C4
:107C5000D4F8B0029B6898472B68D4F8B4029B68AC
:107C600098472B68D4F8AC029B68BDE87040184771
:107C7000D89D0200FC39FF1F08B5222107480CF0EF
:107C800048F848B9422105480CF043F820B90348A8
:107C9000BDE808400CF026B9002008BDFC39FF1FE4
:107CA000012910B504460DD1074A10210CF023F824
:107CB0002046054A18210CF01EF80448BDE8104083
:107CC0000CF072B810BD00BFC8040500FC39FF1FDE
:107CD000034BD3F8BC320846DB681146184700BF97
:107CE000FC39FF1FF8B54A4C4A4DA2694A4B4B4F2D
:107CF000284600210CF035F8494928460CF01DF9BA
:107D0000FE68736803F58472C5F8A42203F59472C3
:107D1000C5F8A82203F57272C5F8AC2203F57A7291
:107D200003F16800C5F8B02203F5816203F58563AD
:107D3000C5F8B8323368C5F8B422DB68C5F8A002CC
:107D400098473368D5F8AC02DB6898473368D5F8B4
:107D5000AC029B6998473368D5F8A4021B69984721
:107D60003368D5F8A8021B6998473368D5F8B8027C
:107D70001B6998473368D5F8B0021B699847336888
:107D8000D5F8B4021B69984773683A69C5F8BC22F4
:107D900003F532735360A369224AC3F80422224ACE
:107DA000C3F8082201221A80204B6362204B236211
:107DB000204BE361204BA362204BE363204BA36382
:107DC000204BE362204B2363204BE364204BA364EE
:107DD000204BA365204B6365204B2365204B6366D6
:107DE000204B236632224FF48C73C4E903321E4BBE
:107DF000E3652B680220D3F8A020D3F8203120754A
:107E0000C5F89822C5F89C32BDE8F840E2E600BF0C
:107E1000885EFF1FFC39FF1FB4970200D89D020047
:107E2000A17C0100797C0100657B0100517B010090
:107E30003D7B0100297B0100157B0100CD7A01000B
:107E4000B97A0100F57A0100D77A0100C16D01000D
:107E5000AD6D01008D6D0100717B0100656D01004C
:107E6000D57B0100816D0100197C010018B9034B1D
:107E70005B680B6070470820704700BFC83CFF1F5D
:107E8000014B00229A607047885EFF1F0428F8B5F6
:107E9000144672D00AD801283DD0A0B102285AD089
:107EA00003280CBF002404242046F8BD062800F057
:107EB0009180C0F08380072800F09480FC2800F0B7
:107EC0009D800424F0E7126832F0030340F0A7809D
:107ED000544B554DDE68D5F894023368D2070BD564
:107EE0001B69984724683268D5F8900214F00204A0
:107EF00009D0136998472CE0DB6898473368D5F8B8
:107F000094029B69EDE7D36898473368D5F89002EF
:107F10009B699847C8E7126844F620639A427EDC62
:107F2000414BD3F8B4023F4BDB6842F210711B683F
:107F30008A42CCBF5B699B699847226842F2117301
:107F400092FBF3F103FB1121384B89B29B680020AF
:107F500098470024A8E7334B1468DD68D5E9003062
:107F600000F5F4703CB1DB689847D5E900309B69B7
:107F700000F5F470BEE79B68CBE72A4B2A4EDF681A
:107F800015683B68D6F8A0024DB1012D11D01B69D0
:107F900098473B68D6F8A0025B6A984707E0DB6821
:107FA00098473B689B69D6F8A0029847284620600E
:107FB000CFE7DB6898473B685B69F4E7194B1A4ADF
:107FC000DB68D2F8AC021B685B6A9847003018BFC8
:107FD0000120ECE7134B144ADB68D2F8B0021B68AF
:107FE0005B6AF2E7104B1268D3F8A8020D4BDB680E
:107FF0001B68012A0CBF5B699B697BE7094B0A4D33
:10800000DE6814683368D5F8A00234B1DB6898479D
:108010003368D5F8A0029B696CE71B6979E71024E7
:1080200042E700BFD89D0200C83CFF1FE00AFF1FC7
:10803000224B70B5DD68224C2B68D4F898029B69FE
:1080400098472B68D4F8B8029B6898472B68D4F8F7
:10805000B4029B6898472B68D4F89C029B689847A9
:108060002B68D4F8A0029B6898472B68D4F8A40228
:108070009B6898472B68D4F890029B6898472B68B8
:10808000D4F894029B6898472B68D4F8AC029B689C
:1080900098472B68D4F8B0029B6898472B68D4F8AF
:1080A000A8029B6898472B68D4F898029B68984769
:1080B000044BBDE870405B68184700BFD89D0200C4
:1080C000C83CFF1FE00AFF1F01480BF0C8BF00BFFC
:1080D000C83CFF1F014601480CF071B8C83CFF1FA7
:1080E00010B5034814460BF0C8FF206010BD00BF58
:1080F000C83CFF1FF8B506461D460C46002940F057
:1081000081868C2A00F0E18279D80E2A00F0D08195
:108110003CD8062A00F041811BD8022A00F0FC80DE
:1081200008D8002A00F0DA80012A00F0E680042452
:108130002046F8BD042A00F00D8140F2FB800028A3
:1081400040F024812621C1480BF097FF3446286077
:10815000EEE70A2A00F05D8107D8072A00F0358192
:10816000082A00F04A810424E2E70C2A00F070811A
:1081700040F25E813421B548002E40F086810BF03C
:108180007CFF00F0010028603446D1E7152A00F09A
:10819000EE811AD8112A00F0B78107D80F2A00F013
:1081A0009581102A00F0A1810424C1E7132A00F070
:1081B000C88140F2B781002840F0D2812B21A3482A
:1081C0000BF05BFF34462860B2E71C2A00F02882DF
:1081D0000AD8182A00F0FC811B2A00F00882172A0E
:1081E00000F0D3810424A3E7212A00F03982222A57
:1081F00000F050821D2A00F02B82042498E7B32A55
:1082000000F04D8436D8A82A00F087831CD8A42A11
:1082100000F0DD8207D8A22A00F0A782A32A00F08E
:10822000BD82042484E7A62A00F0278340F2E78277
:108230006C218648002E40F062830BF01EFF00F098
:108240000F002860344673E7AB2A00F0B48307D8E8
:10825000A92A00F07A83AA2A00F09283042467E70F
:10826000AD2A00F0DF83C0F0C083AE2A00F0F583B2
:1082700004245DE7BB2A00F0F98415D8B62A00F083
:10828000738407D8B42A00F02484B52A00F02E8421
:1082900004244DE7B92A00F0A98400F2C284B82A68
:1082A00000F08984042443E7CC2A00F063850AD8CF
:1082B000BF2A00F01A85C02A00F03C85BC2A00F0D5
:1082C000FD84042434E7D12A00F07A85D22A00F014
:1082D0008885CE2A00F06885042429E730B92D214D
:1082E0005A480BF0CAFE3446286021E71A685748FE
:1082F0002D210BF0B4FE00241AE730B92121534898
:108300000BF0BBFE3446286012E71A684F48212163
:108310000BF0A5FE00240BE730B927214B480BF0EA
:10832000ACFE3446286003E71A68484827210BF062
:1083300096FEFDE6002840F06885222143480BF0B8
:108340009CFE10F4000318BF4FF07F4318432860D1
:108350003446EDE63D4F20B9D7F8BC322B600446D9
:10836000E6E61B68002BB8BF5B4220213846C7F801
:10837000BC320BF082FE0446002840F04985D7F855
:10838000BC22272138460BF06AFED1E61A682F4836
:1083900026210BF064FE0024CAE610212B4836B9D2
:1083A0000BF06BFEC0F3042028603446C0E60BF0EF
:1083B00064FE2B681B0203F4F85320F4F8521A43AE
:1083C000102122480BF04BFEB2E610211F4836B9AF
:1083D0000BF053FE00F01F0028603446A8E60BF0B7
:1083E0004CFE2B6820F01F0203F01F031A431021DC
:1083F00016480BF034FE00249AE6002840F00B8566
:10840000352112480BF039FEC0F340202860344675
:108410008EE6002840F0028535210C480BF02DFE39
:1084200010F0020F0CBF012300232B6034467FE6BF
:10843000002840F0F684352104480BF01EFEC043AE
:1084400000F001002860344672E600BFC83CFF1F00
:108450003421A44836B90BF010FEC0F34000286068
:10846000344665E60BF009FE2C6834B940F0020290
:1084700034219C480BF0F3FD5AE620F0020234212F
:1084800098480BF0ECFD002452E60BF0F6FD2C684A
:1084900034B940F00102342192480BF0E0FD47E688
:1084A00020F0010234218F480BF0D9FD00243FE673
:1084B00030B934218B480BF0E0FD3446286037E6B4
:1084C0001A68884834210BF0CAFD31E630B92421FE
:1084D00084480BF0D2FD3446286029E61A688148AA
:1084E00024210BF0BCFD002422E630B925217D4873
:1084F0000BF0C3FD344628601AE61A687948252136
:108500000BF0ADFD002413E630B9282175480BF0BF
:10851000B4FD344628600BE61A68724828210BF037
:108520009EFD05E630B92A216E480BF0A6FD3446C3
:108530002860FDE51A686B482A210BF090FD0024A5
:10854000F6E530B9232167480BF097FD34462860E3
:10855000EEE51A68634823210BF081FD0024E7E56E
:108560001A6860482B210BF07AFD0024E0E530B951
:108570002C215C480BF081FD34462860D8E51A6850
:1085800058482C210BF06BFDD2E5574C70B91521E2
:1085900054480BF072FD30B14FF08073B3FBF0F331
:1085A0009C4228BF1C462C600024C1E51B686BB1AF
:1085B0004FF0807292FBF3F2A242A8BF22462A60DB
:1085C000152148480BF04BFD0024B1E52246F6E7A3
:1085D00030B9332143480BF050FD34462860A7E5FD
:1085E0001A68404833210BF03AFD0024A0E56C21C5
:1085F0003C4836B90BF041FDC0F3C040286034461A
:1086000096E50BF03AFD2B68DB0403F4002320F41D
:1086100000221A436C2133480BF021FD002487E52A
:108620006C21304836B90BF028FDC0F3804028603B
:1086300034467DE50BF021FD2B689B0403F4802379
:1086400020F480221A436C2126480BF008FD6FE5C8
:10865000002840F0E983234B5B682B60044667E504
:1086600040B901461F480BF008FD00F001002860EA
:1086700034465DE500211B480BF0FFFC2B6820F021
:10868000010203F001031A43002116480BF0E7FC36
:1086900000244DE540B9014612480BF0EEFCC0F352
:1086A00040002860344643E500210E480BF0E5FC0D
:1086B0002B685B0003F0020320F002021A43002142
:1086C00008480BF0CCFC002432E578B96C21054851
:1086D0000BF0D3FC4FF48073C0F3036003412B60B5
:1086E000344625E5C83CFF1FFFFF0F001B68102B19
:1086F00035D00FDC022B2ED006DC012B18D04FF02A
:10870000FF332B60102413E5042B26D0082BF6D161
:1087100005230EE0402B24D003DC202BEFD10323D4
:1087200007E0802B1FD0B3F5807FE8D1296001E0FE
:1087300008232B606C21BA480BF09FFC2B681B06AA
:1087400003F0706320F070621A436C21B4480BF0A0
:1087500086FC0024ECE40723EBE70623E9E7042387
:10876000E7E70223E5E70123E3E76C21AC4836B9EC
:108770000BF083FCC0F3C13028603446D8E40BF022
:108780007CFC2B68DB0303F4C03320F4C0321A43B3
:108790006C21A3480BF063FC0024C9E46C21A048C1
:1087A00036B90BF06AFCC0F3803028603446BFE471
:1087B0000BF063FC2B689B0303F4804320F480429E
:1087C0001A436C2196480BF04AFC0024B0E46C215B
:1087D000934836B90BF051FCC0F3003028603446A2
:1087E000A6E40BF04AFC2B681B0303F4805320F42F
:1087F00080521A436C218A480BF031FC98E46C21BA
:1088000087480BF03AFC00F480449EB944B16C21D7
:1088100083480BF032FCC0F3C3102860344687E471
:10882000C0F3021300F40060034314BF08230023C5
:108830002B607DE484B16C2179480BF01EFC2B6821
:10884000DB0103F4F06320F4F0621A436C217448F6
:108850000BF005FC00246BE42A6811074CBF40F4C0
:10886000006020F40060120120F07000D2B20243D8
:108870006C216B480BF0F3FB5AE46C2168480BF059
:10888000FCFBAEB910F4804408D06C2164480BF0B6
:10889000F4FBC0F302102860344649E4C0F3C3136C
:1088A00000F40060034314BF082300232B603FE45F
:1088B0006C215B480BF0E1FB10F480444FF06C013D
:1088C00057480ED00BF0D9FB2B681B0103F0700347
:1088D00020F070021A436C2151480BF0C0FB0024B9
:1088E00026E40BF0CAFB2B68DB0103F4F06320F4F1
:1088F000F0621A436C214A480BF0B1FB18E40BF00C
:10890000BCFB2B6820F00F0203F00F031A436C210D
:1089100043480BF0A4FB00240AE46D21404836B91B
:108920000BF0ABFBC0F3C0302860344600E40BF022
:10893000A4FB2B68DB039BB220F400421A436D2199
:1089400037480BF08CFBFFF7F3BB6D2134483EB981
:108950000BF093FBC0F3413028603446FFF7E8BBCF
:108960000BF08BFB2B685B0303F4C04320F4C04285
:108970001A436D212A480BF072FB0024FFF7D8BB85
:108980006D2127483EB90BF078FBC0F30320286027
:108990003446FFF7CDBB0BF070FB2B681B0203F4D2
:1089A000706320F470621A436D211D480BF057FB71
:1089B0000024FFF7BDBB6D2119483EB90BF05DFBEC
:1089C000C0F3411028603446FFF7B2BB0BF055FBF3
:1089D0002B685B0103F0600320F060021A436D21F5
:1089E0000F480BF03CFBFFF7A3BB6D210C483EB9D1
:1089F0000BF043FB00F00F0028603446FFF798BBF4
:108A00000BF03BFB2B6820F00F0203F00F031A431F
:108A10006D2103480BF023FB0024FFF789BB00BF47
:108A2000C83CFF1F6D21B6483EB90BF026FBC0F3D2
:108A3000006028603446FFF77BBB0BF01EFB2B6801
:108A40001B0603F0807320F080721A436D21AC483E
:108A50000BF005FB0024FFF76BBB6D21A84876B92E
:108A60000BF00BFB001400F07F0310F0400018BF68
:108A70006FF07F00184328603446FFF759BB0BF0B6
:108A8000FCFA2B681B0403F4FE0320F4FE021A43D5
:108A90006D219B480BF0E3FA0024FFF749BB6C21E2
:108AA00097483EB90BF0E9FAC0F3404028603446DD
:108AB000FFF73EBB0BF0E1FA2B685B0403F40033D5
:108AC00020F400321A436C218D480BF0C8FAFFF7EE
:108AD0002FBB002840F0AB816F2189480BF0CDFA05
:108AE000C0F3044028603446FFF722BB3421844899
:108AF000C6B90BF0C2FA430510D5142180480BF01B
:108B0000BCFA804B30B14FF08072B2FBF0F293426E
:108B100028BF13462B600024FFF70ABB2E603446A3
:108B2000FFF706BB0BF0A9FA2B68002B18BF4FF418
:108B3000806320F480621A43342171480BF08FFA6D
:108B40002968704B71B14FF0807292FBF1F29A423A
:108B5000A8BF1A462A60142169480BF080FA002445
:108B6000FFF7E6BA1A46F5E790B9142164480BF00E
:108B700084FA58B14FF08073B3FBF0F0614B984228
:108B800028BF184628600024FFF7D2BA5D48F9E7ED
:108B90001B6873B15B494FF0807292FBF3F28A421B
:108BA000C8BF0A46142156480BF059FA0024FFF7B3
:108BB000BFBA544AF6E76C2151483EB90BF05DFA52
:108BC000C0F3403028603446FFF7B2BA0BF055FAD4
:108BD0002B685B0303F4005320F400521A436C210A
:108BE00047480BF03CFA0024FFF7A2BA6C21444836
:108BF0003EB90BF042FAC0F3035028603446FFF749
:108C000097BA0BF03AFA2B681B0503F4700320F4B3
:108C100070021A436C213A480BF021FA0024FFF746
:108C200087BA384C78B9132135480BF026FA30B1A1
:108C30004FF08073B3FBF0F39C4228BF1C462C60BE
:108C40000024FFF775BA1B6873B14FF0807292FB76
:108C5000F3F2A242A8BF22462A60132128480BF053
:108C6000FEF90024FFF764BA2246F5E77021244894
:108C70003EB90BF002FAC0F3072028603446FFF734
:108C800057BA0BF0FAF92A68120220F47F4092B228
:108C9000024370211A480BF0E2F9214618480BF004
:108CA000ECF92B68002B20F0040218BF04231A43B0
:108CB000214613480BF0D3F9FFF73ABA7021104858
:108CC00036B90BF0DAF9C0B228603446FFF730BA93
:108CD0000BF0D3F92A7820F0FF00024370210848F6
:108CE0000BF0BDF90024FFF723BA68B970210448DE
:108CF0000BF0C3F9C0F3014028603446FFF718BAFF
:108D0000C83CFF1FFFFF0F001B68032B00F292807F
:108D100070214D480BF0B1F92B681B0403F440336C
:108D200020F440321A43702147480BF098F9002490
:108D3000FFF7FEB948B9702143480BF09EF9C0F324
:108D4000804028603446FFF7F3B91B68012B74D8C4
:108D500070213D480BF091F92B689B0403F48023AC
:108D600020F480221A43702137480BF078F9002450
:108D7000FFF7DEB9702134483EB90BF07EF9C0F33D
:108D8000015028603446FFF7D3B90BF076F92B6811
:108D90001B0503F4401320F440121A4370212A48A3
:108DA0000BF05DF9FFF7C4B9002849D16F212648BF
:108DB0000BF063F9C0F3090028603446FFF7B8B937
:108DC00038B9392120480BF058F934462860FFF7AC
:108DD000AFB91A681C4839210BF041F90024FFF79C
:108DE000A7B938B93A2118480BF047F9344628603A
:108DF000FFF79EB91A6814483A210BF030F90024A5
:108E0000FFF796B90824FFF793B90424FFF790B948
:108E10000024FFF78DB90424FFF78AB90424FFF773
:108E200087B90424FFF784B90424FFF781B9042427
:108E3000FFF77EB91024FFF77BB91024FFF778B94C
:108E40000424FFF775B900BFC83CFF1F07B50192A6
:108E500001AB02460120FFF74DF903B05DF804FBBA
:108E6000134602460020FFF745B908B50348D0F87D
:108E7000BC220BF033FA002008BD00BFC83CFF1F26
:108E800008B50348D0F8BC220BF014FA002008BD46
:108E9000C83CFF1F08B502480BF009FA002008BDC6
:108EA000C83CFF1F08B502480BF0FEF9002008BDC2
:108EB000C83CFF1F08B502480BF0F4F9002008BDBC
:108EC000C83CFF1F08B502480BF0D8F9002008BDC8
:108ED000C83CFF1F01480BF05AB900BFC83CFF1F38
:108EE00038B522210D480D4C0BF0C7F810B92046BB
:108EF0000BF036F90A4BD4F8B402DD682B689B6995
:108F000098472B68D4F890021B6998472B68D4F8CF
:108F100094021B699847012038BD00BFC83CFF1F61
:108F2000D89D0200022804BF0C4B93F8F00038B91A
:108F30000B4BDB681B685B690A4AD2F8980218473A
:108F4000012809D1054B93F8F030012B04D1044BD3
:108F5000DB681B689B69EFE7704700BF885EFF1FF7
:108F6000D89D0200C83CFF1F012908B508D1054A59
:108F700070210BF074F80448BDE808400BF0C6B847
:108F800008BD00BFC8040500C83CFF1F034BD3F851
:108F9000C0320846DB681146184700BFC83CFF1FB7
:108FA00070B5634E634CF5686B6803F16802C4F8F2
:108FB000982203F1A802C4F89C2203F1C802C4F865
:108FC000A02203F59472C4F8902203F5A472C4F8A9
:108FD000942203F5D472C4F8B42203F5E472C4F801
:108FE000B82203F5627203F18800C4F8A82203F5E1
:108FF0006A7203F57273C4F8AC322B68C4F8B022FD
:109000001B69C4F8A40298472B68D4F8A0021B6916
:1090100098472B68D4F89C021B6998472B68D4F8B2
:10902000AC021B6998472B68D4F8B0021B699847BB
:109030002B68D4F8A802DB6898472B68D4F8900214
:109040001B6998472B68D4F894021B6998472B68D2
:10905000D4F89802DB6898472B68D4F8B402DB6830
:1090600098472B68D4F8B802DB6898472B68D4F887
:10907000A8029B6998476B683269C4F8C02203F55F
:10908000327353602C4B2D499A692D48C2F8041253
:109090002C49C2F808120121118058622A4818622E
:1090A0002A48D8612A4898622A48D8632A4898638F
:1090B0002A48D8622A4818632A48D8642A489864FB
:1090C0002A4898652A4858652A4818652A485866E3
:1090D0002A481866197532204FF4F071C3E903105D
:1090E0002749D9652046274B00210AF0EEFF264983
:1090F00020460BF060F823680220D3F8A030C4F8B3
:10910000BC32FFF70FFF2B68D4F8B802DB68984732
:10911000D4F8B8021D4C042343752B681B6898478C
:10912000236898470021A3680846BDE870401847A7
:10913000D89D0200C83CFF1F885EFF1FE18E010022
:10914000C58E0100D58E0100B58E0100A58E0100EF
:10915000958E0100618E01004D8E0100818E01000F
:109160006B8E0100C9800100E1800100D580010003
:109170008D7E01006D7E0100258F0100817E010042
:1091800031800100B4990200698F0100E00AFF1FDD
:1091900018B9034B1B680B6070470820704700BF6D
:1091A000983FFF1F014B00229A607047885EFF1FA7
:1091B000234B70B5DD68234C2B68D4F898029B696B
:1091C00098472B68D4F8A8029B6998472B68D4F875
:1091D000AC029B6998472B68D4F89C029B6898471F
:1091E0002B68D4F8A0029B6898472B68D4F8A40297
:1091F0009B6898472B68D4F890029B6898472B6827
:10920000D4F894029B6898472B68D4F8B0029B6806
:1092100098472B68D4F8B4029B6898472B68D4F819
:1092200098029B6898472B68D4F8A8029B689847D7
:109230002B68D4F8AC029B68BDE87040184700BFAB
:10924000D89D0200983FFF1F024BD3F8B8020BF0E5
:10925000C9B800BF983FFF1F38B5284D00F07F0404
:109260002B1993F80C32DB0705D4D5F8B83203EB91
:109270008404606838BDD5F8BC3200219B68204664
:109280009847D5F8BC3200219B6808469847D5F826
:10929000BC3200219B6808469847D5F8BC320021B3
:1092A0009B6808469847D5F8BC3201219B6800208E
:1092B0009847D5F8BC3200219B6820469847D5F8DE
:1092C000BC3200219B6808469847D5F8BC32002183
:1092D00004029B6808469847D5F8BC320021044335
:1092E0009B6808469847D5F8BC32240204439B6823
:1092F00001210020984724022043BBE7983FFF1F2D
:10930000022804BF0C4B93F8F00038B90B4BDB6814
:109310001B685B690A4AD2F898021847012809D1EC
:10932000054B93F8F030012B04D1044BDB681B682C
:109330009B69EFE7704700BF885EFF1FD89D020062
:10934000983FFF1F012870B506460F4D0F4C07D1FF
:10935000EB6AC4F8C0325B68984784F8C46270BD99
:1093600094F8C432012B03D1D4F8C0329B689847DB
:10937000EB682A695B68C4F8BC2203F5327353605A
:10938000002384F8C432EAE7D89D0200983FFF1F0B
:109390000528F8B50C46154600F0A5801FD8022810
:1093A00069D004D800283ED004242046F8BD032804
:1093B00073D00428F8D1604B604EDF6814683B68B6
:1093C000D6F8A002002C7ED0012C00F087801B690B
:1093D00098473B68D6F8A0025B6A98477BE008286C
:1093E00000F08D8009D80628DED1534B534ADB6844
:1093F000D2F8B4021B685B6A7CE0092800F0888020
:10940000FC28D1D14C4B4D4EDF6814683B68D6F830
:10941000A002002C00F08C80DB6898473B68D6F8EF
:10942000A0029B6916E0126832F0030340F08280CC
:10943000414B424EDF68D6F894023B68D2070BD509
:109440001B6998472C683B68D6F8900214F0020418
:1094500009D01B6998473FE0DB6898473B68D6F81E
:1094600094029B69EDE7DB6898473B68D6F8900269
:109470009B69984799E7304B1468DE68D6E900305D
:1094800000F5F4703CB1DB689847D6E900309B6981
:1094900000F5F470DEE79B68EBE7284BD3F8A802F1
:1094A000254BDB681B6839B1146814F0010401D046
:1094B0005B69CFE79B69DCE75B6A9847003018BFC0
:1094C0000120286071E7DB6898473B689B69D6F804
:1094D000A002984720462860002466E7DB6898478A
:1094E0003B685B69F3E7144B144ADB68D2F8B002BF
:1094F0001B685B6A9847003018BF0120EBE71068D3
:109500000E4B00F0010083F8C502FFF71BFFE3E7F5
:10951000094B1268DC68D4E90030012A00F5F470C8
:1095200004D1DB689847D4E90030B0E79B6891E745
:109530001B699EE7102438E7D89D0200983FFF1F63
:109540007FB52C4B00F07F041A191D4692F80C22AF
:1095500012F0010F06D1D3F8B83203EB840460682F
:1095600004B070BD01220523032101A8ADF8043029
:109570008DF8064006F0FCFDD5F8C0328DF80700E6
:10958000DB699847D5F8C03204215B690DEB010017
:10959000984703F09BF80646D5F8C0321B6A9847F7
:1095A00007281FD9D5F8C03208219B690DEB0100AF
:1095B00098470122072102A89DF80F5006F0D8FD18
:1095C000854214D19DF80830052B10D19DF8093043
:1095D000FF2B0CD19DF80A30A34208D1DDF80B0017
:1095E00000BABDE7304603F081F83228D4D94FF0F5
:1095F000FF30B5E7983FFF1F034A0146D2F8B83263
:1096000000200AF0B6BE00BF983FFF1F024B93F840
:10961000C53203B194E71FE6983FFF1F38B52220FB
:10962000FFF7F4FF094C18B9D4F8B8020AF0D2FEDB
:10963000074BD4F89002DD682B681B6998472B68AC
:10964000D4F894021B699847012038BD983FFF1F4A
:10965000D89D020010B508461446FFF7D7FF2060DA
:1096600010BD2DE9F74F364D9DF8304095F8C56295
:109670009DF8347001F07F0990469A4649F08000C9
:10968000AB46A6B305238DF802008DF80320072111
:1096900001226846ADF800308DF804A08DF8054031
:1096A0008DF8067006F064FDD5F8C0328DF807001D
:1096B000DB6998476D460026DBF8C03215F8010BD0
:1096C000DB6801369847082EF6D1022003F004F833
:1096D00047EA0424DBF8B83244EA0A4403EB890978
:1096E00044EA0864C9F8044003B0BDE8F08FD5F837
:1096F000BC3231469B689847D5F8BC3231469B68EE
:1097000040469847D5F8BC3231469B68504698474A
:10971000D5F8BC3231469B6820469847D5F8BC3214
:1097200001219B68384698474AEA082344EA032403
:10973000D5F8B83247EA042403EB8909D2E700BF21
:10974000983FFF1F07B5D3B20193C2F307230093DD
:10975000C2F30743120EFFF784FF03B05DF804FB6A
:109760000020FFF7EFBF73B50D460646E8B9104C71
:1097700094F8C63243B1D4F8B8322721D3F8A020E8
:10978000FFF7E0FF84F8C66200242A462D2100205E
:10979000FFF7D8FF2046CDE900442346224620218A
:1097A000FFF75FFF204602B070BD0820FBE700BF57
:1097B000983FFF1F38B50C4605462120FFF726FFCE
:1097C0002368C11821602846BDE83840CBE737B58B
:1097D0000D460446C8B90E4B012283F8C62281EA21
:1097E000E172A2EBE1722721FFF7ACFF002DACBFC5
:1097F00001230223CDE900432046234622462021AF
:10980000FFF72FFF204603B030BD0820FBE700BF65
:10981000983FFF1F0021DAE74942D8E7D7E7F8B5BC
:1098200006461D460C46002940F01B86222A00F001
:10983000B38272D80E2A00F0C7813AD8062A00F007
:109840004A811AD8022A00F0FE8008D8002A00F0C7
:10985000DE80012A00F0E98004242046F8BD042AB5
:1098600000F0148140F20381002840F02D81262071
:10987000FFF7CCFE34462860EFE70A2A00F0648147
:1098800007D8072A00F03E81082A00F052810424FC
:10989000E3E70C2A00F0728140F264813420002E4C
:1098A00040F08481FFF7B2FE00F0010028603446EA
:1098B000D3E7152A00F0E18119D8112A00F0AD8113
:1098C00007D80F2A00F08D81102A00F09881042417
:1098D000C3E7132A00F0BC8140F2AC81002840F0BD
:1098E000C5812B20FFF792FE34462860B5E71B2A7E
:1098F00000F0008207D8172A00F0CC81182A00F067
:10990000EB810424A9E71D2A00F02782C0F0098218
:10991000212A00F02A8204249FE7AE2A00F0FE8369
:1099200041D8A72A00F0568321D8A32A00F0AD829F
:1099300007D88C2A00F04782A22A00F08E820424E5
:109940008BE7A52A00F0D08240F2B6826C20FFF7A8
:109950005DFE00F48044002E40F01D83002C00F0DA
:109960000F83000900F070002860344675E7AA2ACA
:1099700000F0788307D8A82A00F04283A92A00F0D3
:109980005683042469E7AC2A00F09F8340F2838366
:109990006D20002E40F0B283FFF738FEC0F3006068
:1099A0002860344659E7BB2A00F09E8415D8B62AB1
:1099B00000F01C8407D8B42A00F0D083B52A00F048
:1099C000D983042449E7B92A00F0508400F268845E
:1099D000B82A00F0318404243FE7CC2A00F0FD844B
:1099E0000AD8BF2A00F0BC84C02A00F0D884BC2A60
:1099F00000F0A084042430E7D12A00F01285D22A96
:109A000000F01F85CE2A00F00185042425E728B93F
:109A10002D20FFF7FBFD344628601EE71A682D2134
:109A20000020FFF78FFE002417E728B92120FFF759
:109A3000EDFD3446286010E71A6821210020FFF769
:109A400081FE002409E728B92720FFF7DFFD34460F
:109A5000286002E71A68002AB8BF52422721204630
:109A6000FFF770FEB34B012283F8C622F5E600280B
:109A700040F0FA842220FFF7C9FD10F4000318BF5C
:109A80004FF07F43184328603446E6E6A94BD3F8ED
:109A9000B82220B9D2F8A0302B600446DDE62B684E
:109AA000002BB8BF5B42C2F8A0302020FFF7AEFD0C
:109AB000044608B10024D0E62A68002AB8BF524202
:109AC0002721FFF73FFEC8E61A6826210020FFF78E
:109AD00039FE0024C1E6102036B9FFF797FDC0F328
:109AE000042028603446B8E6FFF790FD2B681B027F
:109AF00003F4F85320F4F8521A4310212046FFF7DC
:109B000021FEAAE6102036B9FFF780FD00F01F0005
:109B100028603446A1E6FFF779FD2B6820F01F028C
:109B200003F01F031A4310210020FFF70BFE00244F
:109B300093E6002840F09B843520FFF767FDC0F3D3
:109B400040202860344688E6002840F09384352081
:109B5000FFF75CFD10F0020F0CBF012300232B6008
:109B600034467AE6002840F088843520FFF74EFD21
:109B7000C04300F00100286034466EE6342036B958
:109B8000FFF744FDC0F340002860344665E6FFF768
:109B90003DFD2B685B0003F0020320F002021A4334
:109BA00034210020FFF7CEFD002456E6FFF72EFDFE
:109BB0002B6820F0010203F001031A433421002036
:109BC000FFF7C0FD002448E628B93420FFF71EFD4A
:109BD0003446286041E61A6834212046FFF7B2FD7A
:109BE0003BE628B92420FFF711FD3446286034E60F
:109BF0001A6824210020FFF7A5FD00242DE628B9CE
:109C00002520FFF703FD3446286026E61A68252143
:109C10000020FFF797FD00241FE628B92820FFF752
:109C2000F5FC3446286018E61A6828212046FFF71C
:109C300089FD12E628B92A20FFF7E8FC344628609F
:109C40000BE61A682A210020FFF77CFD002404E6B9
:109C500028B92320FFF7DAFC34462860FDE51A68AE
:109C600023210020FFF76EFD0024F6E51A682B2162
:109C70000020FFF767FD0024EFE528B92C20FFF74F
:109C8000C5FC34462860E8E51A682C212046FFF719
:109C900059FDE2E5284C68B91520FFF7B7FC30B153
:109CA0004FF08073B3FBF0F39C4228BF1C462C603E
:109CB0000024D2E51B686BB14FF0807292FBF3F287
:109CC000A242A8BF22462A6015210020FFF73AFDD4
:109CD0000024C2E52246F6E728B93320FFF796FCB8
:109CE00034462860B9E51A6833210020FFF72AFDC1
:109CF0000024B2E56C2036B9FFF788FCC0F3C04001
:109D000028603446A9E5FFF781FC2B68DB0403F4E7
:109D1000002320F400221A436C212046FFF712FD95
:109D20009BE56C2056B9FFF771FCC0F380402860BA
:109D3000344692E5983FFF1FFFFF0F00FFF766FCD8
:109D40002B689B0403F4802320F480221A436C21A7
:109D50000020FFF7F7FC00247FE5002840F0908307
:109D6000BF4B1B682B60044677E530B9FFF74EFC0C
:109D700000F00100286034466FE50020FFF746FC44
:109D80002B6820F0010203F0010300211A4308466A
:109D9000FFF7D8FC002460E530B9FFF737FCC0F3CB
:109DA00040002860344658E50846FFF72FFC2B6832
:109DB0005B0003F0020320F002021A432146204612
:109DC000FFF7C0FC49E550B96C20FFF71FFC4FF4CA
:109DD0008073C0F3036003412B6034463DE51B688C
:109DE000102B34D00FDC022B2DD006DC012B18D029
:109DF0004FF0FF332B6010242FE5042B25D0082BC8
:109E0000F6D105230EE0402B23D003DC202BEFD12D
:109E1000032307E0802B1ED0B3F5807FE8D1002319
:109E200000E008232B606C20FFF7F0FB2B681B067B
:109E300003F0706320F070621A436C210020FFF77A
:109E400081FC002409E50723ECE70623EAE7042365
:109E5000E8E70223E6E70123E4E76C2036B9FFF7E1
